:020000040800F2
:100000000000022085CE0108D5CE0108D5CE01081A
:10001000D5CE0108D5CE0108D5CE010800000000DC
:10002000000000000000000000000000D5CE010824
:10003000D5CE010800000000D5CE0108EB990108DB
:10004000D5CE0108D5CE0108D5CE0108D5CE010800
:10005000D5CE0108D5CE0108E59A0108EB9A010832
:10006000F19A0108F79A0108FD9A0108D5CE010816
:10007000D5CE0108D5CE0108D5CE0108D5CE0108D0
:10008000D5CE0108D5CE0108D5CE0108000000006C
:10009000000000000000000000000000039B0108B9
:1000A0007D880108F58701089188010819880108F1
:1000B0002D8801084188010855880108614401081C
:1000C0006D4401087944010885440108D5CE010832
:1000D000D5CE010825A701083DA7010800000000B2
:1000E000199B0108D5CE010845DF0108000000007A
:1000F000000000000000000000000000D5CE010854
:1001000000000000D5CE010869880108D5CE01089D
:1001100000000000000000000000000000000000DF
:10012000D5CE0108D5CE0108D5CE0108D5CE01081F
:10013000D5CE010800000000000000000000000013
:1001400000000000000000000000000039DF01088E
:10015000D5CE0108D5CE0108D5CE010859A7010892
:10016000914401089D4401080000000000000000C7
:10017000000000000000000000000000000000007F
:1001800000000000D5CE01080000000000000000C3
:08019000D5CE0108D5CE01080F
:1001A000034613F8012B002AFBD1181A01387047B7
:1001B00010F8012B11F8013B012A28BF9A42F7D011
:1001C000D01A70470000000000000000000000008E
:1001D00001F0FF01102A2BDB10F0070F08D010F8F8
:1001E000013B013A8B422DD010F0070F42B3F6D1FC
:1001F000F0B441EA012141EA014122F007047FF015
:1002000000070023F0E80256083C85EA010586EA6B
:10021000010685FA47F5A3FA87F586FA47F6A5FAA7
:1002200087F68EB9EED1F0BC01F0FF0102F00702B3
:1002300032B110F8013B013A83EA010313B1F8D15E
:100240000020704701387047002D06BF354603383F
:10025000073815F0010F07D1013015F4807F02BF78
:10026000013015F4C03F0130F0BC0138704700BFC9
:1002700081F0004102E000BF83F0004330B54FEA57
:1002800041044FEA430594EA050F08BF90EA020FC4
:100290001FBF54EA000C55EA020C7FEA645C7FEA57
:1002A000655C00F0E2804FEA5454D4EB5555B8BF7A
:1002B0006D420CDD2C4480EA020281EA030382EAEB
:1002C000000083EA010180EA020281EA0303362D7D
:1002D00088BF30BD11F0004F4FEA01314FF4801C50
:1002E0004CEA113102D0404261EB410113F0004F62
:1002F0004FEA03334CEA133302D0524263EB430319
:1003000094EA050F00F0A780A4F10104D5F1200EB6
:100310000DDB02FA0EFC22FA05F2801841F1000111
:1003200003FA0EF2801843FA05F359410EE0A5F1E5
:1003300020050EF1200E012A03FA0EFC28BF4CF016
:10034000020C43FA05F3C01851EBE37101F00045CC
:1003500007D54FF0000EDCF1000C7EEB00006EEBD9
:100360000101B1F5801F1BD3B1F5001F0CD3490863
:100370005FEA30004FEA3C0C04F101044FEA4452BA
:1003800012F5800F80F09A80BCF1004F08BF5FEA41
:10039000500C50F1000041EB045141EA050130BD21
:1003A0005FEA4C0C404141EB0101013C28BFB1F533
:1003B000801FE9D291F0000F04BF01460020B1FA7E
:1003C00081F308BF2033A3F10B03B3F120020CDA51
:1003D0000C3208DD02F1140CC2F10C0201FA0CF02F
:1003E00021FA02F10CE002F11402D8BFC2F1200C94
:1003F00001FA02F120FA0CFCDCBF41EA0C0190404A
:10040000E41AA2BF01EB0451294330BD6FEA040492
:100410001F3C1CDA0C340EDC04F11404C4F120027D
:1004200020FA04F001FA02F340EA030021FA04F38F
:1004300045EA030130BDC4F10C04C4F1200220FAE6
:1004400002F001FA04F340EA0300294630BD21FA24
:1004500004F0294630BD94F0000F83F4801306BFEA
:1004600081F480110134013D4EE77FEA645C18BFDE
:100470007FEA655C29D094EA050F08BF90EA020F75
:1004800005D054EA000C04BF1946104630BD91EA6D
:10049000030F1EBF0021002030BD5FEA545C05D170
:1004A0004000494128BF41F0004130BD14F58004AF
:1004B0003CBF01F5801130BD01F0004545F0FE4123
:1004C00041F470014FF0000030BD7FEA645C1ABF58
:1004D000194610467FEA655C1CBF0B46024650EA8F
:1004E000013406BF52EA033591EA030F41F40021BB
:1004F00030BD00BF90F0000F04BF0021704730B541
:100500004FF4806404F132044FF000054FF0000115
:1005100050E700BF90F0000F04BF0021704730B5D6
:100520004FF4806404F1320410F0004548BF4042AB
:100530004FF000013EE700BF42004FEAE2014FEA00
:1005400031014FEA02701FBF12F07F4393F07F4FDB
:1005500081F06051704732F07F4208BF704793F0DE
:100560007F4F04BF41F40021704730B54FF46074F1
:1005700001F0004521F000411CE700BF50EA0102F4
:1005800008BF704730B54FF000050AE050EA01029D
:1005900008BF704730B511F0004502D5404261EB0D
:1005A00041014FF4806404F132045FEA915C3FF44E
:1005B000D8AE4FF003025FEADC0C18BF03325FEAEB
:1005C000DC0C18BF033202EBDC02C2F1200300FA9C
:1005D00003FC20FA02F001FA03FE40EA0E0021FAC1
:1005E00002F11444BDE600BF70B54FF0FF0C4CF4AF
:1005F000E06C1CEA11541DBF1CEA135594EA0C0F61
:1006000095EA0C0F00F0DEF82C4481EA030621EA9B
:100610004C5123EA4C5350EA013518BF52EA0335D6
:1006200041F4801143F4801338D0A0FB02CE4FF088
:100630000005E1FB02E506F00042E0FB03E54FF0B8
:100640000006E1FB03569CF0000F18BF4EF0010EB0
:10065000A4F1FF04B6F5007F64F5407404D25FEAAC
:100660004E0E6D4146EB060642EAC62141EA55515F
:100670004FEAC52040EA5E504FEACE2EB4F1FD0CA1
:1006800088BFBCF5E06F1ED8BEF1004F08BF5FEA1F
:10069000500E50F1000041EB045170BD06F00046D1
:1006A00046EA010140EA020081EA0301B4EB5C047E
:1006B000C2BFD4EB0C0541EA045170BD41F4801176
:1006C0004FF0000E013C00F3AB8014F1360FDEBF9B
:1006D000002001F0004170BDC4F10004203C35DA77
:1006E0000C341BDC04F11404C4F1200500FA05F3FA
:1006F00020FA04F001FA05F240EA020001F000429B
:1007000021F0004110EBD37021FA04F642EB060110
:100710005EEA430E08BF20EAD37070BDC4F10C043A
:10072000C4F1200500FA04F320FA05F001FA04F2FE
:1007300040EA020001F0004110EBD37041F10001EA
:100740005EEA430E08BF20EAD37070BDC4F12005F5
:1007500000FA05F24EEA020E20FA04F301FA05F25D
:1007600043EA020321FA04F001F0004121FA04F205
:1007700020EA020000EBD3705EEA430E08BF20EAD5
:10078000D37070BD94F0000F0FD101F0004640000F
:1007900041EB010111F4801F08BF013CF7D041EA91
:1007A000060195F0000F18BF704703F00046520095
:1007B00043EB030313F4801F08BF013DF7D043EA66
:1007C0000603704794EA0C0F0CEA135518BF95EA1C
:1007D0000C0F0CD050EA410618BF52EA4306D1D1A3
:1007E00081EA030101F000414FF0000070BD50EAC2
:1007F000410606BF1046194652EA430619D094EA4C
:100800000C0F02D150EA013613D195EA0C0F05D135
:1008100052EA03361CBF104619460AD181EA030189
:1008200001F0004141F0FE4141F470014FF0000041
:1008300070BD41F0FE4141F4780170BD70B54FF0DC
:10084000FF0C4CF4E06C1CEA11541DBF1CEA13555C
:1008500094EA0C0F95EA0C0F00F0A7F8A4EB05043E
:1008600081EA030E52EA03354FEA013100F0888035
:100870004FEA03334FF0805545EA131343EA1263FE
:100880004FEA022245EA111545EA10654FEA0026B3
:100890000EF000419D4208BF964244F1FD0404F56C
:1008A000407402D25B084FEA3202B61A65EB0305C8
:1008B0005B084FEA32024FF480104FF4002CB6EB85
:1008C000020E75EB030E22BFB61A754640EA0C0005
:1008D0005B084FEA3202B6EB020E75EB030E22BF45
:1008E000B61A754640EA5C005B084FEA3202B6EB86
:1008F000020E75EB030E22BFB61A754640EA9C0045
:100900005B084FEA3202B6EB020E75EB030E22BF14
:10091000B61A754640EADC0055EA060E18D04FEAD2
:10092000051545EA16754FEA06164FEAC30343EA72
:1009300052734FEAC2025FEA1C1CC0D111F4801F3F
:100940000BD141EA00014FF000004FF0004CB6E738
:1009500011F4801F04BF01430020B4F1FD0C88BFD7
:10096000BCF5E06F3FF6AFAEB5EB030C04BFB6EBE2
:10097000020C5FEA500C50F1000041EB045170BDD5
:100980000EF0004E4EEA113114EB5C04C2BFD4EB02
:100990000C0541EA045170BD41F480114FF0000E86
:1009A000013C90E645EA060E8DE60CEA135594EA02
:1009B0000C0F08BF95EA0C0F3FF43BAF94EA0C0F05
:1009C0000AD150EA01347FF434AF95EA0C0F7FF47A
:1009D00025AF104619462CE795EA0C0F06D152EACE
:1009E00003353FF4FDAE1046194622E750EA4106B2
:1009F00018BF52EA43067FF4C5AE50EA41047FF4C3
:100A00000DAF52EA43057FF4EBAE12E74FF0FF3C27
:100A100006E000BF4FF0010C02E000BF4FF0010CF8
:100A20004DF804CD4FEA410C7FEA6C5C4FEA430C71
:100A300018BF7FEA6C5C1BD001B050EA410C0CBFC0
:100A400052EA430C91EA030F02BF90EA020F002022
:100A5000704710F1000F91EA030F58BF994208BF89
:100A600090422CBFD8176FEAE37040F00100704746
:100A70004FEA410C7FEA6C5C02D150EA013C07D19D
:100A80004FEA430C7FEA6C5CD6D152EA033CD3D0E8
:100A90005DF8040B704700BF8446104662468C46E2
:100AA0001946634600E000BF01B5FFF7B7FF002815
:100AB00048BF10F1000F01BD4DF808EDFFF7F4FF3E
:100AC0000CBF012000205DF808FB00BF4DF808EDC9
:100AD000FFF7EAFF34BF012000205DF808FB00BFEC
:100AE0004DF808EDFFF7E0FF94BF012000205DF80E
:100AF00008FB00BF4DF808EDFFF7CEFF94BF0120C3
:100B000000205DF808FB00BF4DF808EDFFF7C4FFBB
:100B100034BF012000205DF808FB00BF4FEA410C04
:100B20007FEA6C5C02D150EA013C0AD14FEA430CE7
:100B30007FEA6C5C02D152EA033C02D14FF0000024
:100B400070474FF0010070474FEA410212F5001262
:100B500015D211D56FF47873B3EB625212D94FEA04
:100B6000C12343F0004343EA505311F0004F23FAEE
:100B700002F018BF404270474FF00000704750EA43
:100B8000013005D111F0004008BF6FF00040704700
:100B90004FF00000704700BF4A0011D212F500125A
:100BA00011D20DD56FF47873B3EB62520ED44FEAC5
:100BB000C12343F0004343EA505323FA02F0704745
:100BC0004FF00000704750EA013002D14FF0FF3083
:100BD00070474FF0000070474FEA4102B2F1E04326
:100BE00024BFB3F5001CDCF1FE5C0DD901F0004C14
:100BF0004FEAC0024CEA5070B2F1004F40EB830064
:100C000008BF20F00100704711F0804F21D113F18F
:100C10003872BCBF01F00040704741F480114FEAC8
:100C20005252C2F11802C2F1200C10FA0CF320FA51
:100C300002F018BF40F001004FEAC1234FEAD3236E
:100C400003FA0CFC40EA0C0023FA02F34FEA4303D8
:100C5000CCE77FEA625307D150EA01331EBF4FF061
:100C6000FE4040F44000704701F0004040F0FE407C
:100C700040F40000704700BF7BB972B90029BEBFC5
:100C800000204FF0004106E008BF00281CBF6FF0B5
:100C900000414FF0FF3000F057B8ADF1080C6DE99E
:100CA00004CE002909DB002B1ADB25F0C7F9DDF89B
:100CB00004E0DDE9022304B07047404261EB4101EA
:100CC000002B1BDB25F0BAF9DDF804E0DDE9022397
:100CD00004B0404261EB4101524263EB4303704771
:100CE000524263EB430325F0A9F9DDF804E0DDE9A6
:100CF000022304B0404261EB41017047524263EB72
:100D0000430325F09BF9DDF804E0DDE9022304B09C
:100D1000524263EB4303704753B94AB9002908BFF5
:100D200000281CBF4FF0FF314FF0FF3000F00CB82F
:100D3000ADF1080C6DE904CE25F080F9DDF804E092
:100D4000DDE9022304B07047704700BF10B5054CC1
:100D5000237833B9044B13B10448AFF30080012367
:100D6000237010BDE00500200000000000630208B1
:100D700008B5034B1BB103490348AFF3008008BD1E
:100D800000000000E405002000630208014804F0B0
:100D9000E9BE00BFBC070020034B197811B9034816
:100DA00004F058BB704700BFA2110020FC050020D2
:100DB0007FB508201DF026FA5723002402931D4B0F
:100DC0000193012223464FF4805100941A481B4D91
:100DD00004F0E1FD4FF4FA601DF076FB184B02932E
:100DE0000726184B01932246009601230A21284624
:100DF00005F067FE144B0293144B2246CDE90063C5
:100E000003210123284605F05CFE05230193104BC6
:100E10001049114800930A220D2307F05BF906F0F0
:100E2000B3FA4FF4FA61284604B0BDE8704005F00B
:100E3000EFBE00BF30210020FC050020180C002070
:100E40001C640208990D0008246402088D0D000836
:100E5000786402082C64020868110020014805F03B
:100E600093BE00BF180C00200A4B01219960A1F12C
:100E700001110022D96008499A80C3E90A229A71B7
:100E80001A821A839A841A63196083F83820DA6305
:100E9000704700BFFC0500204C6602080348002391
:100EA0001C218360C36019F033BE00BF3C060020E4
:100EB00037B50D46284652491446FFF779F908B967
:100EC00000209BE001A928461EF04EFD0199A94291
:100ED00053EC102BF4D0226063602C2128461EF0C6
:100EE00068FE0028ECD0451C28461DF05AFD2C2138
:100EF000207228461EF05DFE0028E1D0451C2846E1
:100F00001DF04FFD07EE900AF8EEE77A2C2117EE60
:100F1000903A2846C4F821301EF04BFE0028CFD06E
:100F2000451C28461DF03DFD07EE900AF8EEE77AD5
:100F30002C2117EE903A2846C4F825301EF039FED1
:100F40000028BDD0451C28461DF028FD51EC100B93
:100F5000FFF742FE2C21C4F8090028461EF029FEA6
:100F60000028ADD0451C28461DF018FD51EC100B93
:100F7000FFF732FE2C21C4F80D0028461EF019FEA2
:100F800000289DD0451C28461DF008FD51EC100B93
:100F9000FFF722FE2C21C4F8110028461EF009FE9E
:100FA00000288DD0451C28461DF0F8FC51EC100B94
:100FB000FFF712FE2C21C4F8150028461EF0F9FD9B
:100FC00000283FF47DAF451C28461DF0E7FC51EC9E
:100FD000100BFFF701FE2C21C4F8190028461EF063
:100FE000E8FD00283FF46CAF01301DF0D7FC51EC58
:100FF000100BFFF7F1FDC4F81D00012003B030BD58
:10100000116702080000000082B02DE9F0472DEDC5
:10101000028B0AA981E80C001446DDF8452002EE97
:10102000902ADDF8412002EE102ADDF83D201D4611
:1010300001EE902ADDF84930DDF8392008EE903ACB
:1010400001EE102ADDF84D30DDF835200746006846
:1010500008EE103A00EE902A0368DDF831201B6993
:1010600000EE102A9847002868D097F83E309FED90
:101070003A7ADFED3A7A3A4E752B3A4B0CBF17EEBF
:10108000908A17EE108A18BF9A46DFED377A97F8E4
:101090004330B7EE007A0CBF17EE909A17EE109A15
:1010A00014BF4FF4B4764FF0000A73B120462946BE
:1010B00027A3D3E90023FFF7C1FBDFED2C7A68EE0D
:1010C000A78A28EE278A04460D464846FFF734FAD9
:1010D00002460B4620462946FFF7F8FC074698BB18
:1010E0004046FFF729FA02460B4620462946FFF7FD
:1010F0000BFD58BB9DF830300233DBB2012B1DD8FD
:1011000007EE90AAB8EEE77AB4EEE87AF1EE10FABC
:1011100014DC07EE906AF8EEE77AF4EEE87AF1EE86
:1011200010FA0BD4B4EEC87AF1EE10FA06DCF4EE45
:10113000C87AF1EE10FA54BF01200020BDEC028BFA
:10114000BDE8F04702B070470020F7E73846F5E702
:10115000F8C1631ADCA54C4000C8AF4800007A44CF
:1011600020A1070098FEFFFF6F12833AE12E65422F
:101170002DE9F04F2DED028BDDB09846689B6A9FFC
:101180000D46002119701378472B044640F0618109
:101190005378582B05D000205DB0BDEC028BBDE824
:1011A000F08F98F80260002EF5D198F80030412BAE
:1011B00040F0E28098F80130A3F13106082E02DDFC
:1011C00005233B70BEE090F83020303B9342E2D1E3
:1011D000BF484FF4877104F0F8FAC30740F1378134
:1011E00094F830301841C00700F1318106EB8603D6
:1011F00006EBC30101F588712923B54851AA89B2CC
:1012000004F0B6FA94F83030022B00F29D80DDE94C
:101210005101ADA3D3E90023FFF710FBDDF86531E1
:10122000DFEDAC7A519007EE103A27EE877A5291B3
:1012300017EE103ACDF86531DDF8693107EE103A56
:1012400067EE877A17EE903ACDF86931DDE95123E0
:10125000A14943EC102B0BA803F068FBDDF84D010E
:10126000FFF76AF915AE41EC100B9B49304603F0CD
:101270005DFBDDF85101FFF75FF91FAF41EC100B8B
:101280009549384603F052FBDDF85501FFF754F954
:101290000DF1A40841EC100B8F49404603F046FBCA
:1012A000DDF85901FFF748F90DF1CC0941EC100BBD
:1012B0008949484603F03AFBDDF85D01FFF73CF948
:1012C0000DF1F40A41EC100B8349504603F02EFB5C
:1012D000DDF86101FFF730F947AA41EC100B104629
:1012E0007D4903F023FBDDF865319DF94CB100EE3B
:1012F000103A20F09BFCDDF86931B0EE408A00EE38
:10130000103A20F093FC206803689B68F0EE408A56
:101310009847FDEEE88ABDEEC88A47AACDE906A245
:1013200008905B460BAACDE90489CDE902676B49B9
:10133000CDED018A8DED008A28461DF0F7FB699AF4
:1013400000231370012027E7032B3FF47FAFDDF864
:101350006521DFED637A07EE102A87EE277ADDF844
:10136000692117EE103A07EE102AC7EE277ACDF85A
:10137000653117EE903A67E7552B7FF40CAF98F87C
:101380000130392B3FF71CAF90F83020303B9342AF
:101390007FF401AF014651A800F022FF9DF84431CF
:1013A000002B54D04F4C504B9DF84B112846002930
:1013B0000CBF214619461EF0EDFB4C4B9DF8461123
:1013C000284600290CBF214619461EF0E3FB484B76
:1013D0009DF84811284600290CBF214619461EF0E9
:1013E000D9FB444B9DF84511284600290CBF2146E6
:1013F00019461EF0CFFB404B9DF8471128460029A7
:101400000CBF214619461EF0C5FB3C4B9DF84A1106
:10141000284600290CBF214619461EF0BBFB384B5D
:101420009DF84911284600290CBF214619461EF097
:10143000B1FB344B9DF84C11334A284600290CBFB0
:10144000114619461EF0A6FB699B1E707AE702231F
:10145000B7E6532B7FF49FAE5378582B7FF49BAEA7
:1014600098F80030412B7FF496AE98F802302C2B80
:101470007FF491AE16484FF4877104F0A6F998F8FE
:10148000013094F83020303B93427FF484AEC107A2
:10149000DDD540FA02F3DB07D9D498F80330522B9C
:1014A0000DF5A27932D198F804307BBB012393402B
:1014B0001843ADF84401022305484A464FF48771AA
:1014C00004F0A8F93EE700BFF8C1631ADCA54C4060
:1014D000FC050020E12E65425364020859640208AD
:1014E00000007A4442640208346402083864020846
:1014F0003C6402084064020844640208486402082C
:101500004C64020850640208E2730208261D0FCEE4
:101510004D460FC50FCE0FC596E8070003C508F16D
:1015200003012A7020464A46FFF7C2FC00287BD000
:1015300094F83080B8F1020F5ED8DDE951013FA385
:10154000D3E90023FFF750F8DDF86521DFED387AA5
:10155000519007EE102A87EE277ADDF86921529123
:1015600017EE103A07EE102AC7EE277ACDF865314C
:1015700017EE903ACDF8693153AE0FCE6D460FC5D8
:101580000FCE0FC533682B7099E80C0041462046FA
:10159000FFF73AFD002847D094F83010254801396C
:1015A00001EB810301EBC30101F5887129234A4650
:1015B00089B204F02FF9206843680B337FF4C2AE80
:1015C000DDF86121036802EE902ADDF85D21DB6819
:1015D00002EE102ADDF8592101EE902ADDF855219E
:1015E00001EE102ADDF8512100EE902ADDF84D21A0
:1015F00000EE102A9847A5E6B8F1030FBCD0DDF83D
:101600006531DFED0D7A07EE103A27EE877A17EE97
:10161000103ACDF86531DDF8693107EE103A67EE22
:10162000877A17EE903AA5E70623CAE5AFF3008064
:10163000E12E6542FC05002000007A44F8C1631ADF
:10164000DCA54C40006803681B6A1847F8B50446DF
:101650002DED028B002084F82D0084F82F004A48DD
:101660009DF820C0B0EE408A04F1310500F1180663
:1016700050F8047B45F8047BB042F9D100200025E6
:1016800000260027C4F8B0201A7AA4F84C00C4E958
:101690001667A4F84E001E685F6884F85000C4E91D
:1016A0001C00A4F8600084F8620084F86C00A56750
:1016B000E567C4F88050C4F88450C4F88850C4F872
:1016C0008C50C4F8945084F89800304D84F8AC00E5
:1016D000C4F8B400227301F13000D3F8092084F873
:1016E0003010C4F8A450C4F8A85084F83A006660DA
:1016F000A760C4F82520D3F80D20C4F82920D3F81A
:101700001130C4F890300139214B43F821400829A9
:1017100009D8DFE801F0050F11131517191B1D007B
:101720001C4BC4F8B430BCF1030F1BD8DFE80CF03D
:1017300012202224184BF4E7184BF2E7184BF0E77D
:10174000184BEEE7184BECE7184BEAE7184BE8E7C5
:10175000184BE6E7184904F13E001EF0F2FA0023A8
:1017600084F8433084ED258ABDEC028B2046F8BD19
:101770001249F0E71249EEE7114904F13E001EF06C
:10178000E0FA0123ECE700BF186302080000C07F05
:1017900058060020C5270008D1270008DD270008CB
:1017A000E9270008F5270008012800080D2800088F
:1017B00019280008252800087A6402087C640208B9
:1017C0007F6402082DE9F043944E016096F82C30B6
:1017D0008DB004460D460DF1280893B94FF487717A
:1017E000304603F0F2FF94F8302001239340184371
:1017F000ADF82800022342464FF48771304604F0CA
:1018000009F886484FF4877103F0DFFF94F8303011
:1018100010F0010F02BF01229A40024303F1FF368C
:10182000074608BF97B206EB860206EBC20647FAE8
:1018300003F306F5887613F0010FB6B204F104093C
:1018400043D004F12103029304F11D03019304F139
:101850001903009304F1110204F1150304F10D01C1
:10186000284601F020F86D4829234A46314603F006
:10187000D1FF94F830200123934027EA0300ADF80C
:1018800028000223654842464FF4877103F0C2FFE7
:1018900004F10C073146614829234A4603F068FFEA
:1018A0000FCF6E460FC60FCF0FC63B68337099E857
:1018B0000C0094F830102046FFF7A6FB68B94FF0F3
:1018C000000948460DB0BDE8F0835448292231464E
:1018D00003F036FF0028B4D1CBE7D4F8B03050483D
:1018E00093F90C20B3F90210002600969B6804F0CF
:1018F00005F9D4F8B03084F8460093F91C20B3F908
:10190000001000965B69464804F0F8F8D4F8B0304F
:1019100084F8470093F91C20B3F9041000969B69E2
:101920003F4804F0EBF8D4F8B02084F84800B2F94E
:101930000030591C04D0B2F90460F31A5E425E41D3
:101940002B6884F82D601B6828469847814600283C
:10195000B5D02B6828469B6898474F2805D1D4E915
:101960000101FFF739F9C4F82100D4F821202B68D0
:1019700002EE902AD4F81D20DB6802EE102AD4F87B
:10198000192001EE902AD4F8152001EE102AD4F87F
:10199000112000EE902AD4F80D20284600EE102ADF
:1019A00098472B6894F90C105B6828469847D4F840
:1019B0009000FEF7C1FDD4E9016702460B463046B0
:1019C0003946FEF711FEFFF707F92B6800EE100A03
:1019D0005B6B28469847134B18689A889B790A9046
:1019E00088F8063094F83030A8F8042030338DF8A9
:1019F0002A30D4F8B4300C480022CDE90138012354
:101A00001146009305F05DF841F288320446014624
:101A1000054804F067FF6C7253E700BFFC05002027
:101A2000BC07002084640208180C0020034680F8DC
:101A30004410006893F86C30026883F00103526927
:101A40001940104738B504460D4611B980F86210A8
:101A500038BD90F86C303BB1002380F86C300068E2
:101A6000036801215B699847012384F862301CF008
:101A700027FD0544A566EBE7D0B5044610EE100A35
:101A800094F89830BBB9FEF757FDD4E901670246D8
:101A90000B4630463946FEF7A7FD41EC100B21F00E
:101AA0004FFB51EC100BFFF74FF801462068BDE8E3
:101AB000D04000F078BFD0BD70B590F89850044683
:101AC0000E4615B11725284670BD00680368DB6A0D
:101AD0009847B5EE400AF1EE10FAF3D1206803689A
:101AE0003146DB699847EEE710B553EC102B0446FE
:101AF000D0E90101FEF778FD41EC100B20F0BCF8B5
:101B000001462046BDE81040FFF7D6BF036810B578
:101B10000446D86BFEF7FEFCD4E90123FEF78EFEE7
:101B200041EC100B10BD90F860302DE9704355EC7E
:101B3000104B0646CBB1D0F82900FEF7FDFC8046DD
:101B4000894642464B4620462946FEF7DDFF80B9CE
:101B5000D6F82500FEF7F0FC8046894642464B4603
:101B600020462946FEF7B2FF60B945EC104BBDE8B0
:101B7000708320462946D6E91623FEF77DFB0446EE
:101B80000D46DEE720462946D6E91623FEF776FB0A
:101B900004460D46E2E7000090F860302DE9F74F6B
:101BA00055EC104B06468BB3006803681B6A9847D8
:101BB000FEF7B0FCD6E90123FEF740FED6E9168910
:101BC0001E4B82468B46002240464946FEF70CFDDE
:101BD00002460B4606460F4650465946FEF74EFB58
:101BE000CDE90001DDE9002320462946FEF78CFF00
:101BF00088B932463B4650465946FEF73DFB024601
:101C00000B4620462946FEF761FF68B945EC104BAC
:101C100003B0BDE8F08F2046294642464B46FEF70A
:101C20002BFB04460D46DDE72046294642464B463F
:101C3000FEF724FB04460D46DBE700BF0000E03F53
:101C40002DE9F04F90F8603087B08DED000B8246A3
:101C5000002B00F08880FFF79FFFDAF80000036890
:101C60008DED020B1B6A9847FEF754FCDAE901235D
:101C7000FEF7E4FD02460B4604460D46DDE902018F
:101C8000FEF7FAFADDE90223804621F000492046FA
:101C90002946FEF7F1FA21F00047064602463B4688
:101CA00040464946FEF71CFF08B146464F469AEDAE
:101CB000167BDDE9020153EC172B8DED047BFEF75B
:101CC000DDFA02460B46CDE9002322462B46FEF7FD
:101CD000D3FADDE90023824621F0004B2046294655
:101CE000FEF7CAFA21F00049804602464B465046AC
:101CF0005946FEF7F5FE08B1D046D94632463B4676
:101D000040464946FEF7E2FE68BBDDE90423DDE913
:101D10000201FEF7B1FA02460B46CDE90023224646
:101D20002B46FEF7A9FADDE90023804621F00049A1
:101D300020462946FEF7A0FA21F000450446024657
:101D40002B4640464946FEF7CBFE08B144464D4679
:101D500022462B4630463946FEF7D6FE18B99DED91
:101D6000027B8DED007B9DED000B07B0BDE8F08F91
:101D700010B50446FFF710FFD4E9010153EC102B16
:101D8000FEF732FC41EC100B1FF076FF0146206895
:101D90000268BDE81040526A104710B5044600685A
:101DA00003681B6A9847FEF7B5FBD4E90123FEF7E9
:101DB00045FD41EC100B2046BDE81040FFF7B3BED7
:101DC00038B505680446FFF73BFFD4E9010153EC41
:101DD000102BFEF709FC41EC100B1FF04DFFD4F85F
:101DE0000D2007EE902AFDEEE77A014617EE902AC5
:101DF0002846BDE8384000F08DBD000038B50446E7
:101E0000006803682DED028BB0EE408AF0EE608A28
:101E10001B6B9FED120A9847B0EE480AF0EE680A75
:101E200020462568FFF70CFFD4E9010153EC102B85
:101E3000FEF7DAFB41EC100B1FF01EFFD4F80D206B
:101E4000BDEC028B07EE902AFDEEE77A014617EE15
:101E5000902A2846BDE8384000F086BD000000000A
:101E600010B50446FFF7ECFED4E9010153EC102B4A
:101E7000FEF7BAFB41EC100B1FF0FEFE0146206896
:101E8000BDE8104000F06ABD2DE9D043044600686B
:101E900003689B6A98470028B8BF4042FEF73AFBA8
:101EA0000646D4F89400D4E901890F46FEF744FBB6
:101EB00002460B4640464946FEF796FB02460B4655
:101EC00030463946FEF70CFE003818BF0120BDE849
:101ED000D0832DE9D0430446006803689B6A984785
:101EE0000028B8BF4042FEF715FB0646D4F8900024
:101EF000D4E901890F46FEF71FFB02460B46404618
:101F00004946FEF771FB02460B4630463946FEF75E
:101F1000DDFD003818BF0120BDE8D08310B50446B0
:101F2000006800F050FDFEF7F5FAD4E90123FEF752
:101F300085FC41EC100B10BD90F898308BB99FEDEB
:101F4000097A094BC0F8A430C0EE077A90ED247AE4
:101F5000F4EE477AF1EE10FAC8BFF0EE477AC0ED22
:101F6000277A7047000048430000C07F90F89830FF
:101F700053B9DFED067AB4EE670AF1EE10FA48BF06
:101F8000B0EE670A80ED290A704700BFCDCCCC3D8A
:101F900090F898308BB99FED097A094BC0F8A830BA
:101FA000C0EE077A90ED247AF4EE477AF1EE10FA5B
:101FB000C8BFF0EE477AC0ED287A7047000048436A
:101FC0000000C07F90F898300BB980ED2A0A704766
:101FD00090F89800003818BF0120704780ED210A62
:101FE000704780ED230A704780ED200A704700009B
:101FF000D0ED217AF5EE407AF1EE10FA06D0F4EE4B
:10200000407AF1EE10FAC8BFB0EE670AD0ED237A3D
:10201000F5EE407AF1EE10FA06D0F4EE407AF1EEE9
:1020200010FA48BFB0EE670AD0ED297A80ED220A97
:10203000F4EE677AF1EE10FA7FBFC0EE276A9FEDEB
:102040000B7AC6EE877AC0ED277AD0ED2A7AF4EEC5
:10205000677AF1EE10FA7FBFC0EE276A9FED037A30
:10206000C6EE877AC0ED287A704700BF000048436B
:102070002DE9F04190F8612090F86C302DED028B45
:102080000446B0EE408A002A4ED0B5EE400AF1EE8A
:1020900010FA49D1D0ED207AF5EE407AF1EE10FA3F
:1020A00042D15BB990F8623073BB002584F862506E
:1020B0001CF006FA236FC01AA8422CDC25682B6896
:1020C000D3F8308094F84430002B00F0838094F8EB
:1020D0009830D4E90167002B79D1D4ED207A78EEDD
:1020E000277A17EE900AFEF727FA32463B46FEF7AC
:1020F0007BFAFEF771FD00EE100ABDEC028B28465C
:102100004346BDE8F04118471CF0DAF9A36EC01A47
:102110000028CADCD2E72068012384F86C30036809
:1021200029465B699847C9E73BB12068002384F8DA
:102130006C30036801215B6998471CF0C1F9636E3C
:10214000B5EE408A0344F1EE10FA2367B6D0B5EE3F
:10215000C08AF1EE10FA94ED217AD4ED237A1CD5E1
:10216000F5EE407AF1EE10FA08D0F1EE677AF4EE6F
:10217000487AF1EE10FAC8BFB0EE678AB5EE407A41
:10218000F1EE10FA9AD0B1EE477AB4EE487AF1EE59
:1021900010FA48BFB0EE478A90E7B5EE407AF1EE0C
:1021A00010FA06D0B4EE478AF1EE10FA48BFB0EE4E
:1021B000478AF5EE407AF1EE10FA3FF47FAFB4EEC5
:1021C000678AF1EE10FAC8BFB0EE678A76E718EEBC
:1021D000100A88E79FED010A8FE700BF00000000AA
:1021E00010B509680B6804469B699847204610BDE6
:1021F00080F8451070470000F0B50E4601680B6886
:1022000085B09B69044601A898479DF80C5065B9B4
:1022100006F0FD03012B29D12046FFF713FA274BC7
:10222000984205DD012584F82F50284605B0F0BD01
:1022300094F8453043B994F82D30002BF3D194F83D
:102240002E50C5F34005EEE72046FFF7A6FDD4F873
:10225000290057EC106BFEF76FF902460B4630462B
:102260003946FEF751FC0028DCD1E4E7023E012E9E
:10227000D9D82046FFF7E6F9114B9842D2DB94F803
:10228000453043B994F82D30002BCCD194F82E5022
:1022900005F00105C7E72046FFF77FFDD4F82500CC
:1022A00057EC106BFEF748F902460B4630463946AC
:1022B000FEF70CFC0028B5D1E4E700BF0033337310
:1022C00000CDCC8C38B590F844302DED028B04460F
:1022D000B0EE408A1BB390F8985015BB0321FFF76E
:1022E0008BFF00BBB4EE488AF1EE10FA04D6B0EED4
:1022F000480A2046FFF77CFE206800F059FB206862
:102300000023037703680121DB6B9847032384F8DC
:1023100098300023E367BDEC028B284638BD1225B8
:10232000F9E71425F7E71525F5E738B590F84430B7
:102330002DED028B04460D46B0EE408A43B390F873
:102340009830032B26D0FFF757FF28BB6B1E012BBD
:1023500024D8B4EE488AF1EE10FA04D6B0EE480A5A
:102360002046FFF745FE94F898303BB92068836B10
:10237000436303680121DB6B01779847012D14BF8C
:102380000523042384F898300020BDEC028B38BD6F
:102390001220FAE71420F8E71520F6E71820F4E7F2
:1023A00090F8443070B504460D46002B45D090F8A7
:1023B0009860002E43D10321FFF71EFF002840D173
:1023C000D4F8B0309B68013335D0206801230377FF
:1023D000836B436394F8AC3013B9032384F8AC30B7
:1023E00094F898301BB903680121DB6B984794F887
:1023F0004610154803F0AEFB00280CBF052304234C
:1024000084F898309DB9D4F8B03094ED227AD3EDA9
:10241000046AC6EE877A9FED0D7A67EE877A9FEDA4
:102420000C7A67EE877AFCEEE77A17EE905A1CF08A
:1024300047F828446067304670BD1226FBE7142633
:10244000F9E71526F7E700BFBC0700209A99993FE6
:1024500000007A442DE9F04190F830300446002B1A
:1024600000F0AE8190F8983033B103689B7A1BB9C5
:1024700080F898300023836794F84710C04803F031
:1024800069FB94F82E3094F8481060F3000384F848
:102490002E30BB4803F05EFB94F82E3094F82D509C
:1024A00060F3410384F82E3025B1DDB215F0030549
:1024B00018BF012594F8AC302BB394F898301A1F4C
:1024C000012A20D8042B08D194F84610AC4803F018
:1024D00041FB10B9204600F0ABF994F89830052B79
:1024E00008D194F84610A64803F034FB10B12046FA
:1024F00000F09EF91BF0E4FF636FC01A002802DDB4
:10250000204600F0A4F99F4804F03EFB94F8983070
:1025100013B12068027AA2B10026A667002D00F050
:102520004781C4F88060974804F02EFB204694ED64
:102530001E0AFFF79DFD20680368BDE8F0415B6C53
:102540001847012B0BD000F052FA01462046FFF746
:1025500053FE20B12046BDE8F04100F078B994F870
:102560009830032B54D1002DF4D12046FFF78CFC7A
:1025700070B1206803682946DB6B98470023A36786
:10258000236884F8985001221A779A6B5A63CAE735
:102590009FED7D7AD4ED277A67EE877A77EEA77A7A
:1025A00017EE900AFDF7C8FF064620460F46FFF7D4
:1025B000B5FC304653EC102B3946FEF715F8FEF704
:1025C0000BFB00EE100A1FF0E5FED4ED247A206824
:1025D000B4EE670AF1EE10FA48BFB0EE670AD4ED28
:1025E000227AF4EE407AF1EE10FA48BFB0EE670AB4
:1025F00084ED1E0A03689B6A98470028BEBFD4ED8D
:102600001E7AF1EE677AC4ED1E7AA36FE3678AE75C
:10261000013B042B00F2B080DFE803F09127AE030A
:10262000150094ED277AD4ED1E7A77EE877A94ED33
:10263000227AF4EE477AF1EE10FAC8BFF0EE477A4C
:10264000C4ED1E7A6FE794ED277AD4ED1E7A77EE0B
:10265000C77A94ED227AB1EE477AF4EE477AF1EE3A
:1026600010FA48BFF0EE477AEAE7002D7FF472AF28
:10267000D4ED1E7A94ED277AF4EEC77AF1EE10FAD3
:1026800034DD77EEC77AC4ED1E7AF0EEE77AB4EE69
:10269000E77AF1EE10FAFFF646AF206803680021F2
:1026A000DB6B98470023A36794F8AC300022032B20
:1026B00084F8982026D1022384F8AC30D4ED227A15
:1026C0003249B1EE087AF0EEE77A87EE870A2046C3
:1026D000DFED2F7AB4EE670AF1EE10FA48BFB0EEE4
:1026E000670AFFF785FCFFF75BFE1CE7F1EE476A20
:1026F000F4EEE67AF1EE10FA4CBF77EE877ADFED72
:10270000257AC0E7022B15D194F846101C4803F037
:1027100021FA08B90123CFE7D4ED227AB1EE087A85
:1027200067EE877AC4ED227A94F8AC30002B3FF440
:10273000FAAEC3E7012BF7D184F8AC20F3E6D4ED71
:102740001E7A94ED287AF4EEC77AF1EE10FA23DDC2
:1027500077EEC77AC4ED1E7AF0EEE77AB4EEE77A48
:10276000F1EE10FAFFF6DFAE206803680021DB6BA4
:102770009847002384F898300023A367D3E600BF6E
:10278000BC070020180C002000004843C0D4010002
:1027900052499D3900000000F1EE476AF4EEE67AF6
:1027A000F1EE10FA4CBF77EE877A5FED067AD1E74B
:1027B00003212046FFF720FD00287FF4B2AEB2E6E9
:1027C000BDE8F081014B1868FFF744BE58060020B1
:1027D000014B5868FFF73EBE58060020014B986831
:1027E000FFF738BE58060020014BD868FFF732BE0D
:1027F00058060020014B1869FFF72CBE5806002030
:10280000014B5869FFF726BE58060020014B986916
:10281000FFF720BE58060020014BD869FFF71ABE0B
:1028200058060020014B186AFFF714BE5806002016
:1028300090F89820022A09D9026801211177916B3A
:102840005163022280F89820FFF704BE704790F889
:102850009820012A10B40DD902680121946B5463A9
:10286000117700225DF8044B80F8981080F8AC20B6
:10287000FFF7F0BD5DF8044B70478B1E012B02463D
:1028800006D890F82E3013F0010005D001207047D3
:10289000012903D0002070470329F8D192F82E00B7
:1028A000C0F34000704710B5446C0C60816C11603F
:1028B000C26C1A60029B026D1A60039B426D1A6023
:1028C000049B826D1A6010BD80ED110AC0ED120AE2
:1028D00080ED131AC0ED141A80ED152AC0ED162AEA
:1028E00070470023C36372B681634163038562B698
:1028F000704772B6836B436362B6704772B6826B81
:10290000C06B62B61044704772B6836BC91AC1635C
:1029100062B6704730B445680C3504460B4613D197
:10292000816B5B1AA3EB4203002192008A4203EB06
:10293000010004DD90FBF2F502FB150515B9E0631B
:1029400030BC70470131F1E7036830BC5B6A18475F
:1029500072B6426BC06B62B61044704772B6C36BFE
:10296000C91A416362B6704730B445680C350446F5
:102970000B4615D1C16B5B1AA3EB420300219200F9
:102980008A4203EB010004DD90FBF2F502FB150522
:1029900025B972B6606362B630BC70470131EFE7AB
:1029A00030BCFFF7DBBF72B689B2818562B6704773
:1029B00072B6836B036362B6704772B6426B806B0C
:1029C00062B6101A704772B6826B62B6436B006BC8
:1029D000801A9B1A0028B8BF4042002BB8BF5B4248
:1029E0009842A8BF1846704780ED090A70470368EF
:1029F00010B5DB6A04469847B5EE400AF1EE10FACE
:102A000006D0236C002B05DC206CC00F400010BDED
:102A10000020FCE70120FAE77047C06D03681B68DF
:102A20001847C36DB3F93000704710B50446C06D48
:102A300003685B689847E36DB3F93030A4F87030F1
:102A400010BDC06D03689B68184738B50446C86D53
:102A500003680D46DB699847EB6DD3F81D202260B3
:102A6000D3F8212093F8253062602372204638BDC8
:102A7000D0F8803043B107EE903A9FED057AF8EE3A
:102A8000677A87EE270A70479FED020A704700BFFA
:102A90000024744B0000000001314FF000034FF0A0
:102AA000010210B50EBF80F8673080F8672080F80B
:102AB0006830036E08BF80F868200446B3F904004C
:102AC000002803DB94F867101BF08EFC94F8673045
:102AD000DBB284F8693010BD38B5036E0446B3F933
:102AE0000600421C0D460DD010F1120F0AD000282E
:102AF00006DB197A15B9B1FA81F149091BF074FCAA
:102B0000A57238BDE06D036829461B6A9847F7E750
:102B1000036E10B50446B3F90600002802DB197AEB
:102B20001BF062FCE06D03685B6A9847236EB3F9A3
:102B30000600002807DB197AB1FA81F1BDE81040E0
:102B400049091BF051BC10BD30B5C37A87B00446AB
:102B500013B9002007B030BDC37A092BF9D8036E32
:102B6000B3F90400421CF4D0B3F900300133F0D0C3
:102B7000002802DB01211BF0D9FB226E937884F838
:102B8000663094F86630B3FA83F35B0984F86530F5
:102B9000B2F90000002802DB01211BF0C7FB236E05
:102BA00094F86510B3F900001BF01EFC236EB3F916
:102BB0000600002802DB01211BF0B8FB236EB3F9ED
:102BC0000600002805DB197AB1FA81F149091BF0EA
:102BD0000BFC144B186899889B798DF81630E37AB2
:102BE000ADF8141004AA0292303300258DF8153088
:102BF000D4F890300490019329460B4800950123A6
:102C00002A4603F05EFF014684F864000028A0D045
:102C100094F88D301BB104482A4603F01AFE0120B7
:102C200098E700BF8B640208180C0020C06D036891
:102C300009B19B6918475B69FCE700002DE9F8437F
:102C40001F464FF0FF332DED028B436040F201131E
:102C50009FED718AC361714B036000250E464FF4EE
:102C6000FA63012105728572457280F82050C572A1
:102C70000563058580F8645085859DF82880456347
:102C800080ED098A856380ED118AC56380ED128A23
:102C9000016480ED138A80F8655080ED148A80F815
:102CA000661080ED158A80F8675080ED168A80F8EE
:102CB000681080F86950C366A0F87010A0F8721010
:102CC000C0E9205580F87450C0E9245580F88C5034
:102CD000C0F89850751EEBB2082B0446914680ED63
:102CE0001E8A80ED1F8A80F88D1050D86FF00B037C
:102CF0004B4943600C301DF024F8032E06F13003DD
:102D000028BF4FF000082376E672C4F8609084F87C
:102D10008D80E765384600F03BFCE36DE066B3F973
:102D2000102002EE102AB3F90E2001EE902AB3F91A
:102D30000C2001EE102AB3F90A20B3F9083000EE96
:102D4000902A00EE103AB8EEC22AF8EEE11AB8EE78
:102D5000C11AF8EEE00AB8EEC00AF0EE482A2046A2
:102D6000FFF7B2FD2F4B023E43F82540072E05D852
:102D7000DFE806F0121A222A323A424A2A4BC4F8F5
:102D800090302A4BC4F89430294BC4F89830BDECED
:102D9000028B2046BDE8F883264BC4F89030264BC2
:102DA000C4F89430254BF0E7254BC4F89030254B00
:102DB000C4F89430244BE8E7244BC4F89030244BFB
:102DC000C4F89430234BE0E7234BC4F89030234BF6
:102DD000C4F89430224BD8E7224BC4F89030224BF1
:102DE000C4F89430214BD0E7214BC4F89030214BEC
:102DF000C4F89430204BC8E7204BC4F89030204BE7
:102E0000C4F894301F4BC0E71F4BC4F890301F4BE1
:102E1000C4F894301E4BB8E700000000AC64020810
:102E2000926402087C06002095320008C93300082D
:102E3000FD340008A5320008D93300080D3500081C
:102E4000B5320008E93300081D350008C532000816
:102E5000F93300082D350008D53200080934000880
:102E60003D350008E5320008193400084D350008EA
:102E7000F5320008293400085D35000805330008E4
:102E8000393400086D35000815330008493400084E
:102E90007D35000808B50B4690F8641073B190F8C2
:102EA000692090F868309A420CBFD0F89820D0F88A
:102EB0009420044803F0EDFC012008BDD0F89020D8
:102EC000F7E700BF180C0020D0ED097A90ED1F7ACB
:102ED00090F88C3077EEA77A10B5B4EEE77AF1EE81
:102EE00010FA044610D86BB3052380F88C3000210B
:102EF000FFF7D0FFE06D03790BB9437913B3036893
:102F0000BDE81040DB681847EBB972B6037F8BB1A0
:102F1000036C013305D190F8692090F868309A422B
:102F200008D0236C012B08D194F8692094F86730FD
:102F30009A4202D1022384F88C3062B61BF0C0FAA8
:102F4000C4F8880010BD90F88C30032BFAD1C06D06
:102F500003790BB943792BB103681B69984700B219
:102F6000A4F8720001212046FFF794FF042384F89F
:102F70008C30E7E738B504462DED028B4348B0EEC0
:102F8000408A03F001FEB5EEC08AF1EE10FA20DCB3
:102F900021D5B1EE488A4FF0FF35237A0BB194ED7D
:102FA000098AD4ED1E7AF4EE487AF1EE10FA14D1C3
:102FB00094F88C30022B10D872B6256462B6237A4E
:102FC000002B5FD1BDEC028B2046BDE83840FFF7F7
:102FD0007BBF0125E1E70025DFE794F88C3084ED25
:102FE0001F8A012B03D094F88C30042B08D1B4F83D
:102FF00072301BB207EE903AF8EEE77A88EE278A35
:103000009FED237AC7EE087AF4EE677AF1EE10FAB4
:1030100033D69FED207AF4EEC77AF1EE10FA2CD871
:10302000B3EE000A27EE800A20F044FA0246236C31
:10303000C4F88020AB421CBF00232364D4F8843042
:1030400084ED1E8A934208D094F864100F4803F070
:1030500056FCD4F88030C4F88430256494F88C3061
:10306000052B04BF002384F88C3094F88C30042B9B
:1030700004BF012384F88C30A1E700259FED068A68
:103080002A46D4E7BDEC028B38BD00BF180C0020E7
:103090000024744990F4F74C0000000038B5044651
:1030A0000D4690F8651028461BF09EF994F88C3078
:1030B000022B1FD1A16B238DB4F8702011FA83F37A
:1030C00012B293FBF2F102FB11339BB994F8693011
:1030D000FC2B0FD8032384F88C30637A03F0FF02B3
:1030E00043B1674B9918097B21B103EB820301229D
:1030F0001B6C5A7094F88C30022B25D8237F626B9E
:103100002BB1237A1BB9216C636B0B446363A16BF6
:10311000636B994219DC237A2BB194F8691094F807
:103120006830994211D0A16B636B99425CDB237AC2
:103130002BB194F8691094F86730994254D0237AEF
:1031400013B9FD2384F8693038BD94F8691094F8F8
:10315000683099420ED0626394F86830DBB284F82C
:10316000693094F86810236EB3F90400BDE8384064
:103170001BF03AB9238D9BB2002B31D0238D013B3C
:103180009BB22385238D9BB2003B18BF0123237282
:10319000E37A022B20D9236E94F86910B3F9040066
:1031A0001BF022F994ED1B0ADFED367AB8EE400AE7
:1031B00080EE270A20F0B2F9334B3449344A1B68B9
:1031C000B3FBF2F34868BCEEC00A10EE102A53437A
:1031D0004A68121A9342FBDC94F866102846C5E749
:1031E000A26B013AA263D2E794F8691094F86730B1
:1031F000994208D0626394F86730DBB284F8693092
:1032000094F86710AFE7228DA38D92B29BB29A42D9
:1032100031D2238D01339BB22385238DA28D9BB2A6
:1032200092B293422CBF002301232372E37A022B34
:10323000D2D9236E94F86910B3F904001BF0D4F8C6
:1032400094ED1B0ADFED0F7AB8EE400A80EE270AF4
:1032500020F064F90C4B0D490D4A1B68B3FBF2F3E7
:103260004868BCEEC00A10EE102A53434A68121A8E
:103270009342FBDCB0E7A36B0133A3630023D4E7E5
:10328000180C002000007A44F8010020001000E033
:1032900040420F00024B1A211868FFF7FFBE00BF23
:1032A0007C060020024BC4215868FFF7F7BE00BF20
:1032B0007C060020024B18219868FFF7EFBE00BF84
:1032C0007C060020024B1921D868FFF7E7BE00BF3B
:1032D0007C060020024B18211869FFF7DFBE00BFF3
:1032E0007C060020024B4FF0FF315869FFF7D6BE35
:1032F0007C060020024B4FF0FF319869FFF7CEBEED
:103300007C060020024B4FF0FF31D869FFF7C6BEA4
:103310007C060020024B4FF0FF31186AFFF7BEBE5B
:103320007C06002038B504460D4690F86510284606
:103330001BF05AF894F88C30022B3CD8237F2BB129
:10334000B4F87230626B02FA83F36363A26B636B4F
:103350009A4230DAB4F87230A26B02FA83F3A363B4
:10336000E37A022B20D9236E94F86910B3F9040094
:103370001BF03AF894ED1B0ADFED0F7AB8EE400A25
:1033800080EE270A20F0CAF80C4B0D490D4A1B6845
:10339000B3FBF2F34868BCEEC00A10EE102A5343A8
:1033A0004A68121A9342FBDC94F866102846BDE87E
:1033B00038401BF019B838BD00007A44F8010020ED
:1033C000001000E040420F00024B1A211868FFF77E
:1033D000A9BF00BF7C060020024BC4215868FFF73C
:1033E000A1BF00BF7C060020024B18219868FFF7A0
:1033F00099BF00BF7C060020024B1921D868FFF757
:1034000091BF00BF7C060020024B18211869FFF70E
:1034100089BF00BF7C060020024B4FF0FF31586986
:10342000FFF780BF7C060020024B4FF0FF31986908
:10343000FFF778BF7C060020024B4FF0FF31D869C0
:10344000FFF770BF7C060020024B4FF0FF31186A77
:10345000FFF768BF7C06002038B504460D4690F89B
:10346000651028461AF0C0FF94F88C30022B3CD827
:10347000237F2BB1B4F87220636B12B29B1A636383
:10348000A26B636B9A4230DDB4F87220A36B12B268
:103490009B1AA363E37A022B20D9236E94F8691058
:1034A000B3F904001AF0A0FF94ED1B0ADFED0F7AC8
:1034B000B8EE400A80EE270A20F030F80C4B0D4998
:1034C0000D4A1B68B3FBF2F34868BCEEC00A10EE6D
:1034D000102A53434A68121A9342FBDC94F8661090
:1034E0002846BDE838401AF07FBF38BD00007A4456
:1034F000F8010020001000E040420F00024B1A21AA
:103500001868FFF7A9BF00BF7C060020024BC4214A
:103510005868FFF7A1BF00BF7C060020024B1821AE
:103520009868FFF799BF00BF7C060020024B192165
:10353000D868FFF791BF00BF7C060020024B18211E
:103540001869FFF789BF00BF7C060020024B4FF0CF
:10355000FF315869FFF780BF7C060020024B4FF017
:10356000FF319869FFF778BF7C060020024B4FF0CF
:10357000FF31D869FFF770BF7C060020024B4FF087
:10358000FF31186AFFF768BF7C0600207047000013
:10359000B0F90620034B33F912000028B8BF4FF4EE
:1035A000FA607047F4640208F0B5114D07460E4604
:1035B0000FCD8BB001AC0FC40FCD0FC42B682360AF
:1035C000B7F90630102B0FDC01A9002251F8040BCB
:1035D000B04206D1074903EBC3030B4498560BB026
:1035E000F0BD0132092AF1D14FF0FF30F7E700BFFB
:1035F000306302081665020870B52DED048B044691
:10360000F0EE609AB0EE419AF0EE618AB0EE428A36
:103610001EF00CFBBDEEC00A10EE103AB0EE690AC7
:103620001DB21EF003FBFDEEC07AB0EE490A17EEA4
:10363000903A1EB266811EF0F9FABDEEC00A10EE95
:10364000103AB0EE680AA3811EF0F0FABDEEC00A8F
:1036500010EE103AB0EE480AE3811EF0E7FABDEE34
:10366000C00A204610EE103A238294F912309A1CB8
:1036700014BF00230123A37494F91330013304BF52
:103680000623E37494F91430013304BF0523237532
:103690006B1C08BF0125013608BF658129462581BD
:1036A000FFF782FFB4F90A60608631462046FFF7D3
:1036B0007BFF95FBF6F5BDEC048BA086258670BDDF
:1036C00070B52DED028BB0F90610037F1B4A022B5B
:1036D00032F911208CBF4FF4FA634FF496739A427B
:1036E0000546B0EE608A24DC1EF0A0FAFDEEC07A3A
:1036F000B0EE480A17EE904A1EF098FAFDEEC07A36
:10370000621C17EE906A08BF0124A64211DA214616
:103710002846FFF749FF01300BD0731C0BD0314610
:103720002846FFF741FF013018BF0120BDEC028B96
:1037300070BD0020FAE70120F8E700BFF46402083A
:103740005420704707B5B0F90C3090F9121001936E
:10375000B0F90E300093003990F8323090F9132010
:1037600018BF01213C3000F02FFA03B05DF804FBD4
:1037700007B5B0F9103090F912105A1C08BFB0F913
:103780000E30B0F90C20CDE90032003990F832301B
:1037900090F9142018BF01213C3000F015FA03B055
:1037A0005DF804FB30B5044685B0FFF725FFB4F99A
:1037B0000E305A1C5AD0B4F910200132B4F90C2042
:1037C00008BF2382013206D100EE103ABAEEEF0AAA
:1037D0001FF070FEA081A16B207FB1F90230B1F91A
:1037E00000200290B1F908000190B1F90410009195
:1037F00004F13C05B4F90610284600F0ABF9B4F921
:103800000C3094F912100193B4F90E300093003982
:1038100094F8323094F9132018BF0121284600F0A3
:10382000D3F994F915305A1C18BF012262773BB9BD
:10383000A36BB3F90C0000280EDB02211AF076FD11
:1038400094F91530012B07D1A36BB3F90C000028B4
:1038500002DB00211AF06AFDB4F93030013B18BFD9
:10386000012323710023637105B030BDB4F9063024
:103870000C2B40F6C41318BF4FF41673E381238258
:10388000A2E710B504462DED048BB0EE419AF0EEA0
:10389000618AB0EE428AFFF713FFB4F906300C2BB1
:1038A0002CD00D2B2DD140F6B834B0EE490A1EF0C5
:1038B000BDF9FDEEC07A17EE903A591C01D09C423A
:1038C0001FD3B0EE680A1EF0B1F9FDEEC07A17EE14
:1038D000903A5A1C01D0A34213D8B0EE480A1EF009
:1038E000A5F9FDEEC07A17EE900A431C0BD0A0425A
:1038F0008CBF00200120BDEC048B10BD40F2DC54D5
:10390000D3E70020F7E70120F5E790F832103C30CC
:1039100000F090BAB0F93030012B10B5044604DD48
:1039200090F834103C3000F085FAB4F9300010BD46
:1039300038B590F91530991C044640D11AF0C0FDF5
:10394000A36AC01AC82828DD04F13C0000F0D5FAAB
:1039500040B394F8C23094F8C300E37794F8C130D0
:1039600094F8C41094F8C65084F8213094F8C53007
:1039700094F8C020A07784F8201084F8225084F8AE
:103980002330C0B9C9B9002D18BF2B4684F82420B4
:1039900084F825301AF094FDA0622046BDE8384036
:1039A000FFF7F4BD40F20113E38301224FF001332E
:1039B00023621346EAE70346E8E70B46E6E7DBB295
:1039C000012BEAD8836BB3F90C00002809DB1AF04D
:1039D00043FD94F915301A1A5342534184F82530A7
:1039E000DBE70020F5E737B502460C4692F91230C6
:1039F000B2F90E50191E00F13C0092F8323018BF97
:103A0000012154B1B2F90C40CDE9005492F91320D0
:103A100000F0DAF8012003B030BDCDE900540622F1
:103A2000F6E737B590F91330062B044603D090F92A
:103A30001430062B26D1B4F90E3094F91210CDE9CA
:103A40000033003904F13C0518BF012194F83230ED
:103A50000622284600F0B8F84FF47A701AF034FDC8
:103A6000B4F90C3094F912100193B4F90E300093AC
:103A7000003994F8323094F9132018BF01212846F8
:103A800000F0A2F803B030BDF0B52E4D85612E4D8B
:103A900005634FF6FF7585862C4D056000244FF0B9
:103AA000FF350426C0E91254C0E9105580270125CE
:103AB000C0E91D54C0E91444C0E91644C0E91964C2
:103AC000C0E91B44C0E91F44C0E92156C0E9237482
:103AD0008480C0F81D40C0F8214080F825408462F1
:103AE0000466C0E92546C0E92755C0E929571E25C7
:103AF000C0E92C540C25C0E92F54C0E93444C0E976
:103B00003644C0E93844C0F8AC40C0F8C440A0F81E
:103B1000C84080F8CA40A0F8CC40C0F8E84080F81F
:103B2000EC400B4C01778263C0F8B860C0F8F440F9
:103B3000821D03F1100153F8044B42F8044B8B42F1
:103B4000F9D1F0BDAE47E13D0100FFFFB8650208C5
:103B5000B81E053E37B50D46044611461A46A5F176
:103B60000C030020012B84F8B000C4F8B45015D821
:103B70009FED0B7ADFED0B7ABDF91C300D2D08BFE0
:103B8000F0EE477AC4ED2E7A04F1BC000093BDF943
:103B9000183002F031F984F8B000012003B030BDD4
:103BA0009A99993DB81E053E70B500F1BC0441F0EC
:103BB00080012046164602F0C9F9314605462046E6
:103BC00002F010FA284670BD2DE9F74F90F8B0A02A
:103BD00004460E4693461F46BAF1000F00F0E680F9
:103BE000D0F8B4300C3B012B00F2168100F1BC057B
:103BF000284602F013F9D4F8B800FCF79DFC024601
:103C00000B468AA1D1E90001FCF718FEFCF7E4FF9E
:103C1000FCF792FC80460D988946FCF77BFC804BB4
:103C20000022FCF70BFE42464B46FCF707FE7D4B9D
:103C30000022FCF7D9FC41EC100B1FF081FA0C9824
:103C40008DED000BFCF766FC754B0022FCF7F6FDD2
:103C500042464B46FCF7F2FD724B0022FCF7C4FCD7
:103C600041EC100B1FF06CFA6F4B51EC100B002263
:103C7000FCF702FBFCF768FF6B4B002280F30508A2
:103C8000DDE90001FCF7F8FAFCF75EFF4FEA0828CF
:103C900080F30500636908EB000202F5802293427D
:103CA00007D0626110212046FFF77EFF284602F010
:103CB00007F9226DA369934207D0A2611121204622
:103CC000FFF772FF284602F0FBF8626DE36993424A
:103CD00007D0E26113212046FFF766FF284602F075
:103CE000EFF8A26D236A934207D022621521204685
:103CF000FFF75AFF284602F0E3F8D4F8B4300C2B53
:103D000058D1D4E917131A04E36E02EB01221A44C6
:103D1000636E02EB8342236F02EBC342A36E02EB9E
:103D20000352636A934207D0626270212046FFF714
:103D30003BFF284602F0C4F8D4F8B430A6640C2B3C
:103D400052D1A36AE26A03EB067303EB0213226B00
:103D500003EBC213626B03EB4233A26B03EBC23380
:103D6000E26B03EB4243226C03EB8243626C03EB96
:103D7000C2432360FF2F09D022686C2102EB076247
:103D80002046FFF711FF284602F09AF8BBF1060F14
:103D900023690CBF05220122934204D02261002135
:103DA0002046FFF701FF284602F0B6F8504603B060
:103DB000BDE8F08F0D2BBFD1D4E917131A04636F40
:103DC00002EB01221A44636E02EB8342A36F02EB03
:103DD000C342A36E02EB0352E36F02EB0362D4F81B
:103DE000803002EB03729CE70D2BC3D1A36AE26A19
:103DF00003EB067303EB0213226B03EBC213A26BFC
:103E000003EBC233226C03EB8243626C03EBC243CD
:103E1000E26C03EB0253ACE74FF0000AC6E700BFC9
:103E200000408F40000040400000F03FCDCCCCCCA3
:103E3000CCCCD43FF8B590F8B05004460F468DB3C3
:103E4000D0F8B4300C3B012B44D800F1BC0630460E
:103E500001F0E4FFD4F8B4300C2B25D1D4E90B23C6
:103E6000DB0103EB0213A26A1344626B03EB4233E0
:103E7000A26B03EBC233E26B03EB4243226C03EB16
:103E80008243626C03EBC243A26C03EB02732360B8
:103E900022686C2102EB07622046FFF785FE304660
:103EA00002F03AF82846F8BD0D2BF1D1D4E90B23E6
:103EB000DB0103EB0213A26A1344A26B03EBC233D0
:103EC000226C03EB8243626C03EBC243E26C03EBB4
:103ED0000253D9E70025E5E770B500F1BC0501F014
:103EE0007F012846144602F031F82168064628462C
:103EF00002F078F82060304670BD2DE9F74F90F859
:103F0000B0600546002E60D0D0F8B4300C3B012BD9
:103F10004FF000045BD800F1BC07384601F07EFF8B
:103F200001AA6F2128460194FFF7D6FF8046384644
:103F300001F0C6FF01AA6F2128460194FFF7CCFFCC
:103F4000019C14B9B8F1000F34D04FEAD47BC4F30C
:103F5000807AC4F34079C4F30078C4F3C06EC4F32C
:103F6000806CC4F34066C4F30060C4F30441C4F33E
:103F7000C032C4F3090385F88B0085F884B0384655
:103F800085F885A085F8869085F8878085F888E093
:103F900085F88AC085F88960A5F88C1085F88E2090
:103FA000A5F8903001F0B8FF201E18BF012003B023
:103FB000BDE8F08FB346B246B146B046B646B44609
:103FC0002046214622462346D5E73046EFE72046E5
:103FD000EDE700000000000082B02DE9F04F89B04D
:103FE00012A981E80C009DF84AA0BDF948000AF129
:103FF000FF33012B9CBF00F1FF300AF10C0AFCF7E4
:1040000089FA3B4B002204460D46FCF717FC41ECB5
:10401000100B1FF011F8374B00222046294659ECAF
:10402000108BFCF70BFC41EC100B1FF005F828A3DC
:10403000D3E900232046294657EC106BFCF7D4FA4D
:1040400041EC100B1EF0F8FF504655EC104BFCF7FE
:1040500061FA294B0022FCF711F91FA3D3E90023D1
:10406000FCF7C2FA41EC100B1EF0E6FF42464B464D
:1040700000204FF080415BEC10ABFCF7FDF83246BE
:104080003B46FCF7FBF822462B46FCF7F7F8524676
:104090005B46FCF7F3F804469DF84B000D46FCF731
:1040A00039FA02460B4620462946FCF7E7F80CA3EE
:1040B000D3E90023FCF7E2F89FED0B1B41EC100B5A
:1040C00009B0BDE8F04F02B0704700BFAFF3008009
:1040D0000000000000D4764061545227A0993E4071
:1040E00000000080A2423A410000000000000000F1
:1040F00000005940000079400000F03F82B02DE9F7
:10410000F04F91B01AA981E80C001CAB04460FCB0C
:104110008DE80F001AAB20460CCBFFF75DFFDDE901
:104120001C455BEC10AB224FDFF8889000264FF067
:1041300000081F4B002220462946FCF7DBFCA8B9EB
:10414000DFF86C901B4F4FF0000800260022002380
:1041500020462946FCF7BAFCC8B94BEC10AB45EC3D
:10416000114B11B0BDE8F04F02B0704732463B46EC
:1041700020462946FCF780F8424604460D46504644
:1041800059464B46FCF77AF882468B46D1E74246C1
:104190004B4620462946FCF771F8324604460D4648
:1041A000504659463B46FCF767F882468B46CDE7BA
:1041B000000038400000F03F2DE9F047764B86B014
:1041C0000022824651EC100BFCF758F841EC100B22
:1041D0001EF032FF55EC104B5DA3D3E900232046BF
:1041E0002946FCF791FC58B35BA3D3E90023204692
:1041F0002946FCF741F85AA3D3E90023FCF71EFB3C
:10420000FCF7A2FCFCF786F9644B002206460F4639
:10421000FCF7EAF941EC100B1EF00EFF604B59EC75
:10422000108B002220462946FCF728F832463B46F0
:10423000FCF724F842464B46FCF71EF804460D46B0
:1042400049A3D3E9002320462946FCF717F848A3E1
:10425000D3E9002304460D46FCF70EF846A3D3E944
:104260000023FCF7EBFA41EC100B1EF0E5FE57ECD7
:10427000106B41A3D3E9002330463946FCF7B4F96B
:1042800041EC100B1EF0D8FE204653EC102B2946B3
:10429000FBF7F2FF3AA3D3E9002380468946FCF7F7
:1042A000CDFA41EC100B1EF0C7FE55EC104B34A3B9
:1042B000D3E9002320462946FCF796F941EC100B80
:1042C0001EF0BAFE00220023404649468DED000B49
:1042D000FBF7D4FFDDE90023FBF7CEFF41EC100B29
:1042E0001EF0AAFE51EC100BFCF756FC00228AF8D7
:1042F00003002C4B20462946FCF7E8FB0022F8B1CE
:10430000274B20462946FBF7B7FFFCF745FCC0B218
:1043100002288AF8020015D91BA3D3E900233046EE
:104320003946FBF7A9FFFCF70FFC00B2AAF8000022
:10433000002200235046CAE9022306B0BDE8F087F8
:10434000194BDEE712A3D3E90023E8E7AFF30080BF
:10435000000000008C8A414100000040D07D3C41BB
:104360000000000088D5E1400000000000D0974028
:104370006666666666865E400000000000D4764091
:1043800061545227A0993E4000000000006CB240EA
:1043900000000000006BB2400000E03F0000D03F92
:1043A0000000F03F00002B4000002A402DE9F04FB4
:1043B00057EC106B55EC114BDFF8949085B08246AA
:1043C0008B464FF00008214B002220462946FCF77F
:1043D00091FBC0B9DFF874904FF000080022002371
:1043E00020462946FCF772FBF0B9504647EC106BAB
:1043F00045EC114B5946FFF7DFFE5046CAE902452E
:1044000005B0BDE8F08F114B002220462946FBF78E
:1044100033FF424604460D46304639464B46FBF7CD
:104420002DFF06460F46CEE742464B46204629461C
:10443000FBF724FF064B04460D4630463946002262
:10444000FBF71AFF06460F46C8E700BF00003840DA
:104450000000F03F06292DE9F341044662D1D0F86F
:10446000B8201AB1002002B0BDE8F081416880F8A0
:104470006C20032940F23A6314BF50214121A0F877
:10448000683080F86A1003F03A03232180F86B103B
:10449000A3F13A020421C0F8B810D2B2012A74D8AC
:1044A000A26E22F07F4222F0FF02B2F50C5F62D0D2
:1044B0003B2B0CBF01230023237068D104F1680754
:1044C0003846FBF76DFEC5B26E1EF6B2042E60D9FB
:1044D000A6F10308384600220346663B10F8011F88
:1044E0001B1B0A449845D2B2F6DC26442D4901A88C
:1044F0001AF01CFBA04496F8673084F8BC309DF895
:10450000042098F868309A4243D19DF8052096F827
:1045100066309A423DD1043D54FA85F5002385F872
:10452000683034E0A1F10A03DBB2162B04D81E4A2E
:1045300042FA03F3DB0795D5D4F8B8304E2B20DCD4
:10454000D4F8B8002518013023180022232985F853
:104550006810C4F8B80083F8682083D194F86830F4
:104560000128A3F13A02D2B298DC012A0DD895F8BD
:104570006820232A94D10023C4F8B83084F8683026
:1045800070E74E23C4F8B830DAE700232370012027
:1045900069E7064BA366002384F86C300423C4F853
:1045A000B830F4E7E0650208F6FFBFFF3A063023B3
:1045B000B0F86930838200228275436923F07F431B
:1045C00023F0FF03B3F50C5F08BF4275143070474A
:1045D000D0F8B8200023042A10B50376044600F171
:1045E000180306DD00F16B01043A18461BF029FBA5
:1045F0000346D4F8B820144400222275184610BD92
:10460000024B90F8BC201A7018467047000000203A
:10461000D0F8B830ABB1C21892F86720232A06D17F
:10462000012B02BF0023C0F8B83080F86830D0F802
:10463000B830184490F86700A0F12303584258415D
:104640007047184670470023C0F8B83080F86830CB
:10465000012070470020704730B590F810410246A5
:10466000002354FA83F1CDB252FA81F1D8B2097C19
:1046700041B192F81111A94204D00133B3F5807F02
:10468000EFD1FF2030BD000070B500234FF47A72E7
:10469000174D184C0374C0E90132174A2B78026099
:1046A000227842FA03F1C90706D40121037401FA02
:1046B00003F31343237070BD591CC9B242FA01F6CB
:1046C000F607297003D4012301748B40F1E7991C8C
:1046D000C9B242FA01F6F6075DBF01238B401A43C7
:1046E000033329705ABF017422702B70E3E700BFB7
:1046F000A1060020B8070020F065020838B5037C49
:1047000004460D4613B90A4818F084FA237C012B9D
:1047100004D108480622294618F002F9237C022B0E
:1047200005D129460448BDE8384001F081BA38BDBA
:1047300058250020A4060020E007002010B5037CC7
:10474000044613B9084818F067FA237C012B02D1FC
:10475000064818F0BFF8237C022B04D1BDE81040B6
:10476000034801F06EBA10BD58250020A4060020B1
:10477000E007002007B524230093C222C321034889
:1047800017F0E0FF03B05DF804FB00BFA4060020B3
:1047900010B4037C0C4623B911485DF8044B18F0A3
:1047A00086B9012B04D10F485DF8044B17F0DDBE2C
:1047B000022B12D10C4A92F81332D118013303F0B4
:1047C0007F0382F813321A44002381F8124101203A
:1047D00082F812315DF8044B70474FF0FF30F9E773
:1047E00058250020A4060020E0070020F0B403466E
:1047F0000D461B7C10461BB9F0BC124818F06AB974
:10480000012B03D1F0BC104817F006BF022B15D0C6
:104810004FF0FF30F0BC704794F81332AF5CE618ED
:10482000013303F07F0384F81332234486F81271B6
:10483000013283F812118242EEDBEBE70022034CD7
:104840001146F8E758250020A4060020E0070020C4
:1048500008B5037C23B9BDE80840094818F05EB9E3
:10486000012B04D1BDE80840064817F05BBE022BBF
:1048700003D10548FFF7F0FE08BD0020FCE700BFAC
:1048800058250020A4060020E0070020037C13B96F
:10489000074818F049B9012B02D1064818F082B830
:1048A000022B02D1044801F0ACB94FF0FF30704741
:1048B00058250020A4060020E007002010B5037C46
:1048C00023B9BDE810400C4818F094B9012B04D16D
:1048D000BDE81040094817F02DBE022B09D1084C45
:1048E0002046FFF7B9FE20B194F810311C44207C1B
:1048F00010BD4FF0FF30FBE758250020A406002034
:10490000E007002010B5037C044613B9054818F0F1
:1049100077F9237C012B04D1BDE81040024817F041
:10492000EDBE10BD58250020A40600202DE9F0435F
:104930002DED028BB0EE408AF0EE608A0F4687B014
:104940000646252138461BF034F90546002D45D092
:104950006878662847D02E2809D1AB78303BD9B289
:104960000929F5D8EB78662BF2D104243DE03038E4
:10497000C0B20928ECD8AB782E2BE7D1EB782F2BDF
:10498000E4D9392BE2D82A79662ADFD1303BD9B273
:10499000052401AA40B2B0EE480AF0EE680A18F009
:1049A00055F90023EA1B5FFA83F9914503F10103EE
:1049B0001DDB4FF0000801A8FBF7F2FB09EB08072D
:1049C0008045FFB218D33F1BFFB22846FBF7E8FB38
:1049D0003B198442DBB21AD30022F25407B0BDEC7B
:1049E000028BBDE8F083022400210020D1E717F8F4
:1049F000091006F80910D6E708F118036B4408F10E
:104A0000010813F8143CF3555FFA88F8D3E72A5DE0
:104A1000F2540134E4B2D8E72DE9F0478EB01E46D7
:104A2000002355EC104B0F46ADF81C3072B100223C
:104A3000002320462946FCF749F8002874D005F1E8
:104A400000435B491D4607A81BF07BF9032E6DD17F
:104A500051A3D3E9002320462946FBF70FFC044667
:104A60000D4645EC104B1EF0E7FA59EC108B204632
:104A700042464B462946FBF7FFFB4E4B0022FBF715
:104A8000B3FD41EC100BCDE904011EF0D5FADDE9D0
:104A9000040153EC102BFBF7EFFB464B0022FBF716
:104AA000A3FD454B08AA04460D4603F1100E92469D
:104AB000186859689446ACE80300083373456246A9
:104AC000F6D118689B88CCF800004946ACF8043051
:104AD0004046FCF739F88046DDE90401FCF734F87C
:104AE000032E814626D145EC104B1EF0A5FA204638
:104AF00053EC102B2946FBF7BFFB29A3D3E9002376
:104B0000FBF772FDFCF720F8294602902046FCF7DF
:104B10001BF84346CDE9009007AA514638461AF0E3
:104B200005F80EB0BDE8F08724498CE71EA3D3E951
:104B3000002390E7022E0FD100238DF83030294654
:104B40002046FCF701F84346CDE9009007AA5146FC
:104B5000384619F0EBFFE4E7012E11D100238DF860
:104B600030302E238DF82B3031238DF82E30204617
:104B70002946134B0022FBF761FE04460D46DEE793
:104B8000002EDCD10090434607AA514638468DF8E6
:104B90002B6019F0CBFFC4E7094890169BD94D3E16
:104BA000000000000088C340F78F85E81038223FDE
:104BB0001466020800004E401866020816660208D5
:104BC00000001840000000002DE9F04F8FB017469C
:104BD000002255EC104B9DF86080ADF81C200E466D
:104BE00073B10022002320462946FBF76FFF0028FF
:104BF0006DD005F1004362491D4607A81BF0A1F8DE
:104C0000B8F1030F65D15AA3D3E900232046294602
:104C1000FBF734FB82468B464BEC10AB1EF00CFAD4
:104C200055EC104B504622462B465946FBF724FBC9
:104C3000544B0022FBF7D8FC82468B464BEC10AB62
:104C40001EF0FAF9504653EC102B5946FBF714FBB3
:104C50004C4B0022FBF7C8FC4B4BCDE9040108AAE2
:104C600003F1100E186859689446ACE80300083345
:104C700073456246F6D118689B88CCF80000B8F1FD
:104C8000030FACF8043028D00023B8F1010F8DF8E1
:104C9000303050D017B133238DF82430B8F1020FE3
:104CA00046D129462046FBF74FFF0446DDE90401C3
:104CB000FBF74AFF594601905046FBF745FF234654
:104CC000009007AA08A9304619F030FF30E02F49BC
:104CD00093E729A3D3E9002398E79DED040B1EF089
:104CE000ABF9DDE9040153EC102BFBF7C5FA284BB7
:104CF0000022FBF779FC804689469FBB2046294667
:104D0000FBF722FF494604464046FBF71DFF029091
:104D1000DDE90401FBF718FF594601905046FBF707
:104D200013FF2346009007AA08A9304619F0FEFE9B
:104D30000FB0BDE8F08F8DF82B3017B133238DF80D
:104D4000243029462046FBF7FFFE594604465046CC
:104D5000FBF7FAFE2346009007AA08A9304619F08F
:104D6000E5FEE5E733238DF82430C7E7AFF3008095
:104D7000052D1AEE00A8823EF78F85E81038223FF5
:104D80001466020800004E402E66020816660208ED
:104D900000408F4070B508460C4616461D46FBF78E
:104DA000FFF900B208B9002070BD0628FBDC00281E
:104DB0000CDD23782B2B15D02D2B13D00023E25C98
:104DC000303A092AEFD801339842F8DC204619F02E
:104DD000E8FD00F5FF437F33B3F5803FE3D2308039
:104DE0000120E1E7002DDED00023ECE72DE9F74FAD
:104DF0001578002306460F461446ADF8063025B94F
:104E00000024204603B0BDE8F08F1046FBF7C8F938
:104E10000628F5D82D2D33D101344FF0FF383A2133
:104E200020461AF0C6FE054680BB2146002301AA93
:104E30003046FFF7AFFF04460028E1D0BDF9060079
:104E4000FBF768FB1F4B0022FBF7F8FC8246BDF91D
:104E500004008B46FBF75EFB02460B465046594664
:104E6000FBF70CFA824640468B46FBF753FB0246A3
:104E70000B4650465946FBF7B7FBC7E90001C0E7B0
:104E80002B2D08BF01344FF00108C8E74FF000098F
:104E900005F8019B2846FBF783F90228B0D14B4661
:104EA0000DF1060229463046FFF774FF0028A7D00F
:104EB000BDF906302D2BB8D01E2BB6D0002BB4D0A8
:104EC0009EE700BF00004E4013B514461278ADF8BF
:104ED00006200DF10602FFF75DFFBDF80620BDF9C3
:104EE0000630FF2A8CBF0020237002B010BDF8B539
:104EF00008460E4617461C46FBF752F900B200283A
:104F00000EDD35782B2D12D02D2D10D000232E2D17
:104F10001AD01A46303D092D11D8013398420ADCC7
:104F2000304619F03BFD87ED000B0120F8BD44B978
:104F300035782346EBE7F55C2E2DEBD122B100202E
:104F4000F4E700231A46E8E70122E6E70000000044
:104F50002DE9F04F074687B08A4600200021CDE9B1
:104F600004011E461578202D144602F10102F9D0E5
:104F70002046FBF715F90D2884BF002363732046F4
:104F8000FBF70EF9A6F102095FFA89F9B9F1010FF1
:104F900000B208D808280AD0092808DC00252846CD
:104FA00007B0BDE8F08F012E01D10728F6D1637854
:104FB0008DF805304FF0000843466A4601A938468F
:104FC0008DF804508DF80680FFF7E4FE0028E5D048
:104FD000A3783A2BE2D1E3788DF8083023798DF865
:104FE00009300DF10202434602A938468DF80A80C5
:104FF000FFF7D0FE05460028D0D0B9F1010F5DD8EB
:1050000063793A2BCAD1434604AAA11D3846FFF75B
:105010006EFF0028C2D0BDF80030BDF900B0172BDC
:10502000BCD8BDF80230BDF902803B2BB6D80024B5
:10503000DDE904670022002330463946FBF746FDD0
:105040000028ABD130A3D3E9002330463946FBF723
:105050005BFD0028A2D14046FBF75CFA284B0022FA
:10506000FBF7ECFB804658468946FBF753FA0246AD
:105070000B4640464946FBF701F9804620468946E3
:10508000FBF748FA1F4B0022FBF7D8FB02460B4602
:1050900040464946FBF7F2F817A3D3E900238046C0
:1050A000894630463946FBF7C9FB02460B46404667
:1050B0004946FBF7E3F8CAE9000170E7012EAAD1DF
:1050C00063792E2B7FF46AAFBDF80030A479BDF967
:1050D00000B0172B3FF662AFBDF80230BDF9028079
:1050E0003B2B3FF65BAF303CA4B2092C3FF656AFEA
:1050F00024B29DE7AFF30080000000000020AC4028
:1051000000004E4000C082409CA223B9FCFF4D40ED
:1051100070B5032304460D461646FFF719FF70B914
:105120000223324629462046FFF712FF38B932469D
:10513000294620460123BDE87040FFF709BF012042
:1051400070BD0000000000002DE9F04F074687B059
:105150008A4600200021CDE904019DF84060984670
:105160001578202D934602F10102F9D05846FBF73D
:1051700017F80D2884BF00238BF80D305846FBF735
:105180000FF8A6F102095FFA89F9B9F1010F00B22F
:1051900008D809280CD00A280ADC0024204607B0C9
:1051A000BDE8F08F012E03D1062802D00928F4D1E2
:1051B0000026B8F1000F00F093802D2D00F08D80B7
:1051C0002B2DEAD101259BF801308DF804309BF896
:1051D00002308DF805306A46002301A938468DF863
:1051E0000630FFF7D7FD0028D7D00BF1030B9BF853
:1051F000003003F0EF022A2A01D0DF2BCDD19BF83B
:1052000001308DF808309BF802308DF809300DF12F
:105210000202002302A938468DF80A30FFF7BAFDD2
:1052200004460028B9D0B9F1010F72D9B8F1000FC6
:10523000BDF900B015BF6FF0590200225A234FF498
:10524000B4739345A9DB9B45A7DCBDF80230BDF9DB
:1052500002603B2BA1D8DDE90489002200234046EF
:105260004946FBF733FC002897D13AA3D3E9002342
:1052700040464946FBF748FC00288ED13046FBF7F4
:1052800049F9334B0022FBF7D9FA064658460F4638
:10529000FBF740F902460B4630463946FAF7EEFF77
:1052A00029A3D3E9002306460F4640464946FBF7AB
:1052B000C5FA02460B4630463946FAF7DFFF064686
:1052C00028460F46FBF726F902460B46304639467C
:1052D000FBF78AF9CAE9000160E74FF0FF3572E792
:1052E0009BF801308DF805309BF802308DF80630C0
:1052F0006A46434601A938468DF804508DF8078068
:10530000FFF748FD00283FF448AF0BF1030B0125E0
:105310006DE7002E8AD19BF803303A2B0AD10BF1AE
:105320000401002304AA3846FFF7E1FD00287FF4BA
:105330007DAF32E79BF80430272B7FF42EAF0BF1C3
:105340000501EEE7AFF30080000000000020AC4054
:1053500000004E401D5A643BDFFF4D40F7B54FF053
:10536000030CCDF800C004460D4616461F46FFF755
:10537000EBFE10B1012003B0F0BD022300933246D2
:105380003B4629462046FFF7DFFE0028F2D10123E5
:10539000009332463B4629462046FFF7D5FEEAE712
:1053A000012070470020704770B50023058A838470
:1053B0009AB2AA42818C03D3B1FA81F0400970BD40
:1053C000D408066A345D02F0070244FA02F2D207FA
:1053D00044BF013181840133EAE710B50446084631
:1053E000A18052B9A362003B18BF012384F82D307D
:1053F000012322822383012010BDA362003B18BF3A
:10540000012384F82D30CB08013321822383002926
:10541000F1D013F0EEFA6061208B13F0EAFAE0614C
:10542000208B13F0E6FA00232062FF20218B9AB232
:1054300091420AD800231846218B9AB29142DAD9B8
:105440009AB2216A01338854F6E79AB2E1690133CE
:105450008854EBE7038A2DE9F0410446002B58D02D
:1054600090F82F30002B54D10368DB68984707462B
:1054700000284ED114264FF00108E389228A013317
:105480009BB29A42E38107D894F82E300BB184F88E
:105490002F80E78184F82E8094F82D305BBBE28961
:1054A000216AD30802F00702CB5C134103F0010329
:1054B000E589E169EA0805F007008A5C024102F02B
:1054C000010203B90AB3002084F82E001BBB02B30B
:1054D000236866691B692946204698477055E38909
:1054E000E069D908012203F007039A40435C23EAEC
:1054F000020343540DE018F0E3FF236BC01A0028A9
:10550000CDDA84F82E700023D2E7013E16F0FF06B4
:10551000B3D1BDE8F0812689B5FBF6F306FB135342
:105520009BB27BBB2B469AB2501B80B286421BD8E3
:10553000236862699F692A44F3B229462046B84726
:105540000022012790B28642E3D9E389256A99189F
:10555000C910034403F00703685C07FA03F320EA69
:1055600003036B540132EDE7278ABB42184609DA80
:10557000C01002F00702085C40FA02F2D20703F101
:105580000103D0D50126D3E7036870B59B680D4EA3
:105590000446984718F094FF0546236820469B6808
:1055A0009847014668B9236820465B689847012000
:1055B00018F08AFF18F084FF401BB042EDDD012394
:1055C000A37170BD20BF0200038A2DE9F04104469B
:1055D0000D460BB1037B33B12368294620461B6976
:1055E000BDE8F0411847C369CE0801F007079B5D8D
:1055F0003B41DB070DD503681B6998476369585524
:10560000E16901228B5DBA4023EA02038B55BDE8B4
:10561000F0814369585CFAE7002370B580F82F30B9
:10562000037B04460D46164623B1437B13B903683A
:105630005B699847238AB3B9637B73B9227B23687C
:1056400032B91B69294620469847B04205D02368E5
:105650005B69324629462046984718F031FFA36A15
:105660001844206370BD29462046FFF7ADFF8642EF
:10567000F3D063695E55EA08206A05F00705012347
:10568000815CAB40DBB219438154E069815C21EA63
:1056900003038354E1E7000073B50A4604460D4650
:1056A0006846084919F042FA0026A388B1B28B4235
:1056B00001D802B070BD2A462046FFF7ADFF013683
:1056C000F3E700BFE065020870B500250446857168
:1056D000FF21FFF7E1FF2046FFF756FF0123237369
:1056E0002E46A388A9B2013B994216DB0025294624
:1056F00020462573FFF7D0FF2046FFF745FF012323
:105700002373A388A9B2013B99420EDB00232373C4
:105710000EB10123A371A07970BD2046FFF754FF9D
:10572000FF2818BF01360135DBE72046FFF74CFFA5
:1057300000B101360135E4E7FFF746BFFFF744BF8C
:10574000F8B5141EB8BF644207460E46B8BF24B26F
:105750000025731999B22BB29C4201DC0120F8BDDF
:105760003846FFF731FF01350028F2D00020F6E778
:10577000002B2DE9F04106460D4617460FDB0B4482
:105780009CB2A5421FD029463046FFF71DFF05F108
:1057900001081FFA88F807F8010B4546F1E75B425C
:1057A0001CB24FF000080FFA88F305EB08019C4289
:1057B00089B208DD3046FFF707FF07F8080008F157
:1057C00001080028EFD1BDE8F08107B502230DF1F3
:1057D0000602FFF7CDFFBDF8060003B05DF804FB3D
:1057E00007B504230DEB0302FFF7C2FF019803B0D6
:1057F0005DF804FB012370B5067B03730D460021A1
:105800000446FFF7EDFF431B5842584184F82C0033
:10581000267370BD002B2DE9F04107460E46154654
:105820000FDB0B449CB2A64221D006F101083146A1
:1058300015F8012B1FFA88F83846FFF7EDFE4646AB
:10584000F1E75B421CB2551E4FF000080FFA88F3D7
:1058500006EB08019C4289B209DD15F8012F384694
:10586000FFF7DAFE2B7808F10108002BEED1BDE836
:10587000F08137B5012385898381042301910DEBE4
:10588000030200210446FFF7C5FFA58103B030BD28
:1058900010B5044618F014FEE36BC01AC00F10BD1B
:1058A0000368C9B21B681847F8B504460F46154689
:1058B0001E4623682046DB6898470028F9D194F8F3
:1058C0003810606B0EF044F9606B390AFFF7E8FF9F
:1058D000606BF9B2FFF7E4FF2E44AE42606B06D175
:1058E0000EF05AFA18F0ECFD0A30E063F8BD0368D8
:1058F00015F8011B1B689847EFE770B504460D4685
:10590000164623682046DB6898470028F9D194F8AA
:105910003810606B0EF01CF9606B290AFFF7C0FFAE
:10592000606BE9B2FFF7BCFF606B036831461B6830
:105930009847606B0EF030FA18F0C2FD0A30E06351
:1059400070BD38B504460D4623682046DB6898478D
:105950000028F9D194F83810606B0EF0F9F8606BFC
:10596000290AFFF79DFFE9B2606BFFF799FF606BB3
:105970000EF012FA94F83810606B01220EF009FA5A
:10598000606B03681B69984720B1606B03685B69B3
:105990009847C0B238BDF0B585B016460B9D9DF84E
:1059A00030709DF828C0CDF800C0CDE901570446FD
:1059B000FFF713FD0EB10823A3602846656384F842
:1059C000387000210EF0ACFA94F8381028460EF02A
:1059D000BFF828460EF0E0F9B0FA80F0400905B0B3
:1059E000F0BD70B504468669257A00688DB118F05F
:1059F00019FCD4E9033299188142D8BF01269B1AB9
:105A00008342C8BF00266068A661831B5842584184
:105A100070BD002802DB18F01FFD0546636AAB422B
:105A200003D018F04DFDC4E9095018F049FDA36AF0
:105A3000C01A23698342D8BF666AE4E770B5057A65
:105A400086690446A5B90068002802DB18F004FD49
:105A50000546636AAB4203D018F032FDC4E9095031
:105A600018F02EFDA36AC01A23698342B8BF666A84
:105A7000A66170BD10B504460068237A4BB118F0DA
:105A8000D1FBE3689842D4BF00200120A06160628E
:105A900010BD002802DB18F0DFFCF7E71846F5E739
:105AA00070B504460025C3F349060846AE421146C8
:105AB00003F001026260C3F3C92314BF01222A4626
:105AC000C4E90655C4E90855A5622060E660236173
:105AD000227206D0F218B2F5806F0BDA9E420BDB11
:105AE0002361002801DB18F021FC2046FFF7C2FFEC
:105AF000204670BD2B46F3E72561F2E72DE9F04122
:105B000015464A1C04460F469DF818001E4603D051
:105B1000731C02D100201BE0D0B12378072BF9D8E9
:105B2000B6F5001FF6D215B1AB1E012BF2D82C2012
:105B300012F05DFF33462A4639468046FFF7B0FF34
:105B4000237804EB83020133D8B2C2F804802070BA
:105B5000BDE8F0810346084619B153F82100FFF76C
:105B600040BF7047F8B5084F044606460025237825
:105B7000AB4200DCF8BD56F8040FFFF75FFF384674
:105B800001F002F80135F2E7180C0020014B002269
:105B90001A707047BC070020036810B51B690446E3
:105BA000984720B194F810311C44207C10BD4FF070
:105BB000FF30FBE7704790F81332C218013303F04F
:105BC0007F0382F8121180F813321844002380F802
:105BD0001231012070472DE9F04106460F46154667
:105BE0000024A54203DCA8464046BDE8F0813368A6
:105BF000395D1B683046A04698470028F4D0013430
:105C0000EFE7036810B51B690446984768B194F83C
:105C10001131234400221A7494F81031E218107CD8
:105C200010B1013384F8103110BD4FF0FF30FBE7A5
:105C3000002380F81232A0F8103180F8123103747A
:105C400070477047F8B5134C00254FF47A73C4E9D8
:105C50000153FC22104B2360294604F114002561F6
:105C60001AF009F80D4BA4F810517F261F7884F81C
:105C700012713246294604F2131019F0FCFF324625
:105C8000294604F2931084F8927119F0F4FFA4F8F5
:105C90001252F8BDE007002070660208E2730208A5
:105CA000FE2AF8B506460F4615460DDD0020F8BD64
:105CB0003368395D1B68304698470028F6D00134B8
:105CC000A542F5DC0120F2E70024F9E790F816126E
:105CD000034600200A1853FA82F292F8122102B900
:105CE00070470130F6E790F816228118034691F8C4
:105CF000120118B1013283F816227047FF20704755
:105D000090F81632184490F81201002808BF4FF09E
:105D1000FF3070472DE9F04104460E4618F0D0FBE5
:105D200094F81051DFF84080013D0746EDB294F839
:105D30001131AB420BD0E2180133DBB2167484F898
:105D400011311C44002323740120BDE8F08140463A
:105D500000F01AFF18F0B4FBD4F81832C01B9842B8
:105D6000E5D90020F1E700BF180C002070B504460B
:105D700018F0A6FB094E0546304600F005FF94F8E2
:105D8000103123441B7C002BF6D118F099FBD4F87A
:105D90001822431B9342EFD370BD00BF180C0020A4
:105DA00038B5124C00254FF47A73C4E90153FC2234
:105DB0000F4B2360294604F11400256119F05BFFA5
:105DC0000C4BA4F810511B7884F81231FF2229469D
:105DD00004F2131019F04FFF5023A4F8125284F864
:105DE0001652C4E98635A4F8145238BDF4090020CF
:105DF0009C660208E273020810B54180BDF90840B4
:105E0000048001318280C38005D0013203D0581C48
:105E100018BF012010BD0020FCE7000070B504464B
:105E2000B0F90600002802DB012118F07FFAB4F96E
:105E30000600002802DB012118F0D6FA1D4E1E4D87
:105E400071682B681D4AB3FBF2F273685B1A9A42C1
:105E5000FBDCB4F90400012118F068FAB4F904007D
:105E6000012118F0C1FAB4F90000002118F05EFA1F
:105E70000121B4F9020018F059FA71680D4E2B682F
:105E80000E4AB3FBF2F273685B1A9A42FBDCB4F978
:105E90000600002802DB002118F0A6FA7168054808
:105EA0002A68064BB2FBF3F243685B1A9A42FBDCAA
:105EB00070BD00BF001000E0F801002040420F005C
:105EC00038B50446B0F90600002802DB012118F0BD
:105ED0008BFA0E490E4D48682B680E4AB3FBF2F25E
:105EE0004B681B1A9A42FBDCB4F90600002802DB5F
:105EF000002118F079FA05492A684868054BB2FB79
:105F0000F3F24B681B1A9A42FBDC38BD001000E02C
:105F1000F801002040420F00B0F90600002808B543
:105F200002DB012118F060FA0549064B48681A683F
:105F3000054BB2FBF3F24B681B1A9A42FBDC08BD1F
:105F4000001000E0F801002040420F002DE9F0476A
:105F5000DFF88490DFF8848004460F46072600258A
:105F6000B4F90400DFF878A0002118F03DFA47FAF0
:105F700006F101F00101B4F9020018F035FAD9F880
:105F80000410DAF80030B3FBF8F2D9F804305B1AE9
:105F90009A42FADCB4F90400012118F025FAB4F9A8
:105FA000000018F059FA0123B340DBB280B11D4361
:105FB000D9F80410DAF80020B2FBF8F2D9F804306E
:105FC0005B1A9A42FADC013ECAD22846BDE8F08745
:105FD00025EA0305ECE700BF001000E040420F0097
:105FE000F80100202DE9F0471E4FDFF87C900446B1
:105FF00088461F260025B4F90400DFF870A00021B0
:1060000018F0F2F928FA06F101F00101B4F90200E2
:1060100018F0EAF97968DAF80030B3FBF9F27B6836
:106020005B1A9A42FBDCB4F90400012118F0DCF998
:10603000B4F9000018F010FA0123B34070B11D4309
:106040007968DAF80020B2FBF9F27B685B1A9A42B1
:10605000FBDC013ECFD22846BDE8F08725EA0305E8
:10606000EEE700BF001000E040420F00F801002002
:1060700010B5064C00210E2018F0B6F9217804481E
:1060800000F04AFC0023237010BD00BF140C002058
:10609000180C002010B5012104460E2018F046F916
:1060A00000210E2018F0A0F90123637010BD00003C
:1060B000437813B5BBB10378ABB10C4C01210E2072
:1060C00018F092F9217811B1094800F041FD094B0F
:1060D000019306230093002305481A464FF47A7172
:1060E00000F0B9FC207002B010BD00BF140C0020FD
:1060F000180C002071600008104908B50B889BB28D
:10610000012B08D80B889BB2A3B90D4B0D4A1B88F5
:106110009BB2D3620DE00C4A138801339BB213800B
:106120000A8892B2B3FBF2F002FB10339BB2002B51
:10613000E8D008BD054B1B689847E6E7460D0020F0
:106140001200002000480140340D0020380D0020CE
:10615000104908B50B889BB2012B08D80B889BB25D
:10616000A3B90D4B0D4A1B889BB2D3620DE00C4ABC
:10617000138801339BB213800A8892B2B3FBF2F00A
:1061800002FB10339BB2002BE8D008BD054B1B6807
:106190009847E6E7440D0020100000200040014031
:1061A000280D00202C0D0020104908B50B889BB24B
:1061B000012B08D80B889BB2A3B90D4B0D4A1B8845
:1061C0009BB2D3620DE00C4A138801339BB213805B
:1061D0000A8892B2B3FBF2F002FB10339BB2002BA1
:1061E000E8D008BD054B1B689847E6E7420D002044
:1061F0000E000020000800401E0D0020200D002091
:10620000012A02D1016000207047022A05D0032A2A
:10621000F9D0002AF7D10260F5E70B680360F2E7D6
:1062200003681847194B4A1E9A4210D8102938BFE4
:1062300010218A0C01328B08B3FBF2F3013B72B6DA
:10624000013803280DD8DFE800F0060E141A0022EA
:106250004FF47A63F3E70E499BB20B800D4B92B279
:106260001A8062B670470C499BB20B8092B20B4BFE
:10627000F6E70B499BB20B8092B20A4BF0E70A4952
:106280009BB20B8092B2094BEAE700BFFFD7CA7FEF
:1062900012000020460D002010000020440D0020B8
:1062A0000E000020420D00200C000020400D0020B8
:1062B0007FB5064608460C46154611F04AFF0122F6
:1062C00011464FF0FF33204612F040F801228023A0
:1062D0001146204612F03CFA0023CDE90033CDE907
:1062E000023325B1164B0393164B009502936A4671
:1062F0000121204612F01EFB029B1BB169460322BE
:1063000008469847204612F0B7F90F49B0FBF1F163
:10631000204612F00FF9204600224FF47A6112F065
:10632000F1F900223146204612F0C0F8204611F063
:10633000EBFF204612F0D8F8012004B070BD00BF7A
:10634000216200080162000800093D00024B034A77
:106350001968FFF7ADBF00BF3C0D0020F9600008D1
:1063600008B5044B186811F0F4FE034B00221A60C4
:1063700008BD00BF3C0D0020380D0020024B034A31
:106380001968FFF795BF00BF300D0020516100086C
:1063900008B5044B186811F0DCFE034B00221A60AC
:1063A00008BD00BF300D00202C0D0020024B034A19
:1063B0001968FFF77DBF00BF240D0020A961000808
:1063C00008B5044B186811F0C4FE034B00221A6094
:1063D00008BD00BF240D0020200D002038B5044664
:1063E00001256570A5830D46B1FA81F100204909A8
:1063F000C4E9080020702061E076A06284F82C00D7
:106400002063A176E5606261237603B963709DF82D
:1064100010306376059B236318F052F820622844FD
:10642000A0620349A01C19F08CFC204638BD00BFB7
:10643000E273020810B50378022B044607D0032B41
:1064400008D0012B01D1FFF78BFF204610BDFFF7CD
:106450009FFFFAE7FFF7B4FFF7E700000000000036
:106460004B1E032B2DE9F04704460D4617464DD829
:1064700090F818A0BAF1000F48D0437E002B45D108
:10648000032948D0042948D0022914BF364B374B82
:106490001B68002B3AD1237FE668002B43D0012BE9
:1064A0003DD14FF47A535E43314B1868FAF722F826
:1064B0002BA3D3E90023FAF7C1F980463046894679
:1064C000FAF718F802460B4640464946FAF78CF8A8
:1064D000284B0022F9F7D2FEFAF75EFB064672B6A9
:1064E00062B601462846FFF79DFE032D236B24D09C
:1064F000042D2AD0022D18D0DFF86C803846C8F859
:106500000030FFF723FF20BBC8F800004FF0000A5F
:106510005046BDE8F087184BBAE7184BB8E7022B96
:10652000C2D13601C0E71E46BEE7DFF840803846DC
:10653000C8F80030FFF722FFE5E7DFF83C80384677
:10654000C8F80030FFF732FFDDE70C4B00221A607D
:10655000DCE703232570E6602377D9E7AFF30080FB
:106560000000000080846E41380D00202C0D0020BA
:10657000080000200000E03F200D0020480D002012
:1065800082B00191019B036372B60378013B032B38
:1065900006D8DFE803F002080B0E019A064B1A60DA
:1065A00062B602B07047019A044BF8E7019A044BB7
:1065B000F5E7019A034BF2E7380D00202C0D00207F
:1065C000200D0020480D0020F8B503780446E3B9FB
:1065D000C37ED3B9C368002B5AD0037F022B16D1D8
:1065E00017F070FF6378054613B100236370A06253
:1065F000A66A761B09D50123E376236B9847284BBF
:106600001F780022E2762FB11A700020F8BD17F033
:1066100057FFE7E794F82C3043B1022B05D1237FD5
:10662000022B32D117F04EFF05463E46637F03B37F
:106630001C4B1868F9F75EFF17A3D3E90023FAF79C
:10664000FDF8064620690F46F9F754FF02460B464F
:1066500030463946F9F7C8FF134B0022F9F70EFE12
:10666000FAF79AFA72B6E06062B60026637F237783
:106670006677E368F34248BF5E422B443344A3622B
:10668000237E002BC1D1E360BFE717F019FFCBE7F2
:1066900001234370B9E700BF0000000080846E4111
:1066A0001D0D0020080000200000E03F10B504464A
:1066B000406938B117F004FF236A62691344C01AB5
:1066C000C043C00F10BD01234361036A013B036255
:1066D000704710B507220446023019F089FA0023EA
:1066E000637210BD00000000427FF8B50446002A26
:1066F0003CD0012A03693AD14FF47A5253432361C3
:106700000323A383244B1868F9F7F4FE20A3D3E9ED
:106710000023FAF793F8064620690F46F9F7EAFED8
:1067200002460B4630463946F9F75EFF1B4B002206
:10673000F9F7A4FDFAF730FAE56872B6E06062B6E0
:10674000E1682078FFF76EFD154B9D420ED9E36896
:106750009D420BD92378022B0DD0032B10D0012B97
:1067600004D1104B104A1B889BB2D362F8BD022A99
:10677000C6D11B01C3E70D4B0D4A1B889BB2F4E742
:106780000C4B0D4A1B889BB2EFE700BFAFF30080B4
:106790000000000080846E41080000200000E03FFF
:1067A000006A18001200002000480140100000207C
:1067B000004001400E0000200008004003780BB1AB
:1067C000FFF792BF704710B5037804462BB1BDE8C0
:1067D000104001614277FFF787BF032A0FD100EE17
:1067E000101ABBEECE0A1CF065FE01460222E368D9
:1067F00073B90120A076E1602277637710BD012A8A
:10680000F5D1B1F57A7FF2D24FF47A735943EDE7BF
:106810000023A37621616277F0E72DE9F041044679
:1068200000F10C0500F1440600F13C0815F8013FA9
:1068300043B1376837B13846FFF7FCFD342138469D
:1068400012F0D9F8454506F10406EFD12046BDE81F
:10685000F08138B504460846B1B14B1EE118487BBB
:1068600090B194F83D5035B194F83E1069B194F868
:106870003F1061B9022504EB8303691C586CFFF7D4
:10688000EFFD2C4484F83D0038BD0125F3E70020DE
:10689000FAE713B50B46019259B14218147B2CB19B
:1068A00000EB83000199006CFFF76AFE204602B0FE
:1068B00010BD0C46FAE739B143181B7B23B100EB3E
:1068C0008100006CFFF77ABF70470B46114643B159
:1068D000C218127B2AB100EB83000122006CFFF783
:1068E00072BF70470B46114643B1C218127B2AB1E2
:1068F00000EB83000222006CFFF765BF70470B4678
:10690000114643B1C218127B2AB100EB8300032267
:10691000006CFFF758BF704739B143181B7B23B198
:1069200000EB8100006CFFF7CEBE70470B461146AE
:106930003BB1C218127B22B100EB8300006CFFF761
:10694000C8BE704738B50D4604460749074819F0D8
:10695000F8F93DB163191B7B23B104EB8504206C6E
:10696000023038BD0148FCE7E27302081C0D00202C
:10697000034608461A18411C527BC8B21AB9197846
:106980008142F7D8104670470021FFF7F1BF0000A1
:106990000E4B1A680E4B1968914270B514D00D4811
:1069A0001A60FFF7F1FF044670B10A4E3025214608
:1069B0003046FFF780FF21463046FFF7D9FF013D03
:1069C000044601D0002CF2D170BD00BF08000020A9
:1069D00004000020180C0020F8B505460E46FFF70D
:1069E000D3FF044608B92046F8BD21462846FFF7E4
:1069F000A9FF3146074619F00EF940B13846F9F7BC
:106A0000CFFB07463046F9F7CBFB8742EBD0214658
:106A10002846FFF7ADFFE4E710B500230178437087
:106A2000DAB200EB82024478526C527E0133944217
:106A300038BF4270DAB28A42F2D910BD0246002352
:106A400002F83D3B2F2312F8011D09B10370704776
:106A5000013BF8D270472DE9F74F9DF83070072FB2
:106A60000446884691469A4604D90025284603B034
:106A7000BDE8F08F4378BB4238BF477000F10C038C
:106A8000002513F8012F2E460135EDB2B2B934209E
:106A900011F0ADFF0D9B4A46CDE9007341465346C8
:106AA0008346FFF79BFC04EB86032644C3F844B0FF
:106AB000012373732046FFF7C1FFD7E7302DE0D1E4
:106AC000D3E737B5079C01949DF81840009405461C
:106AD000FFF7C1FF089A044601462846FFF726FF44
:106AE000204603B030BD000030B5154A4FF40023F6
:106AF00003601368C0F8053000255368C0F80930FA
:106B000085B004460571C0F83D50294630220D304D
:106B100019F0B1F82946C02204F1440019F0ABF88D
:106B2000084B0293084B0193072300932A46012345
:106B30004FF47A710548FFF7C4FF204605B030BD19
:106B400054630208C066020891690008180C00200E
:106B500070B50446B9B14D1E05446B7B9BB100EB8B
:106B600081010E6C36B13046FFF764FC34213046AB
:106B700011F041FF00236B732046FFF75FFFBDE874
:106B80007040FFF749BF70BD2DE9F843044616F089
:106B90000FF90025A678EFB2B74233D22278A7705A
:106BA0004FF0000804EB070999F805300133DBB218
:106BB000934288BF0023E21889F80530527BCAB19E
:106BC00004EB8303586C437EBB4213D1FFF76EFD89
:106BD00099F8051038B10131C9B22046FFF7B8FF66
:106BE000A670BDE8F88304EB8101486CFFF7ECFC6C
:106BF0000028F5D1227808F101085FFA88F39A425B
:106C0000D2D2A67062780135EBB29A42C2D2E8E7DE
:106C100038B50C46054617F053FC044417F050FCF9
:106C2000031B002B00DB38BD2846FFF7ADFFF5E75F
:106C300038B50C46054617F045FC044417F042FCF5
:106C4000031B002B00DB38BD2846FFF79DFFF5E74F
:106C500010B5B02011F0CBFE0E49044611F022FE13
:106C60000D4BB0201C6011F0C2FE0C49044611F01F
:106C700019FE0B4BB0201C6011F0B9FE0949044607
:106C800011F010FE084B09481C60BDE81040FFF7EA
:106C90002BBF00BF004801403C0D002000400140D8
:106CA000300D002000080040240D0020180C0020AA
:106CB0000148FFF7B2BD00BF180C00202DE9F84FC6
:106CC0000C460546682120680CF042FF20680368E6
:106CD00000211B68984720680DF05EF8207130B1E4
:106CE0000021284613F0C4FF2846BDE8F88F20682D
:106CF000072268210DF04DF8072802D004232371E4
:106D0000EEE7206803685B69984700F07F0014F0A5
:106D10001CF80646206803685B699847C0B214F007
:106D200014F80746206803685B699847C0B214F0FE
:106D30001CF88046206803685B69984720680368F0
:106D40005B699847C0B214F000F881462068036878
:106D50005B69984783465FFA80FA206803685B693D
:106D60009847C0B213F0F1FF1BF0800F044608BF34
:106D700000F5FA640AF07F0018BF04F6340413F03B
:106D8000E4FFA4B230342C70687085F8029085F866
:106D900003802F716E71A7E72DE9F041037A8CB063
:106DA0000C46002B5AD0324904A8FFF787FF9DF804
:106DB00010309DF811109DF812209DF813809DF859
:106DC00014609DF8155003F5FA6340F2E1708342B8
:106DD00044D9481E0B2841D8501E1E283ED8B8F171
:106DE000170F3BD83B2E39D83B2D37D8ADF818308C
:106DF0000CAB8DF81A108DF81B2013E90F008DE8ED
:106E00000F00DDE906231B48FDF7E6F8304684ED68
:106E1000000B84ED021BF9F77DFB174B0022F9F7FD
:106E20000DFD064640460F46F9F774FB02460B4639
:106E300030463946F9F722FA064628460F46F9F752
:106E400069FB09A3D3E90023F9F7F8FC02460B46D6
:106E500030463946F9F712FAC4E902010CB0BDE830
:106E6000F08100BFAFF30080000000000020AC40C4
:106E7000600D0020A006002000004E4038B50446FA
:106E80000D46006868210CF063FE206803682946FF
:106E90001B68984720680CF07FFF207140B920687C
:106EA000012268210CF075FF012803D0042323710F
:106EB000002038BD206803685B699847C0B2F8E7D6
:106EC00010B50E210446FFF7D9FF03065DBF2079F8
:106ED000B0FA80F04009002010BD70B504460E469F
:106EE0000068682115460CF033FE206803683146BF
:106EF0001B6898472068036829461B6898472068E4
:106F00000CF04AFF207170BD38B5002104462248BC
:106F10000DF006F8214920480CF000FE68211E48BB
:106F20000CF01EFE1C480CF037FF014688BB1C4DC0
:106F300028680CF0F5FF184818490CF0EFFD2846BA
:106F4000FFF7BEFF48B90E212846FFF797FF0E2135
:106F500000F07F022846FFF7C0FF1148FFF7B0FF9F
:106F6000B8B10E210E48FFF789FF00F0B80242F0D9
:106F700040020B480E21FFF7B0FF0E210848FFF733
:106F80007DFF0E2100F0E7020548FFF7A6FF012371
:106F90002372207A38BD00BF30210020A086010076
:106FA000600D00202DE9F8430D460F210446FFF740
:106FB00065FF0F2100F07F022046FFF78EFF20685B
:106FC00068210CF0C5FD2068036800211B68984704
:106FD0002668687933681F6813F0BEFE01463046A4
:106FE000B8472668287933681F6813F0B5FE014654
:106FF0003046B8472668E87833681F6813F0ACFE5F
:1070000001463046B8472E78632E88BF643E284636
:1070100086BFF6B24FF080084FF0000813F086FEEE
:10702000276800283B6808BF0720D3F8009013F0BA
:1070300093FE01463846C8472768A8783B68D3F8CE
:10704000009013F089FE01463846C84768782768E3
:1070500013F082FE3B6840EA0801C9B21B6838465B
:10706000984725682B6830461F6813F075FE014667
:107070002846B84720680CF08FFE2071BDE8F883E1
:1070800073B5C8B289B2B1F5FA6F24BF3030C0B25F
:107090009DF818609DF81C509DF820408DF8000068
:1070A000D2B2DBB207488DF8012069468DF8023074
:1070B0008DF803608DF804508DF80540FFF772FFDE
:1070C00002B070BD600D00202DE9F047037A8EB04C
:1070D0008DED061B0446002B50D02D4908A8FDF766
:1070E0006BF8DDE9060323F0004127A3D3E9002371
:1070F000F9F7C4F806460F4647EC106B1BF09CFFEF
:1071000051EC100BF9F720FD0546F9F703FA02469A
:107110000B4630463946F9F7AFF81E4B0022F9F717
:1071200063FA8046894649EC108B1BF085FF57ECCB
:10713000106B404632463B464946F9F79DF8154BE1
:107140000022F9F751FA41EC100B1BF075FF51ECDE
:10715000100BF9F7F9FC394602903046F9F7F4FCC8
:107160009DF823A09DF82290BDF92080CDE9005024
:1071700053464A4641462046FFF782FF0EB0BDE81F
:10718000F08700BFAFF30080F78F85E81038223F0B
:10719000A006002000004E40024B034A1A60002265
:1071A0001A717047600D0020302100204FF41653F3
:1071B0002DE9F0410025044643604FF04C083F2381
:1071C0000372C0E908550E461746058085700573A1
:1071D000056142462946283018F04DFD42462946B1
:1071E000656704F1780018F046FDC4F8C45084F8CF
:1071F000C85004F1CC00FDF747FA277266602046BC
:10720000BDE8F0812DE9FF47DDE90C95044600203B
:107210002070CDE901544448CDF800900E469046C8
:107220001F4600F0BFFC82462078BAF1000F6BD1F8
:10723000431E012B68D998F80030062B12D198F81C
:1072400001303370302B07D13849304618F079FDC2
:1072500000232B70207857E0012386F801A089F8DD
:107260000030F5E7532B3DD198F80130422B59D12E
:107270003B78412B11D104F1CC062D49304615F055
:10728000C3FB32212B48FFF7C3FC4FF4613130467A
:10729000FDF734FA85F800A0DCE7422B0CD104F1AD
:1072A000CC062349304615F0AFFB32212148FFF7C9
:1072B000AFFC4FF4E121EAE7A3F13006092E0ED826
:1072C00004F1CC071A49384615F09EFB19483221C3
:1072D000FFF79EFC184B384653F82610D8E70523D5
:1072E0002370B7E7472B1DD198F80130582B0ED1EA
:1072F0003B78392B16D17B78462B13D1BB788BB9D1
:10730000012302202B70207004B0BDE8F087452BCC
:1073100008D13F7837B962780849304617F006FC43
:107320002F7097E70320EFE768110020C866020876
:1073300088670208180C0020E4660208F269020857
:1073400037B50F4B00241B788DF8043008460D46E6
:10735000ADF80540F8F724FF2B4628442246834227
:1073600009D1084901A817F0E1FB01A9284618F046
:1073700011FC03B030BD13F8011B0A44D2B2EEE792
:107380005C630208E065020830B585B0184C194B03
:10739000029305250022184B019311460123009505
:1073A0002046FFF78EFB40F6C41201462046FFF749
:1073B00099FA124B0293124B0022CDE90053114669
:1073C00001232046FFF77DFB40F6C412014620460C
:1073D000FFF788FA0B4B02930B4B0022CDE90053C9
:1073E000032101232046FFF76CFB05B030BD00BF31
:1073F000180C0020D066020879750008D5660208CE
:1074000085750008DA6602089175000808B5412202
:107410004FF416510848FFF7C9FE42224FF41651A7
:107420000648FFF7C3FEBDE8084005484C224FF46C
:107430001651FFF7BBBE00BF280F0020480E0020EA
:10744000680D002008B50548FDF778F90448FDF7F8
:1074500075F9BDE808400348FDF770B9340E002007
:10746000140F0020F40F0020F0B5837899B0044683
:1074700000F1CC0643B9C82017F026F86168304601
:10748000FDF73CF90123A37004F10C053046FDF72C
:10749000DFF948B13046FDF7F9F9C7B23946284659
:1074A000FCF7D8FF232FF1D12846FDF7B1F80028CB
:1074B00038D0002739464C2205A8049718F0DBFB8A
:1074C000012328468DF80E308DF80F70FDF770F807
:1074D00007462846FDF77CF80DF10E0201920DF1EA
:1074E0000F020346009204A93A462046FFF78AFE9F
:1074F0009DF80E3020704BB101288CBF1B491C49F0
:1075000004A818F01EFC01238DF80F309DF8102000
:10751000237B4AB94BB92378192B18BF63702846CF
:10752000FDF791F819B0F0BD93B104A92046FFF71B
:1075300007FF2846FDF764F8014604A818F02AFB67
:1075400000238DF80F300B4904A818F023FB03E04B
:107550009DF80F30002BF6D004A8F8F721FE04A9FF
:1075600002463046FDF742F9D5E700BF1167020831
:1075700088670208DF6602080148FFF775BF00BF91
:10758000280F00200148FFF76FBF00BF480E002002
:107590000148FFF769BF00BF680D00202DE9F047E3
:1075A0004F4E0446307886B018B1207806B0BDE85A
:1075B000F087607004F1480104F1900E4FF02058FC
:1075C0000B4651F808AF4F68B7F1FF3F08BFBAF15B
:1075D000FF3F49D0474508BF824545D0473B382249
:1075E000C2F12009A2F1200C2AFA02F507FA09F9E2
:1075F00045EA090527FA0CFC083A45EA0C0512F1A0
:10760000080F03F8015FEBD16378013363707145B4
:10761000D6D13448DFF8CC9013F071FA324A94F89E
:1076200001801068516804AB03C30025012204A93E
:10763000484613F097FA0746D8B901462B4813F08D
:107640002FFC6378002B49D0294A2A480123237054
:107650000292294A019207220092FA213A46FFF744
:1076600030FA01233370A0E743F8460C43F8420C8C
:10767000CDE7072104A813F0E5FA9DF817308342FF
:10768000D4D19DF81030102B01D0282BCED1B8F1D9
:10769000000FCBD1082D0FDC05F10053093304EBAB
:1076A000C3034FF0205253F8080F5968914208BFA6
:1076B000404505D0092D01D10135B7E70135F2E785
:1076C000092DF9D004AA677803CA04EBC50308376B
:1076D000C3F80200C3F806106770EDE72370C0E737
:1076E000EC1000203C06002060630208F01000202F
:1076F0000C670208180C0020E178000838B5037800
:107700000446E3B107291AD801F10A0300EBC300CC
:1077100054F833204368B3F1FF3F08BFB2F1FF3F95
:1077200001F1260506D1074800F0B2F904EB850304
:1077300083ED000A04EB850494ED000A38BD9FED4B
:10774000020AFBE7180000200000C07FDFED117A7D
:107750009FED117A70EE277AF0EEE77AF4EEC77AB1
:10776000F1EE10FA12D4DFED0D7AB4EEE70AF1EE85
:1077700010FA0BD4DFED0A7AB4EE670ADFED097A6E
:10778000F1EE10FAC8BFB0EE670A70479FED050A28
:10779000704700BF0000FE426F12833A0000C8C26B
:1077A00000008C420000C07FF8B50278454D2DEDF9
:1077B000048B2B680446002A7AD0002B424E0ADA4A
:1077C00016F07EFE01213060404813F0B1FB10B18D
:1077D0002B6801332B6016F073FE3368C01AC7287C
:1077E0006DDD2B680A3304EBC30154F833204B687A
:1077F000B3F1FF3F08BFB2F1FF3F59D0334FDFED88
:10780000348A9FED349A1626296804EBC1010122BF
:107810000231384613F051FC70EE287AB0EE408AFF
:10782000F0EEE77AF4EEC97AF1EE10FA17D4B0EE82
:10783000480A2046FFF78AFFB4EE400AF1EE10FA3C
:1078400014D716F03DFE2B6804EB8304D4F8BC304B
:10785000C01A0028C4BF204BC4F8983028E01F4845
:107860000221FFF7D5F9013ECED1E0E72B6804EB0A
:107870008303D3ED267AF4EE677AF1EE10FA68BF4F
:1078800083ED260A93ED267AF2EE027AA7EE270A16
:10789000B2EE047AC0EE077AC3ED267A16F010FE37
:1078A0002B6800F5EA4004EB83033030C3F8BC00DA
:1078B0002B680133082BC8BF4FF0FF332B60BDECA2
:1078C000048BF8BD14000020E8100020F010002008
:1078D0000000FC426F12833A0000C07F180C0020A9
:1078E0000148FFF761BF00BF08100020F8B50F4E38
:1078F0000F491048104C13F059FA3046002704F194
:10790000080120F8507B4822503418F00CFA0FCCB4
:1079100006F198050FC50FCC0FC523682B602422F4
:10792000394606F1BC0018F0A6F9F8BD0810002091
:107930003C060020F0100020606302081FB5002301
:10794000044643700F4A1048762113F06FFD10B1C2
:107950004FF4817323800D490A480CF0DFF86378F7
:1079600063B10B4B02930B4B0193072300930A481F
:10797000012300224FF47A71FFF7A3F8607804B076
:1079800010BD00BF3021002014110020A08601008E
:1079900013670208857A0008180C0020F8B54378B0
:1079A0002DED028B04468BB12D4B1E7876B92D4DF3
:1079B0002B680133022B2B600BD0032B13D0012B30
:1079C00017D1294813F056FD84ED010ABDEC028B56
:1079D000F8BD254813F096FD9FED247AC0EE077A96
:1079E000C4ED037AF2E7204813F080FE2E6084EDA8
:1079F000040A1F4A94ED018A13781BB10023137007
:107A000084ED028AB4EE488AF1EE10FA19491CD6C8
:107A10000023A0680B70F8F78FFD174B0022F8F7D2
:107A2000E3FD064618EE100A0F46F8F785FD0246FC
:107A30000B4630463946F8F721FC104B0022F8F788
:107A4000FDFEF9F7C9F8A060C0E70B780E2B85BFE3
:107A50000B4BA3600133012394BF0B701370B5E788
:107A6000A211002010110020141100200000C842B3
:107A70002C0000200C1100200000224000002440B7
:107A80000000C07F0148FFF789BF00BF1800002039
:107A900090ED020A704700000346007888B9DFEDD8
:107AA0000A7AB4EEE70AF1EE10FA0BDBDFED077AA3
:107AB000B4EEE70AF1EE10FA04D583ED010A83ED86
:107AC000020A0120704700BF0000C8C20000C8427F
:107AD00090ED030A704700000346007878B9DFEDA7
:107AE000097AB4EEE70AF1EE10FA09DBDFED067A67
:107AF000B4EEE70AF1EE10FA02D583ED030A012095
:107B0000704700BF0000FA430080BB4490ED040AB8
:107B1000704700000378012B0DD8B5EEC00AF1EED6
:107B200010FA0ADBDFED067AB4EEE70AF1EE10FA9E
:107B300003D580ED040A012070470020704700BF84
:107B40000000C842D0B504468068F8F7F5FC064648
:107B500020690F46F8F7F0FC02460B460020094961
:107B6000F8F78AFB084B0022F8F768FE02460B463E
:107B700030463946F8F780FBF9F72EF800EE100A88
:107B8000D0BD00BF0000594000001440014813F070
:107B90009BBA00BF14110020014813F09DBA00BF2A
:107BA000141100202DE9F04786B0DDE90E97DDF8CD
:107BB0004080CDF800908246CDE90178AB480D4673
:107BC00016461C4602F0E0FA002840F0D280CDE9CB
:107BD0000178A748CDF8009023463246294607F0A1
:107BE0004DFC002840F0C580CDE90178A148CDF8D2
:107BF0000090234632462946FDF7D4FB002840F08A
:107C0000B880CDE901789C48CDF8009023463246F3
:107C100029460BF03DFC002840F0AB80CDE901780F
:107C20009648CDF8009023463246294605F028FDB7
:107C3000002840F09E80CDE901789148CDF8009071
:107C400023463246294609F0EBFE002840F0918099
:107C5000CDE901788B48CDF800902346324629467D
:107C600008F096FC002840F08480CDE90178864831
:107C7000CDF800902346324629460AF011FA002832
:107C800077D1CDE901788148CDF80090234632467E
:107C9000294609F0D5F800286BD1CDE901787C4858
:107CA000CDF8009023463246294608F013FB002801
:107CB0005FD1CDE901787748CDF800902346324670
:107CC00029460AF035F9002853D1CDE901787248E8
:107CD000CDF80090234632462946F9F749FA0028A4
:107CE00047D1CDE901786D48CDF800902346324662
:107CF0002946F9F73DFA00283BD1CDE901786848DB
:107D0000CDF8009023463246294601F085FA80BB23
:107D1000CDF80090CDE901786248234632462946E5
:107D200000F074FA814620BB3378422B0BD1737874
:107D30002B2B05D12378D3B1484606B0BDE8F08798
:107D40002D2BF9D1F6E7452B67D17378432B1AD148
:107D5000254620262046F8F723FA2B1B98420BD8FD
:107D600028B10138235C262B01D1002323540023A2
:107D70003B704FF00109DFE715F8013B5F2B08BFAF
:107D800005F8016CE6E7522B23D12378452B40D12F
:107D90006378532B3DD1A378452B3AD1E378542B0C
:107DA00037D12379002B34D13F48FDF7EDFB3F4815
:107DB0004FF47A71FEF72CFFBFF34F8F3C493D4BD8
:107DC000CA6802F4E0621343CB60BFF34F8F00BF79
:107DD000FDE74E2B1DD12378562B1AD16378522BF9
:107DE00017D1A378452B14D1E378532B11D12379E4
:107DF000452B0ED16379542B0BD1A4794CB92A4869
:107E00002146FDF736FD2C49284617F09AFF3C70B5
:107E1000AFE7032388F80030ABE7472B40F0A5809D
:107E20007378562B61D16378002B85D12378442B4E
:107E300005D10AF10D01284617F083FF97E74D3B66
:107E4000072B4ED8DFE803F0043C4D484D4D4D4A1A
:107E50000AF10A0301939AF8093000939AF808305E
:107E600016495246284616F061FE80E7F8180020B1
:107E70005C010020B9070020C8010020B81E0020C6
:107E80008020002038200020A82000205C20002036
:107E9000F01F002094200020A0160020481400208D
:107EA0000014002030000020FC050020180C0020E9
:107EB00000ED00E00400FA051B67020847670208AE
:107EC0000AF10A0300939AF809309AF808205549F4
:107ED000284616F02BFE4AE75146ACE70AF121018D
:107EE000A9E7032388F8003041E7582B7FF424AF3B
:107EF000A678002E7FF420AF2378392B24D1637825
:107F0000412B0ED14848FFF7C3FD10EE100AF8F7D9
:107F100013FB41EC100B45492846FCF707FD3E706A
:107F200027E7422B03D14048FFF7D2FDEDE7432B73
:107F300003D13D48FFF7EAFDE7E7452B7FF4FCAEB0
:107F40003948FFF7FFFDE0E7412B7FF4F5AE63789A
:107F5000302B7FF4F1AE36484FF48771FDF735FCD6
:107F6000C3073FF506AF022354E7532B7FF4E4AE7B
:107F70007378582B7FF4E0AEA3782C2B7FF4DCAE23
:107F80002378392B28D1E51C05A9284617F0ECFCED
:107F9000059B9D4251EC100B0ED0F8F71DFE00EE34
:107FA000100A6378412B0AD11F48FFF775FD00289E
:107FB0007FF4DFAE05232DE79FED1E0AF1E7422B8C
:107FC00003D11948FFF788FDF1E7432B7FF4B4AEE6
:107FD0001548FFF79FFDEAE7412B7FF4ADAE6378CC
:107FE000432B7FF4C6AE2379002B7FF4C2AEE37837
:107FF000303B012BDED84FF487710D48FDF7E5FBD0
:10800000E378302B0CBF40F0010020F0010080B27B
:10801000ADF814000223064805AA4FF48771FDF756
:10802000F9FBA6E64A670208180000205467020818
:10803000FC0500200000C07F16490B78102B9ABF6A
:108040000133DBB200230B70134B1B7813F00102DA
:108050000ED198070BD49A060FD458070FD4DA061E
:108060000FD418070FD400211B2016F0BDB902222F
:108070000B78D90709D40121F6E70322F8E7042297
:10808000F6E70522F4E70622F2E7B2EB530FEAD84F
:10809000704700BFA0110020A11100204FF6FF7310
:1080A00010B50121C38604461A2016F03FF90121BC
:1080B000C42016F03BF90121182016F037F90121F0
:1080C000192016F033F90121182016F02FF9204657
:1080D00010BD000070B5044686B016461D4617F068
:1080E00030FE0A992672657204F10A0017F029FE23
:1080F0000B9B23733349344E04F10D0017F021FE1E
:10810000324904F1210017F01CFE31492E48FDF7D9
:1081100071FB10B93046FDF7D7FA2E482E4DFDF70A
:108120003FF918B92B7843F020032B702B48FFF749
:1081300005FC2B48FFF732FA2A4802F03DFD2A4899
:108140000BF04AFC294801F0CBFC264802F084FEE3
:10815000264801F0CBFE264800F0E6FA96F82C30CF
:10816000C3B9E38EADF81630174802230DF116029D
:108170004FF45071FDF74EFB96F82C3053B914496B
:108180001148FDF776FB1048FDF7FEF910490E483F
:10819000FDF730FB2B78B279012162F300031B203D
:1081A0002B7016F0C3F8134B0293134B0193042367
:1081B0000093002201234FF4FA711048FEF781FC6E
:1081C00006B070BD5A670208FC0500206667020809
:1081D000660CCE22B9070020A11100201800002053
:1081E00008100020F8180020C8010020001400200A
:1081F000300000206F67020839800008180C00204A
:108200000148FFF74BBF00BF681100202DE9F04780
:108210002DED028BC0B01E464A9B0446002018700C
:108220001378472BDDE94B780D4640F049815378B0
:10823000582B40F0178196F80290B9F1000F40F0EA
:1082400011813378582B40F0F38096F80190A9F112
:108250003103072B00F20D8104EB43125E01B2F9EA
:108260001420012A07D0023A032A00F25982DFE8DB
:1082700002F0020B630204EB4313B3F92220B2496C
:10828000684616F053FC50E02644B06A00F056FDF4
:10829000AD490246684616F049FC6946284617F083
:1082A00079FCAA49284617F075FCB06A00F099FCE1
:1082B00010EE100AF8F740F941EC100BA44968469B
:1082C000FCF734FB6946284617F064FC9F492846B2
:1082D00017F060FCB06A00F0D9FC10EE100AF8F755
:1082E0002BF941EC100B9A496846FCF71FFB6946D5
:1082F000284617F04FFC9549284617F04BFCA9F18A
:1083000030019448FFF7FAF99348B0EE408AFFF73E
:1083100019FC78EE407A17EE900AF8F70DF941EC67
:10832000100B8B496846FCF701FB6946284617F09D
:1083300031FC00233B7094E004EB0608B2EE048AA3
:10834000D8F82C0000F04EFDFDEEC07A7E4917EE05
:10835000902A684616F0EAFB6946284617F01AFC90
:108360007A49284617F016FCD8F82C0000F034FDA6
:10837000F7EE007AB4EEE70AF1EE10FA52D4B4EE5A
:10838000C80AF1EE10FA4FD4F3EE0E7AB4EEE70A13
:10839000F1EE10FA4CBF0121002110EE100A5FFA35
:1083A00081F8F8F7C9F86A4641EC100B4146002005
:1083B00014F04CFC6946284617F0ECFB634928464C
:1083C00017F0E8FBA319D86A00F009FDB4EEC80A5B
:1083D000F1EE10FA2AD4F3EE0E7AB4EEE70AF1EEDB
:1083E00010FA4CBF0121002110EE100A5FFA81F84B
:1083F000F8F7A2F86A4641EC100B4146002014F051
:1084000025FC26446946284617F0C4FB4F492846F8
:1084100017F0C0FBF06A00F0EAFCFDEEC07A17EE40
:10842000902A2CE70321B8E70221B6E70221DBE717
:10843000592B40F077817278302AA2F1310316D19E
:1084400001F10803B4F91420511C0CBF3022312271
:108450002A7005F8019FAB4204F12004F2D187F89D
:108460000090012040B0BDEC028BBDE8F087072BE7
:1084700001D9062307E05E0104EB4313B3F914208E
:10848000013203D1022388F80030EAE7196968460F
:1084900017F057FC6846F7F783FE26440A2869461A
:1084A000284688BF8DF80A9017F04BFC27492846CC
:1084B00017F070FBB6F91420052A08BF0122DEE68A
:1084C000532BCFD15378582BCCD1B3782C2BC9D187
:1084D0003378582BC6D196F80190A9F13107072FB0
:1084E000C7D804EB47137D01B3F91430013300F012
:1084F000178106F1040A6946504617F041FA009BBD
:108500009A45B0EE408AB4D01AF0D4FFF378562BD7
:1085100001460DD1002806DA6319B3F91430012B96
:108520000BD10523AFE7FF28F6DC04EB4713588493
:108530006319B3F91430012B14D0023B032B90D8EC
:10854000DFE803F0385A991076670208426402089F
:108550005467020808100020180000200000614540
:1085600000007F43F378562B83D10129D9D804EB3F
:108570004919A9F5C063B3F90000002808DBA9F286
:10858000FC53B3F900305B1A5942594115F02CFFE6
:108590002544B5F91430052B7FF463AFA9F2FE59D9
:1085A000B9F90030002B3FF45CAF2744322387F841
:1085B000103156E7F378562B7FF45BAFFF29B0D824
:1085C00004EB47173B8CB7F92040FF2B3FF649AF30
:1085D00007EE901AB8EEE77A5FED1F7A87EE270A6A
:1085E00020EE270A19F022FBFCEEC07A204617EE97
:1085F000901A15F02DFE34E7F378562B08D1012997
:108600008FD8254401F00101A86A00F099FB28E702
:108610005A2B16D1F9EE047AB4EEE78AF1EE10FA8D
:10862000FFF67FAFF3EE047AB4EEE78AF1EE10FACC
:108630003FF677AF2544B0EE480AA86A00F0D4FAB6
:108640000FE7532B7FF415AFF9EE047AB4EEE78A07
:10865000F1EE10FAFFF665AFF3EE047AB4EEE78AB6
:10866000F1EE10FA3FF65DAF2544B0EE480AA86A75
:1086700000F012FBF5E6F378562B09D101293FF6FD
:1086800050AF254401F00101E86A00F0D9FBE8E6AB
:10869000452B14D1B5EEC08AF1EE10FAFFF641AFCA
:1086A0005FED527AB4EEE78AF1EE10FA3FF639AF99
:1086B0002544B0EE480AE86A00F076FCD1E6442B87
:1086C00016D1F7EE007AB4EEE78AF1EE10FAFFF673
:1086D00028AF5FED5E7AB4EEE78AF1EE10FA3FF66E
:1086E00020AF2544B0EE480AE86A00F083FCB8E603
:1086F000432B7FF4BEAEB5EEC08AF1EE10FAFFF662
:1087000010AF5FED697AB4EEE78AF1EE10FA3FF64A
:1087100008AF2C44B0EE480AE06A00F06DFBA0E61A
:108720000323B0E648469DE62DE9F0412DED028B8E
:1087300000269FED618A84B00746044635464FF017
:108740000008B4F92030043304BF37F9163023840D
:10875000B4F92230991C0DD101236384B4F914308B
:10876000012B0CD0023B042B28D8DFE803F0435F39
:108770007E0808009BB2FF2B88BF6584EEE7B4F942
:108780002000002802DB012115F0D0FDB4F9200003
:10879000002808DBB4F92210B4F92430CA1A514277
:1087A000514115F021FEB4F91430052B1CD1B4F958
:1087B00022301BB107F5887332229A550136082EF4
:1087C00004F12004BDD13D4B02933D4B01930623A0
:1087D00000930022012314213A48FEF772F904B0F5
:1087E000BDEC028BBDE8F081062BE7D14FF6FF739D
:1087F000A382E3E7B4F92000002802DB012115F091
:1088000095FDB4F9223007EE903AF8EEE77A87EE5C
:10881000880A20EE080A19F009FAFCEEC07AB4F9C9
:10882000200017EE901A15F013FDC7E7182010F07E
:10883000DEF8254AC260254A0581C0E9005502617B
:108840004561A062314600F0ABF8B4F92000002881
:1088500002DB012115F06AFDB4F92210A06A00398B
:1088600018BF012100F06CFAA8E7202010F0BFF833
:108870003146C0E90355C0E905550580C0F80480BC
:10888000C0F80880C561E06200F04CFCB4F920003B
:10889000002802DB012115F049FDB4F92000002871
:1088A0008CDBB4F92210B4F92430CB1A5942594167
:1088B00015F09AFD82E700BF00007F437967020848
:1088C00091890008180C00200000A0C00000704131
:1088D0002DE9F8432DED028B2B4FDFF8B0800446D5
:1088E00000F588760025B4F91430052B05F1010553
:1088F0001BD133787BB1013BDBB233705BB9B4F988
:1089000020006384002806DBB4F92410B1FA81F159
:10891000490915F069FD082D04F1200406F101064E
:10892000E1D1BDEC028BBDE8F883032B1ED12946B3
:108930003846D4F82890FEF7E1FE4046B0EE408A73
:10894000FFF700F9484638EE400A00F0FDF8B4F9A8
:108950002090B9F1000FDEDBA06A00F0F5F9B4F960
:1089600024100B1A594259414846D2E7042BD2D160
:10897000E06A00F0EBF9B4F92090B9F1000FCADB1E
:10898000E06A00F066FAEAE708100020180000200C
:108990000148FFF79DBF00BF30000020000000002D
:1089A000F8B5654F2DED028B416101EB41018CB2B1
:1089B00097F82C3004F54A7604F229340546B6B20D
:1089C000A4B27BBBC068F7F7B7FD5C4B0022F7F79A
:1089D00055FC5B4B0022F7F707FE41EC100B1AF039
:1089E000AFFB51EC100BF8F7D7F83146C2B238465E
:1089F000FCF712FE2869F7F79FFD504B0022F7F7AE
:108A00003DFC00224E4BF7F7EFFD41EC100B1AF046
:108A100097FB51EC100BF8F7BFF82146C2B238466D
:108A2000FCF7FAFD31464448FCF788FEF7F772FD83
:108A3000434B0022F7F702FF404B0022F7F71CFCE4
:108A4000F8F7CAF807EE900AB9EE048AF4EEC87A8D
:108A5000F1EE10FA56D4B3EE047AF4EE477AF1EE62
:108A600010FAC8BFF0EE477AC5ED037A21463248C6
:108A7000FCF764FEF7F74EFD314B0022F7F7DEFE00
:108A80002E4B0022F7F7F8FBF8F7A6F895ED037ADE
:108A90002861B4EE487AF1EE10FA07EE900A06D19A
:108AA000F4EE487AF1EE10FA04BF264B2B61D5EDB7
:108AB000047AF4EEC87AF1EE10FA26D4F3EE046AE2
:108AC000F4EE667AF1EE10FAC8BFF0EE667AB4EE14
:108AD000E77AF1EE10FAC5ED047A10DBF4EEC87A0D
:108AE000F1EE10FA14DD17EE900AF7F725FD10A34A
:108AF000D3E90023F7F7C0FBF8F76EF8E860BDECA8
:108B0000028BF8BDF0EE487AAEE7F9EE047ADEE7C4
:108B100017EE100AF7F710FD05A3D3E90023F7F7C6
:108B2000ADFBF8F759F82861E9E700BFAFF3008023
:108B30009A9999999999B93FFC0500200000144031
:108B4000000024400000A04170B52DED028BB4EE72
:108B5000400AF1EE10FA82B0044602D700232372D5
:108B600029E0437A3BB3B2EE048A20EE080A1AF0F9
:108B7000A1FC94ED030A20EE080A05461AF09AFCBF
:108B800094ED040A20EE080A06461AF093FC00232E
:108B900002463146009328464FF4FA6314F04CF82D
:108BA000054615F08DFC21686060421AA2F5FA6254
:108BB000002A04DD206002B0BDEC028B70BDB5F56B
:108BC000FA6FA8BF4FF4FA65227A431A002DA8BFA6
:108BD0005B1B1AB9002BEEDC0123C0E7002BBDDCC8
:108BE000E9E790ED030A7047F9EE047AB4EEE70A7C
:108BF000F1EE10FA10B504463ADBF3EE047AB4EE67
:108C0000E70AF1EE10FA33D8D0ED047A80ED030ACA
:108C1000F4EEC07AF1EE10FA0BD817EE900AF7F7DF
:108C20008BFC18A3D3E90023F7F726FBF7F7D4FF53
:108C3000E060E068F7F780FC0F4B0022F7F71EFBBF
:108C400000220E4BF7F7D0FC41EC100B1AF078FA2B
:108C500051EC100BF7F7A0FF616901EB410101F541
:108C60004A71C2B2BDE81040054889B2FCF7D4BCD5
:108C700010BD00BFAFF3008000001440000024408E
:108C8000FC0500209A9999999999B93F90ED040AA9
:108C90007047000000000000F9EE047AB4EEE70A25
:108CA000F1EE10FA10B504463ADBF3EE047AB4EEB6
:108CB000E70AF1EE10FA33D8D0ED037A80ED040A1A
:108CC000F4EEC07AF1EE10FA0BDB17EE900AF7F72C
:108CD00033FC18A3D3E90023F7F7D0FAF7F77CFFAA
:108CE00020612069F7F728FC0F4B0022F7F7C6FA3E
:108CF00000220E4BF7F778FC41EC100B1AF020FA2B
:108D000051EC100BF7F748FF616901EB410101F2EB
:108D10002931C2B2BDE81040054889B2FCF77CBCDD
:108D200010BD00BFAFF300800000144000002440DD
:108D3000FC0500209A9999999999B93F407A704712
:108D40000023037241727047007A704738B5437848
:108D500004462BB10378012B16D103690BB90380AC
:108D600038BD013B03610323037015F0A9FB0546E1
:108D70006068F7F7E1FB174B0022F7F735FCF7F7D0
:108D80000BFF28446061EBE7032B16D115F098FB2D
:108D90006369C01A002810DD0523237015F090FBCD
:108DA0000546A068F7F7C8FB0A4B0022F7F71CFC42
:108DB000F7F7F2FE2844A061D2E72378052BCFD144
:108DC00015F07EFBA369C01A0028C4BF01232370DD
:108DD000C6E700BF00408F4090ED010A704790ED5C
:108DE000020A704790ED040AB8EEC00A704790ED91
:108DF000030AB8EEC00A70470378DBB9B5EEC00AC3
:108E0000F1EE10FA16DBDFED0C7AB4EEE70AF1EEC4
:108E100010FA0FD8FDEEC07AC169C0ED037A17EEE3
:108E2000902A01EB410101F22A310448D2B289B201
:108E3000FCF7F2BB704700BF00007F43FC05002039
:108E4000417021B1C16801230161037070470B4675
:108E5000FAE70078C31E584258417047DFED457A63
:108E6000B4EEE70AF1EE10FA08B5B0EE407A78D920
:108E7000DFED417AB4EEE70AF1EE10FA74D9DFEDD6
:108E80003F7AB4EEE70AF1EE10FA70D9F7EE007A05
:108E9000B4EEE70AF1EE10FA14D8F2EE007AB0EE72
:108EA000000AA7EE270AB5EEC00AF1EE10FA58D470
:108EB000DFED337AB4EE670AF1EE10FAC8BFB0EE18
:108EC000670A4AE0F2EE047AB4EEE70AF1EE10FA2D
:108ED00004D8F1EE007AB1EE080AE2E7F3EE0E6A8A
:108EE000B4EEE60AF1EE10FA04D8F0EE007AB3EE32
:108EF0000A0AD6E7DFED236AB4EEE60AF1EE10FACD
:108F000004D8DFED217A37EE870ACCE7DFED1F6A60
:108F1000B4EEE60AF1EE10FA06D8F2EE0E6AC0EEF2
:108F2000267A9FED1B7AEEE7DFED1A6AB4EEE60AC9
:108F3000F1EE10FA06D8DFED186A9FED187AC0EE50
:108F4000267AE0E7DFED166AB4EEE60A9FED0C0A3A
:108F5000F1EE10FA88BFB0EE670A1AF0ABFAC0B2B1
:108F600008BD9FED100AF8E7B7EE000AF5E7B0EE8E
:108F7000000AF2E7DDB5843C6E34003D0000803D20
:108F800000007F430000F0420000604200001644F1
:108F90000000284300005245000070420000464394
:108FA0000000614500000000027810B5E2B9B5EE9E
:108FB000C00AF1EE10FA17DB9FED0C7AB4EEC70A87
:108FC000F1EE10FA10D8C16980ED010A01EB410100
:108FD00001F54A74FFF742FFA4B202462146044855
:108FE000BDE81040FCF718BB10BD00BF0000614594
:108FF000FC050020027810B5F2B9B7EE007AB4EEA5
:10900000C70AF1EE10FA17DB9FED0C7AB4EEC70A2F
:10901000F1EE10FA10D8C16980ED020A01EB4101AE
:1090200001F22934FFF71AFFA4B202462146044890
:10903000BDE81040FCF7F0BA10BD00BF000061456C
:10904000FC050020002951D0012952D0022953D01B
:109050000A290CD807EE901AB8EEE70AF0EE007A6B
:1090600030EE670AF4EE007A20EE270A70472E29C8
:109070000AD807EE901AB8EEE70AF1EE087A30EE59
:10908000670AF5EE007AEFE756290AD807EE901A3C
:10909000B8EEE70AF3EE0A7A30EE670AF6EE007AE7
:1090A000E2E7B02908D807EE901AB8EEE70ADFED3C
:1090B000157A30EE670A7047D0290AD807EE901A61
:1090C000B8EEE70ADFED107A30EE670AF2EE0E7ABC
:1090D000CAE7FF2913D007EE901AB8EEE70ADFEDD2
:1090E0000B7A30EE670ADFED0A7ABDE79FED090AD9
:1090F00070479FED090A70479FED080A70479FED82
:10910000080A704700006042000028430000464300
:10911000000070429318843C0000003D0000803D38
:10912000000061452DE9F041C16101EB41018BB2C5
:10913000DFF8808003F54A7703F2293603F22A33F9
:109140009CB298F82C300546BFB2B6B2BBB990EDD0
:10915000010AFFF783FE394602464046FCF75CFAF7
:1091600095ED020A2846FFF779FE31460246404651
:10917000FCF752FA2A7B21464046FCF74DFA394665
:109180000C48FCF7DBFA01462846FFF75BFF314647
:1091900085ED010A0748FCF7D1FA01462846FFF79A
:1091A00051FF044885ED020A2146FCF7C7FAE86042
:1091B000BDE8F081FC05002037B50D4D0D4B0E4A82
:1091C000012404212846FAF75FFC2B460B4A009441
:1091D00004210B48F9F732FD9FED0A0A0A4B0B4AAE
:1091E000009404210A48F8F731FA03B030BD00BFFB
:1091F000FC1200200668020816680208FC670208D4
:109200006012002000000000C4670208DC6702084A
:10921000A8110020000000002DE9F04F2DED048B77
:1092200091B0DDE91E960446002089F80000AA48A6
:10923000209F0068884692461D4630B1CDE90167FF
:10924000CDF80090F7F794FF90BB9AF80030682BA8
:109250001CD19AF80130502B0DD1297829B920461C
:1092600000F098FD80B901233B70002011B0BDECE7
:10927000048BBDE8F08F522BF7D129780029F4D167
:10928000204600F0C7FDEDE73870EEE7462BECD145
:109290009AF80130412B21D195F800A0BAF1000FC6
:1092A00013D1E26A8C4B53F822301BB902233B7076
:1092B0000120DBE789490132404615F037FC0123E4
:1092C00086F800A089F80030F2E76B78002BCCD14B
:1092D000BAF1310F40F04081E362E9E7313B052B01
:1092E0001BD82A78CAB17C4951F823100029BCD078
:1092F0007B498AF801200B6008A8691C16F021FD43
:1093000008A9284616F01DFDDFF8D491D9F800B061
:10931000BBF1000F05DA0323C9E7714BE26A1A605B
:10932000F2E79AF801A06F48514616F042FC18B1D6
:109330002A780AB10623BAE7674B53F82B20536803
:10934000049393680593DDE904010792F7F744FC61
:10935000514608EE100A644816F02BFC079AF7EE07
:10936000007A28BB87EE889AF0EE488AF0EE679A7A
:10937000BAF1610F9CD0BAF1540F22D11046F8F720
:1093800027FEE0B15949404616F0DBFCD9F8001041
:1093900030232046ADF8203000F0B2FA30308DF89E
:1093A000200008A9404616F0F5FB002333707FE744
:1093B000F0EE489AF0EE678AB0EE679AD8E74C492B
:1093C000E1E7BAF1700F07D15946204600F02CFAB8
:1093D00000287FF46DAF69E75046079215F0E6FA72
:1093E0004928079A10D1D2F8253000EE103A29EE1C
:1093F000800A18F01BFCFDEEC07A3E4917EE902A59
:10940000404615F093FBD0E74D2802D1D2F8293021
:10941000EBE7BAF1650F1ED15946204600F010FA6D
:1094200090B1204600F0FAF92046D9F80010B0EECD
:10943000408A00F018FA78EE407A17EE900AF7F7B3
:109440007BF841EC100B01E09FED210B2A494046CF
:10945000FBF76CFAA9E7BAF1740F05D1204600F0CA
:10946000DDF910EE100AEAE7BAF1750F09D1DDE96E
:10947000042322490020F7F7E1F941EC100B2049C1
:10948000E5E742283ED12A7852B95946204600F0F5
:10949000F2F900EE100AB8EEC00A20EE090AA8E7B9
:1094A000284615F07EFA00EE100AB8EEC00A20EE4B
:1094B000280A18F0BBFBFDEEC07A594617EE902A39
:1094C000204600F009FC3870F2E600BFAFF30080E0
:1094D0000000000000000000301400207667020841
:1094E000FC1300202468020838680208406802085B
:1094F0004268020884710208546702080000F03FC5
:1095000044680208BAF1430F28D195F800A0BAF1D7
:10951000000F10D15946204600F097F910EE100ABE
:10952000F7F70AF841EC100BB8494046FBF7FEF993
:1095300086F800A0BCE6284615F030FA51EC100B76
:10954000F7F74AFBD9F8001000EE100A204600F0A9
:1095500097FB00287FF4ACAE0523A8E6BAF1630FB1
:1095600028D1297821B95946204600F069F92FE71A
:109570006B7843B9B1F1300218BF01225946204639
:1095800000F060FB9FE7442840F08F80284615F0EC
:1095900008FA00EE100AB8EEC00A20EE280A18F009
:1095A00045FBFDEEC07A594617EE902A204600F0A2
:1095B00081FBCEE744281BD195F80090B9F1000F4C
:1095C000E4D15946204600F048F900EE100AB8EE02
:1095D000C00A20EE090A18F029FBFDEEC07A8C497A
:1095E00017EE902A404615F0A1FA86F800905FE643
:1095F000BAF1500F20D15946204600F015F9002845
:109600003FF489AE95F800A0D9F80090BAF1000FA8
:1096100009D14946204600F009F97E4902464046F4
:1096200015F084FA84E7284615F0BBF9494602464E
:10963000204600F0FDF88CE7BAF1510F03D1104637
:10964000F9F7F6F8B1E6AAF13101082914D82A7819
:109650007AB9AAF13002042A04DC5946204600F007
:1096600010F9A2E6AAF134025946204600F056FB52
:109670009BE606233B7098E6BAF1570F06D11422F9
:1096800002FB0B436349B3F91A20B9E6BAF12B0F79
:1096900006D101225946204600F008F9387084E6C8
:1096A000BAF12D0F1ED10222F4E747281CD0522810
:1096B0002BD053287FF42FAE2A78002A3FF43AAEFD
:1096C000284615F06EF907EE900AF8EEE77A59464B
:1096D00067EEA87A2046FDEEE77A17EE902A00F0B2
:1096E00063F9F0E647280ED1106803681B6A9847B3
:1096F000D9F8003004EB83035B68C01A07EE900AC8
:10970000B8EEE70AC9E652281CD12A78002AB0D060
:1097100004EB8B02284692ED078A15F042F907EE1A
:10972000100AB8EEC88AB8EEC77AF0EE487AE7EECB
:10973000287AFDEEE77A17EE902A5946204600F087
:1097400033F9ABE75328B7D0BAF15A0F1AD1142125
:1097500001FB0B430025DD7429461046F8F7ACF9F0
:10976000D9F800102C4B3870204653F8217000F0C7
:1097700082F800EE100A3846B8EEC00AF8F77CF915
:10978000357095E5BAF1480F1DD1142101FB0B434B
:109790000025DD74D2F8293000EE103AD2F82530D9
:1097A000049207EE903A30EE270AF6EE007A20EEA9
:1097B000270A18F03BFA28EE008A049AFDEEC87AD0
:1097C00017EE901AC9E7BAF1680F7FF4A4ADD2F88A
:1097D000B0108968013104D000211046F8F7E0FD8F
:1097E00066E5D2F82930D2F8252000EE103A07EECF
:1097F000902A30EE270AF6EE007A20EE270A18F0BB
:1098000015FA28EE008AFDEEC87A94E7446802084B
:109810008471020876670208301400200148002194
:10982000FDF76CBF08100020002070470020704733
:1098300021B9642A8CBF00200120704700207047A6
:1098400009B9007A70470020704721B9D0F8093073
:1098500000EE103A70470023FAE711B9B0F90D0095
:1098600070470020704721B9D0F80F3000EE103A51
:1098700070470023FAE711B9B0F9140070470020CF
:109880007047032A10D0042A05D0012A18BF0A22E3
:1098900040F821207047142303FB0103B3F91A2079
:1098A00002EBD2725210F3E76422F1E770B505467D
:1098B0001646D9B9104C2068D0B1EB7C012B19D8D1
:1098C000F8F786FB40B920689FED0C0AF8F78CFB8F
:1098D00023681868F9F70DF895ED000A20683146FD
:1098E000B8EEC00ABDE87040F8F71FBD032070BD98
:1098F0000520FCE70A20FAE73014002000000000F1
:10990000F8B5142303FB01F63044B0F91A00F6F75A
:1099100001FE224B3344044658880D46F6F7FAFD03
:109920001F4B002206460F46F6F788FF02460B46FD
:1099300020462946F7F7CAF850BB1A4B002230469A
:109940003946F6F77BFF02460B4620462946F7F7D5
:10995000BDF8F8B9134B002230463946F6F744FEFD
:1099600002460B4620462946F7F7B0F8A0B90C4B43
:10997000002230463946F6F737FE02460B462046AF
:109980002946F7F7A3F8002814BF04200520F8BDE6
:109990000120FCE70220FAE70320F8E754680208F8
:1099A0000000FC3F0000F43F70B504461646D1B9F4
:1099B000104D2868C8B1E37C012B18D89FED0E0A22
:1099C000F8F712FB2B68616818683144F8F7C6FF96
:1099D000B4F91A30286800EE103ABDE87040B8EECD
:1099E000C00AF8F76FBC032070BD0520FCE70A2011
:1099F000FAE700BF3014002000000000142370B507
:109A000003FB01F60D4601EB81010446890006F1D6
:109A1000080201F2A5212644024489B22B48FBF733
:109A2000A7FED6F809209FED2A7A07EE902AF0EEDD
:109A3000E77AF4EEC77AF1EE10FA07DD0022C6F8F5
:109A40000920244A137843F002031370142303FB04
:109A5000054303F10802B3F90D30013B9BB242F21A
:109A60000F718B4208D90123537100239371194A56
:109A7000137843F002031370142303FB054303F12F
:109A80000802D3F80F309FED147A07EE903AF0EE0B
:109A9000E77AF4EEC77AF1EE10FA07DD0F4BC2F861
:109AA00007300C4A137843F002031370142303FBAE
:109AB000054442F21073A28A9A4206D9054A00234D
:109AC000A382137843F00203137070BDFC050020DD
:109AD00000C07944A1110020000070420000204124
:109AE00070B5494E49494A4D04463046F7F76AFE7B
:109AF00000287DD1474A137843F004031370464889
:109B000090F82C30002B75D100234FF48072C4E9FB
:109B10000232C4E90433414BA3613F48142304F1EA
:109B2000080240F2A521FBF775FE20460021FFF751
:109B300065FF286800236422C4E90023C4E90733D1
:109B400084F8243000285DD0E26A2372013208BF15
:109B5000E362D0F82530D4F8162007EE903A07EEED
:109B6000102AF4EEC77AF1EE10FA06DD294AC4F89D
:109B70001630137843F002031370D0F82930D4F86C
:109B8000162007EE903A07EE102AF4EEC77AF1EEAF
:109B900010FA06D51F4AC4F81630137843F00203B2
:109BA00013700021F7F788FF2B6893F8982022B9EB
:109BB000B4F914101868F8F7F6FE28689FED180A33
:109BC000F8F70FFA2868B3EE040AF8F707FA2868DE
:109BD0009FED130AF8F70CFA2868B0EE000AF8F7C0
:109BE000C5F92868B7EE000ABDE87040F8F7EAB991
:109BF0002E6084E7142240F2A521FBF7A1FD002886
:109C000082D192E770BD00BFA81100206012002031
:109C100030140020A1110020FC0500200000DC050C
:109C20000080BB44142303FB010201EB8101890086
:109C300001F2A5210248083289B2FBF7EBBD00BF53
:109C4000FC05002010B50446B1B9C37C012B15D822
:109C500002725AB1FFF7E2FD10EE103AC4F80F306D
:109C600020460021FFF7DEFF002010BDC3694168D8
:109C700042600B44C361F3E70320F6E70A20F4E7F0
:109C800008B581B99FED0A7AF0EEC07AF4EEC77A92
:109C9000F1EE10FA09DA10EE103AC0F80930FFF7C9
:109CA000C1FF012008BD0020FCE70846FAE700BF1D
:109CB00000007A4470B551B9561E42F20F75AE429B
:109CC00007D8A0F80D20FFF7ADFF012070BD0020E0
:109CD000FCE70846FAE7000038B505460C46A9B986
:109CE00042F210739A4213D8C37C012B12D882829D
:109CF000FFF798FFB5F9143000EE103A064BB8EEB6
:109D0000C00A1868F7F7B8FE204638BD0320FCE704
:109D10000520FAE70A20F8E73014002038B51A4B7E
:109D20000C46142101FB0433013A05465888042AE5
:109D300013D8DFE802F0030A121D2200F6F7EAFB4F
:109D4000124B0022F6F750FC05E0F6F7E3FB104B50
:109D50000022F6F773FDF6F7F7FE142303FB045316
:109D600000B2588321462846BDE83840FFF75ABF65
:109D7000F6F7D0FB064B0022E4E7F6F7CBFB0246F2
:109D80000B46F6F77BFAE6E7546802080000E03F6E
:109D90000000F83F70B50A46044681BB1A4E33688E
:109DA0005BB3C37C022B28D0012B2AD0033B012BB1
:109DB00027D9FFF747FF9FED150A3068F7F75CFEDC
:109DC0003068F7F7EAFF51EC100BF6F705FF054690
:109DD000F6F7B2FB41EC100B3068F8F70FF89FED87
:109DE0000C0A3068F8F76EFA40B901230146C4F84E
:109DF0001650E3742046FFF715FF002070BD0520C4
:109E0000FCE70B20FAE700BF301400200000000040
:109E10000080BB44F8B5044600295CD1304E306860
:109E200058B3E37C012B58D0033B012B55D90121BA
:109E3000F7F7FCFDE57C1DBBD4F81600F6F77CFBBC
:109E400041EC100B3068F7F793FF3368D4F8160035
:109E5000D3E90167F6F770FB0B46024639463046F8
:109E6000F6F7C2FB41EC100B17F006FF6368C01A4F
:109E7000E06129462046FFF7D5FE00252846F8BDBB
:109E80009FED180A3068F7F7F7FDD4F81600F6F7DB
:109E900053FB41EC100B3068F7F792FFB4F9143024
:109EA000306800EE103AB8EEC00AF7F7E5FDD4F8D6
:109EB0001600F6F741FB41EC100B3068F7F7D0FFC6
:109EC0009FED090A3068F8F7FDF905460028D5D15D
:109ED0000423E374B9E70525D0E70B25CEE700BFDF
:109EE00030140020000000000080BB4430B5104D4D
:109EF0002B6885B004461BB1186803681B6C984733
:109F00000C4B02930C4B0193062300930B48012347
:109F100000224FF47A71FCF7D4FD2B6833B1002195
:109F2000204605B0BDE83040FFF774BF05B030BD36
:109F3000301400204A680208A5A00008180C002070
:109F4000F8B5836A544D01332DED048B83620446CA
:109F5000FFF764FC2B68B0EE409A002B00F098806D
:109F60001868F8F7F5FC63682E68C01AE061F6F728
:109F7000D1FAD6E90123F6F761FCF6F72DFE08EEDB
:109F8000100A3046F8F724F840B9D4F8163007EE36
:109F9000903AB4EE678AF1EE10FA03D1A36A03F5A2
:109FA000967323622868F8F713F8064600286FD1E5
:109FB000E37C012B12D12868F7F766FF002867D0F1
:109FC00028683146F7F732FD0223E374BDEC048BB9
:109FD00020460021BDE8F840FFF724BE042B06D13F
:109FE0002868F7F751FF002852D0E674EEE7002BFF
:109FF0004ED1237A002B49D02848FCF7C5FDB4EE9A
:10A00000499AF1EE10FA28D6D4F80F302F68B4F937
:10A010000D6008EE903AD4F8093078EEC98A07EE60
:10A02000903AD7E9010168EEA78AF6F7D5FD07EE69
:10A03000106A07EE900AB8EEC70A67EEA87A87EEB4
:10A04000800A19F037FA63687043834205D0E169EA
:10A05000606001443868F8F781FC2868F7F714FF5E
:10A06000034678B928680268B3EE040A1377F7F755
:10A07000BBFFA26A236A9A420AD918EE103AC4F8C2
:10A080001630A3E79FED060A2868F0E76360F0E763
:10A09000BDEC048BF8BD00BF30140020180C00206C
:10A0A000000000000148FFF74BBF00BF0014002074
:10A0B000034B00214FF0FF32C3E90A12704700BF83
:10A0C0000014002070B52DED028B1B4D9FED1B8AF7
:10A0D0001B4B1C4A1C4E82B0012401212846F9F773
:10A0E000D3FC2B4621460325184A00941848F8F75C
:10A0F000A5FDB0EE480A2146164B174A00951748B1
:10A10000F7F7A4FA164B174A02213046F9F7BCFCC0
:10A110003346154A009402211448F8F78FFD144B7A
:10A12000144A0095B0EE480A02211348F7F78EFA58
:10A1300002B0BDEC028B70BDF417002000000000DF
:10A140000A6902081A6902089C15002000690208C1
:10A1500058170020C8680208E0680208A01600200E
:10A16000AA680208BA680208A06802080015002060
:10A1700068680208806802084814002000680368C4
:10A18000DB6A1847000000002DE9F0471D461378F0
:10A19000B2B0472BDDE93B7A04460E46904640F0CC
:10A1A000C0815378412B22D12B783BB16A78002AA9
:10A1B00040F0C680482B18D006235EE2022502221A
:10A1C000214622A800F0C8FFA1A3D3E90023DDE9BE
:10A1D0002801F6F709FA41EC100B00950123002243
:10A1E000A3483146FAF7F0FC3EE00325E7E7442BAD
:10A1F00017D12B784BB16A78002A40F0A180482B08
:10A2000001D0652BD8D1032500E00225012221468B
:10A2100022A800F0A1FF8EA3D3E90023DDE92601E7
:10A22000D7E7522B23D12B784BB16A78002A40F024
:10A230008780482B01D0612BBED1032500E0022589
:10A240000122214622A800F087FF83A3D3E900233F
:10A25000DDE92201F6F7C8F92B4641EC100B00228C
:10A2600083483146FAF7D8FB00233B7041E0542B7A
:10A2700019D12B78002B63D190F8603023B97D4938
:10A28000304615F05EFDEFE70068F6F755F974A368
:10A29000D3E90023F6F7A8F941EC100B76493046D4
:10A2A000FAF744FBE0E7582B40F0FA80AA78002A3E
:10A2B00046D12B78342B39D13A706B78303B032B55
:10A2C00030D8DFE803F0021A1C2D6C48F7F765FD63
:10A2D0005FA3D3E9002351EC100BF6F785F90223B5
:10A2E0000093012341EC100B1A4661483146FAF7FE
:10A2F0006BFC012032B0BDE8F0876148E6E75F48BB
:10A30000F7F74BFD52A3D3E9002351EC100BF6F7FE
:10A310006BF941EC100B5B493046FAF707FBE8E7B5
:10A320005748EDE701233B700323A6E1452B36D1C7
:10A330006B78452B2DD005D8342B16D0352B26D055
:10A340000020D7E7462B00F097814D2BF8D14E48DF
:10A350004FF48771FBF739FAC30790D5BE214A48FD
:10A36000FBF7ECF9494902460DE0444BD3E9010102
:10A3700037A3D3E90023F6F761FA41EC100B18F08C
:10A3800067FF43490246304614F0D0FB6CE73C4B74
:10A39000ECE731230B703A9B01221A7064E7462BDD
:10A3A0003BD16B78412B35D005D8332B1AD0342BC9
:10A3B000C6D1334C17E0472BC2D13148F7F7A6FB83
:10A3C00022A8B0EE401AF0EE601A32499FED260B3B
:10A3D00002F05EFC1EA3D3E90023DDE92E01F6F7AF
:10A3E00003F90CE0254C2068F8F701FB0128204612
:10A3F00009D1FFF7C3FE10EE100AF6F79DF841EC05
:10A40000100B20494BE7FFF7B9FEF1EE407A17EE4B
:10A41000900AF2E720493222B5E7542B90D16B78AD
:10A42000442B0DD190ED047AF2EE0E7A67EE277A86
:10A4300017EE900AF6F780F841EC100B17492EE75B
:10A44000522B7FF47DAF90ED037AEDE7AFF3008000
:10A45000F8C1631ADCA54C40C4ACAEA4C88E0E4053
:10A46000DFA1E5F206154E400000000000000000EC
:10A47000020000201167020828690208A0160020C7
:10A48000481400202E690208FC05002076670208A7
:10A4900084710208681900203469020839690208C9
:10A4A0005A2B7FF44DAF2B7873B36A78002A7FF470
:10A4B00047AF482B7FF480AE03250322214602A834
:10A4C00000F04AFEB6A3D3E90023DDE90A01F6F75E
:10A4D0008BF800220023F6F7F9FA03222146A8B1EF
:10A4E00012A800F039FEAEA3D3E90023DDE91A017A
:10A4F000F6F77AF8B04B0022F5F7C0FE41EC100BEE
:10A500000095002301226BE60225D6E722A800F081
:10A5100023FEA3A3D3E90023DDE92A01F6F764F8BB
:10A52000ECE7532B40F0C2815378542B41D122A940
:10A53000284615F019FA229BAB4257EC106B18D045
:10A540009E4B002230463946B04627F00049F6F7C8
:10A55000D1FA30B19A4B002230463946F6F7B6FAB6
:10A5600048B991A3D3E9002340464946F6F7AEFA2D
:10A5700048B9052381E08CA3D3E90023304649463E
:10A58000F6F7A4FA20B10021204600F047FCB0E61F
:10A590008C4B1B78022B3FF4ACAE85A3D3E9002390
:10A5A00030463946F6F74AF9F6F716FB01212060E6
:10A5B000EAE7582B7FF4C4AEAB782C2B7FF4FCADCC
:10A5C0002B78342B40F00F816B78303B042B3FF617
:10A5D000ABAEDFE803F00320306D7100EE1C3046B7
:10A5E00022A915F0C1F9229B55EC104B9E42764EE4
:10A5F0001CD0714B204625F000410022F6F770FA7E
:10A60000A0B167A3D3E9002320462946F6F716F93F
:10A61000C6E900016DE6EE1C304622A915F0A4F94A
:10A62000229B55EC104B9E42684EE1E7684B00229E
:10A63000C6E900239DE7EB78312B7FF45AAE2B79E6
:10A64000002B7FF456AE634D284603F0C3FF00286D
:10A6500040F0C68095F8173195F8162113B19A424B
:10A6600040F2BE80584BD3E9006732463B46304645
:10A670003946F6F753FA18B102238AF8003038E663
:10A68000524DD5E9002310461946F6F747FA00283F
:10A69000F2D194F86130002BEED147EC106B4E48AC
:10A6A000F7F766FB95ED000B4C48F7F761FB20E6EA
:10A6B000002380F861301CE6EE1C304622A915F01C
:10A6C00053F9229B9E4259EC108B4FF0000060D052
:10A6D000394B404629F000410022F6F701FA0028E4
:10A6E00056D02FA3D3E9002340464946F6F7A6F8F3
:10A6F000354DC5E900012C21304615F05AFA00F11C
:10A70000010822A9404615F02FF9229B434557EC3A
:10A71000106B40D0284B304627F000410022F6F75E
:10A72000DFF9002837D0304639461DA3D3E900238E
:10A73000F6F784F806460F46D5E90023DFF88C804B
:10A740001046C8E900671946F6F7E8F9002893D1E2
:10A7500032463B4630463946F6F7E0F900288BD1C1
:10A7600094F86130002B87D11A4C204603F032FF59
:10A77000B0BB94F8173194F816210BB19A422FD937
:10A7800095ED000B1448F7F7F3FA98ED000B8BE703
:10A7900000200F49ACE70E4F0026CDE7AFF3008055
:10A7A000F8C1631ADCA54C409A9999999999B93FD7
:10A7B000DFA1E5F206154E400080764000003E40E5
:10A7C00000805640802000205001002048010020D9
:10A7D0000000F87FB81E0020A016002048140020BA
:10A7E0008AF8000085E5452B0FD16B784D2B7FF45F
:10A7F000A7ADE81C14F0D5F803283FF6BAAEC2B2F4
:10A80000BE21B748FAF708FF73E5542B7FF498ADE3
:10A810006B78442B23D122A9E81C15F0A5F851EC44
:10A82000100BF6F7D9F99FEDAF7A07EE900AF4EE28
:10A83000C77AF1EE10FA0FD49FEDAB7AF4EE477AB7
:10A84000F1EE10FAC8BFF0EE477AF2EE0E6A87EE2C
:10A85000A67A84ED047A4CE5DFEDA27AF5E7522B77
:10A860007FF46EAD22A9E81C15F07EF851EC100BB8
:10A87000F6F7B2F99FED9B7A07EE900AF4EEC77AED
:10A88000F1EE10FA0FD49FED987AF4EE477AF1EEDC
:10A8900010FAC8BFF0EE477AF2EE0E6A87EEA67A9B
:10A8A00084ED037A25E5F0EE477AF5E7542B40F086
:10A8B000DC80297800297FF443AD53786F2B2BD1AE
:10A8C00003232375894B93F94435032B05D1237D4D
:10A8D000032B40F0B080042323759AF80030002B3E
:10A8E0007FF407AD98F801304C2B00F2A9804A2B79
:10A8F00000F2AA802B2B00F0A7802D2B00F0A48063
:10A9000098F801306F2B00F2A2806D2B40F2A280EC
:10A910004FF07E5323609DE0532B35D84A2B05D84A
:10A920002B3BDAB2072A19D9032381E04B3B082BD2
:10A93000FAD801A252F823F0DDA90008E5A9000821
:10A9400029A9000829A9000829A9000829A900089F
:10A95000EDA900082BAA0008D3A90008072BE3D80B
:10A9600001A252F823F000BFF3A9000829A90008AA
:10A9700015AA000829A9000829A9000829A9000882
:10A98000B3A90008BFA900086E2B10D00BD8642B08
:10A9900006D0652BC8D1564B1B78022B47D001211E
:10A9A00000F03CFA8EE7722BBED1012389E70175D6
:10A9B00088E7037D022BF8D0042B83D180E7037D49
:10A9C000012B01D102237CE7032B7FF47BAF04230F
:10A9D00077E700230375474B236073E70023037574
:10A9E000454BF9E700230375444BF5E74FF07E53E1
:10A9F000F2E7434807F047FFF5F77CFD34A3D3E9BE
:10AA00000023F5F739FCF6F7C7F801463C4807F094
:10AA10003DFF57E73A4807F036FFF5F76BFD2CA3EB
:10AA2000D3E90023F5F72AFCEDE73649EEE70A23E0
:10AA30008AF8003046E7012B7FF44FAF02234BE743
:10AA4000513B022B3FF65CAF00233B7058E7722B63
:10AA50003FF45EAF2248092304F11402B521FAF74E
:10AA6000D9FE204600F0FEF843E4242B62D153784F
:10AA7000422B7FF465AC0123234822AAE918FAF798
:10AA800089F900283FF498ABBDF88830BDF98800FB
:10AA9000B3F5616F3FF66DAD2B78442B38D1F5F7E8
:10AAA00039FD0DA3D3E90023F5F7C8FEF6F794F8B6
:10AAB00000EE100AC4F819001448F6F7DDFF084844
:10AAC000092304F11402B521FAF7A4FE11E400BF32
:10AAD0005C55854D55D5B44079AD3173C62D0941CE
:10AAE000FC0500200000E1C40000E14468190020DA
:10AAF000802000200F4D7F3F34E17F3F905D763F07
:10AB0000A82000205979F3000200002048140020FA
:10AB1000522B7FF409ACF5F7FDFC21A3D3E9002308
:10AB2000F5F78CFEF6F758F800EE100AC4F8150099
:10AB30001D48C2E7252B7FF403AC5378422B7FF4EA
:10AB4000FFAB95F80180B8F1000F7FF4F9AB2B78DB
:10AB5000442B1FD1D0F81900F5F7EEFC10A3D3E970
:10AB60000023F5F741FD41EC100B18F0E9FA51EC28
:10AB7000100BF5F7E9FFB0F5616FA8BF4FF4616006
:10AB800020EAE0720949304613F0D0FF87F80080D0
:10AB9000FFF7AFBB522B7FF4C7ABD0F81500DBE754
:10ABA00079AD3173C62D0941A016002076670208E1
:10ABB000006803681B6C184738B5044600F114059B
:10ABC000204890F82C3023B909232A46B521FAF7FA
:10ABD00021FEB5211B4809232A46FAF7C9FD642046
:10ABE00013F072FC18491948F6F7ECFD20B9184A21
:10ABF000137843F004031370D4F81530134800EEB3
:10AC0000103AF6F739FF00211048F7F7F1FA6420FF
:10AC100013F05AFC0F491048F6F7D4FD20B90C4A3E
:10AC2000137843F004031370D4F819300A4800EE87
:10AC3000103AF6F721FFBDE8384007480021F7F742
:10AC4000D7BA00BFFC05002058170020A01600202E
:10AC5000A1110020001500204814002080F8611088
:10AC60007047000038B54D4B1B782DED028B044624
:10AC7000002B40F08A804A4D2B78012B00F2858012
:10AC800090F86020012A1EBF0022426082602A7C68
:10AC90000AB1012B73D1D5ED017A424BD4ED018A73
:10ACA0009FED417A414878EEA78AD3ED007A404B78
:10ACB00078EEA78AD3ED1E7AF8EE677A87EE270A38
:10ACC0009FED3C7AC8EE877A9FED3B7A67EE877AF4
:10ACD00020EE270AF7F788F96B7C13B12B78012B4C
:10ACE00050D1D4ED027A95ED027A314B334837EEEC
:10ACF000878AD3ED1E7A9FED2C7AF8EE677A87EE7D
:10AD0000270A9FED2C7AC8EE077A9FED2B7A67EE23
:10AD1000877A20EE270AF7F767F9F0EEE88AF0EE77
:10AD2000C87AF4EEE87AF1EE10FA9FED257AD8BFF2
:10AD3000F0EE687AF4EEC77AF1EE10FA2CD4B0EEA9
:10AD4000087AF4EEC77AF1EE10FA23DCDFED1D6A23
:10AD500086EEA77AFDEEC77A17EE904A1A4B1A686C
:10AD6000A24209D0214619481C6008F08BFE631EE0
:10AD70005C425C41164B1C70BDEC028B38BDDFEDB4
:10AD8000158AA9E79FED138AC7E79FED120A0B48C2
:10AD9000F7F72AF90124E1E70024DFE7B81E0020D5
:10ADA0005C010020942000205979734BA0160020EC
:10ADB000A8200020F3DB5646B759803F48140020F6
:10ADC000CDCC4C3E0000FA4360190020C8010020A1
:10ADD000A21100200000000038B50C4689B10B4DCF
:10ADE0002B7813B10A4808F00DFE00232B70214682
:10ADF0000848F6F71BFE21460748BDE83840F6F73D
:10AE000015BE80F86010FFF72DFFF0E75801002015
:10AE1000C8010020A01600204814002010B50446E8
:10AE200091B10121FFF7D8FF094B93F844301BB9CA
:10AE3000084B93F8443013B1012384F86030204666
:10AE4000BDE81040FFF70EBF80F86010F7E700BFC5
:10AE5000A0160020481400207FB504462A482B4E37
:10AE60002B4DFFF7A5FE00212748F6F7DFFD294807
:10AE7000FFF79EFE00212748F6F7D8FD264808F088
:10AE8000B5F8304601F098FE00232375234805F0FD
:10AE90004BFA0121214805F0E7FA284606F06CF943
:10AEA0001F4804F087FC96F944351E48022B02BF68
:10AEB0001D4BAB60EB601D4D04F02AFA1C4805F0F9
:10AEC00099FF0026284606F045FE84F8606020467B
:10AED000FFF7C8FE2B78022B03D13146284606F037
:10AEE00055FF144B0293144B019306230093002249
:10AEF00001234FF47A711148FBF7E3FD204604B0BB
:10AF0000BDE87040FFF7AEBEA01600206819002013
:10AF10005C20002048140020A8200020F01F002002
:10AF20005C010020B81E0020DB0FC94080200020FB
:10AF3000382000203F69020835B60008180C0020B0
:10AF400038B510EE100A2DED048BF5F7F5FA40A395
:10AF5000D3E9002304460D46F5F7D6FD002868D155
:10AF60003DA3D3E9002320462946F5F7CDFD00286F
:10AF700062D13BA3D3E9002320462946F5F77EF9A9
:10AF8000F5F72AFE08EE100AB5EEC08A34A3D3E91D
:10AF90000023F1EE10FA2046294648BF9FED288A8B
:10AFA000F5F76AF9F5F718FE08EE900AF5EEC08A93
:10AFB000F1EE10FA18EE100A48BFDFED218AF5F71E
:10AFC000BBFA04460D4645EC104B1E4802F0A8F9AA
:10AFD000204653EC102B2946F5F74EF9F5F7FCFD0A
:10AFE00009EE100A18EE900AF5F7A6FA04460D4687
:10AFF000144845EC104B02F093F9204653EC102B0B
:10B000002946F5F739F9F5F7E7FD07EE900A38EE2E
:10B01000688A39EE679AF7EE007A88EE090AB4EE8C
:10B02000670AF1EE10FAC8BFB0EE670ABDEC048BF8
:10B0300038BD9FED050AF9E79FED040AF6E700BF6A
:10B04000000000006819002020FF7F3FD1FD7F3FF6
:10B0500072532525AF13F93FA0841AC23CFEF83F76
:10B06000E79AD29E46DF713F2DE9F0412DED028B2C
:10B07000074690B03448DFF8D8800E46F6F78DFECC
:10B080003248B0EE408AF0EE608AF6F786FE6C46F3
:10B0900041466846B0EE401AF0EE601AB0EE480A3B
:10B0A000F0EE680A01F0F4FD0FCC07F120050FC5A2
:10B0B0000FCC0FC50FCC0FC594E80F0085E80F002B
:10B0C00098F94435032B07F120012FD1012E01D02F
:10B0D000042E02D11E4802F08BF81B481D4CF6F7D7
:10B0E0005CFED4E90A2351EC100BF5F7C5F80022F9
:10B0F00021F000410023F5F7F3FC90B11348F6F777
:10B100004CFED4E90C2351EC100BF5F7B5F80022F6
:10B1100021F000410023F5F7E3FC10B1002387F88C
:10B12000583010B0BDEC028BBDE8F081022E03D187
:10B13000404602F01BF8D0E7033E012ECDD8404632
:10B1400001F04AFFC9E700BFA01600204814002004
:10B1500068190020F01F002038B50D46044611463E
:10B160002846FFF781FF20460349002305F120020E
:10B1700002F04DFA204638BD6819002070B50C4623
:10B180000646114620462034FFF76EFF0FCC3546A9
:10B190000FC50FCC0FC50FCC0FC594E80F0085E885
:10B1A0000F00304670BD00002DE9F04F2DED048BEF
:10B1B00090F86030A7B004464BB900234360A36009
:10B1C00027B0BDEC048BBDE8F04FFFF74BBD0C4F33
:10B1D00097F94435032B15D0037D9BB9D0ED037A45
:10B1E000F5EE407AF1EE10FA0CD1D0ED047AF5EEDE
:10B1F000407AF1EE10FA05D1036843600023DEE7E0
:10B200006819002004212046FFF72EFF94ED0E7BE5
:10B2100004F12006C24831468DED047BD4E90CAB25
:10B2200002F0EAF997F94435032B03D1BC483146C3
:10B2300001F0DEFF35460FCD0DF1180CACE80F0024
:10B240000FCDACE80F000FCDACE80F0095E80F0074
:10B250008CE80F000FCE0DF1580CACE80F000FCEAC
:10B26000ACE80F000FCEACE80F0095E80F008CE8BB
:10B270000F00AC48FBF788FC9DA3D3E90023DDE970
:10B280000801F4F7FBFF9AA3D3E90023CDE90801F5
:10B29000DDE91801F4F7F0FF97F94435032BCDE908
:10B2A00018010DD106A99E4801F096FE9D48FBF7B6
:10B2B0006BFC9B4816A901F08FFE9A48FBF764FCD3
:10B2C000237DDA1E012A00F2848106A9944802F047
:10B2D000A3F89448FBF758FC16A9914802F09CF893
:10B2E0009048FBF751FC06A98D4801F0B5FC8D484C
:10B2F000FBF74AFC8A4816A901F0AEFC8948FBF727
:10B3000043FC237D022BDDE90A6703D0042B01D027
:10B31000CDE91A672069F5F70FF977A3D3E9002380
:10B32000F5F78CFA804B0022F5F75EF9F5F754FC3F
:10B330000546E068F5F700F96FA3D3E90023F5F7B8
:10B340007DFA794B0022F5F74FF9F5F745FCF5F753
:10B35000F3F88046894602460B46DDE90801F4F71A
:10B360008BFFDDE91823CDE90001CDE90801404656
:10B370004946F4F783FFCDE90201CDE918012846DB
:10B38000F5F7DAF832463B4680468946F4F776FF11
:10B390004B4606460F464246DDE91A01CDE90A67EB
:10B3A000F4F76AFF80465E4890F944358946032BDE
:10B3B000CDE91A8940F01D8106A901F00DFEDDE9F5
:10B3C0000E01F5F709FC0546DDE90C01F5F704FC73
:10B3D00009EE100ADDE91E01F5F7FEFB08EE100A82
:10B3E000DDE91C01F5F7F8FB08EE900A2846F5F7B1
:10B3F000A3F8804618EE100A8946F5F79DF840A399
:10B40000D3E9002306460F4640464946F5F75EFB62
:10B4100088B13DA3D3E9002330463946F5F774FBE4
:10B4200048B13BA3D3E9002340464946F4F726FF41
:10B43000F5F7D2FB054632A3D3E90023304639465F
:10B44000F5F744FB98B12846F5F776F82EA3D3E933
:10B450000023F5F759FB50B12DA3D3E90023304663
:10B460003946F4F70BFFF5F7B7FB08EE100A07EEC5
:10B47000905A77EEC87A9FED2D8A17EE900AF5F76D
:10B480005BF825A3D3E90023F5F7D8F9F5F7A4FB7A
:10B49000D4ED016A07EE900A36EEE77AB0EEC77A8D
:10B4A000B4EEC87AF1EE10FA09D8B2EE027AE6EEFE
:10B4B000877AB2EE047AB0EE676AC6EE077AC4ED18
:10B4C000017A79EE687A17EE900AF5F735F812A34B
:10B4D000D3E90023F5F7B2F9F5F77EFB94F858307D
:10B4E000D4ED026A07EE900A022B21E0AFF3008050
:10B4F000A396CF574B10333FD485BD587EDBCA404F
:10B50000152D4454FB21F9BF152D4454FB21F93F5F
:10B51000182D4454FB211940A396CF574B10433F9D
:10B5200068190020180C0020000010400AD7A33B27
:10B5300008BFF1EE677A36EEE77AB0EEC77AB4EE7E
:10B54000C87AF1EE10FA09D8B2EE027AE6EE877AFE
:10B55000B2EE047AB0EE676AC6EE077A30A3D3E99A
:10B56000002350462BF00041C4ED027AF5F7CCFAE7
:10B5700058B12D4B93F94435032B4FF0000318BFFE
:10B580002268A36008BF1A46626025A3D3E900239E
:10B59000DDE90401F5F7B8FA98B1234B9FED238A52
:10B5A00093F94435032B38D0D4E90E01F5F714FB99
:10B5B00000EE100A2046FFF7C3FC84ED010A84ED7B
:10B5C000028A2046FFF74EFB27B0BDEC048BBDE896
:10B5D000F08F013B012B3FF694AE06A9124801F013
:10B5E0001BFF1348FBF7D0FA0F4816A901F014FF10
:10B5F00084E6DDE90001F5F7EFFA39460546304605
:10B60000F5F7EAFA09EE100ADDE90201F5F7E4FAC6
:10B61000494608EE100A4046E4E6B0EE480ACCE798
:10B62000CFB895CF89BCF73F681900200000000013
:10B63000180C00200148FFF7B7BD00BFF818002024
:10B64000084B4FF07E5200211A6000225A609A6027
:10B65000DA601A611975C3F81520C3F81920A3F828
:10B6600060107047F8180020F8B500F2A4452023B8
:10B670002A46EE2104465648FAF77AF82868F4F785
:10B680005BFF4FA3D3E9002306460F46F5F71EFAEA
:10B6900038B94DA3D3E9002330463946F5F734FADB
:10B6A00008B100232B6004F595652868F4F744FF82
:10B6B00043A3D3E9002306460F46F5F707FA38B946
:10B6C00041A3D3E9002330463946F5F71DFA08B106
:10B6D00000232B6004F2BC43D3ED007A9FED3D7A4A
:10B6E000F4EEC77AF1EE10FA06D4DFED3B6AF4EE21
:10B6F000E67AF1EE10FA01DD00221A6004F5986393
:10B70000D3ED007ADFED356AF4EEE67AF1EE10FA69
:10B7100006D4DFED336AF4EEE67AF1EE10FA01DDDD
:10B7200000221A6004F2B443D3ED007ADFED2D6AF3
:10B73000F4EEE67AF1EE10FA06D4DFED2B6AF4EEC1
:10B74000E67AF1EE10FA01DD00221A6004F5976343
:10B75000D3ED007AF4EEC77AF1EE10FA06D49FED3D
:10B760001E7AF4EEC77AF1EE10FA01DD00221A60BB
:10B7700004F2AC43D3ED007A9FED1C7AF4EEC77A65
:10B78000F1EE10FA06D4DFED1A6AF4EEE67AF1EE85
:10B7900010FA01DD00221A6004F59664D4ED007AF7
:10B7A000F4EEC77AF1EE10FA06D49FED117AF4EEBA
:10B7B000C77AF1EE10FA01DD00232360F8BD00BF67
:10B7C000182D4454FB2119C0182D4454FB21194055
:10B7D000FC050020000080C300008043000000C37F
:10B7E00000000043000000C600000046000080C6C4
:10B7F0000000804600F2A44220230248EE21FAF71E
:10B8000009B800BFFC0500200F4B002200F2A44144
:10B810001A7000230B6000F595610B6000F2AC41DB
:10B820000B6000F596610B6000F2B4410B6000F50F
:10B8300097610B6000F2BC410B6000F598610B60F2
:10B8400080F8C424704700BF6419002038B50D4645
:10B850002DED028BFFF7D8FF032D0446F0EE408A52
:10B8600014D016F031FEB0EE408AB0EE680A16F041
:10B87000FFFF84F8C55404F5996383ED008ABDEC9D
:10B88000028B04F2CC4484ED000A38BD9FED028A9D
:10B89000B7EE000AEDE700BF2EBD3BB31FB590F831
:10B8A0004035044673B9084A08481170084A0292A4
:10B8B000084A01920622009201211A46FBF701F97B
:10B8C00084F8400504B010BD64190020180C002055
:10B8D0004669020809C600082DE9F04F85B090F8C6
:10B8E00040A5DDF838900192054688461F46BAF11A
:10B8F000000F65D14E1E082E62D8531E082B5FD84C
:10B90000D9E90201F5F768F92C2404FB06540390E9
:10B910002062D9E90401F5F75FF960620290D7E986
:10B920000201F5F759F9C4F8AC018346D7E90401DF
:10B93000F5F752F9C4F8B00195F9C5140329DDE90A
:10B94000023238D12048494601F046FBD9E90801C6
:10B95000F5F742F92060D9E90601F5F73DF93946D6
:10B96000A060194801F038FBD7E90801F5F734F970
:10B97000C4F88C01D7E90601F5F72EF92C2303FB57
:10B98000065699F83830C6F89401022B0CBF4FF0D8
:10B99000FF330123B8F1010FC6F8B431B36206D00A
:10B9A000019B984503D141462846FFF777FF504653
:10B9B00005B0BDE8F08F2260A360C4F88CB1DDE76C
:10B9C0004FF0070AF3E700BF681900202DE9704324
:10B9D0002DED108B91ED06EAD1ED058A91ED07DA98
:10B9E000D1ED04BAB7EE007AC7EE0E7A1D4600F527
:10B9F000996300F2CC4016460C4660EE800AD3ED07
:10BA000000FAD0ED009A27EEA0FAD1ED0A7AF8EE0E
:10BA1000E7CA6FEEA87A21EE401A17EE900A20EEE0
:10BA200021CA20EE23AA21EE0DBA20EE028A60EE92
:10BA300003DAB0EE409AF0EE62AAF4F77DFD80469C
:10BA40001EEE100A8946F4F777FD02460B460020E9
:10BA50002349F4F7F3FE02460B4640464946F4F705
:10BA6000C3FD80461AEE100A8946F4F765FD0246CA
:10BA70000B4640464946F4F7B7FDF5F7ADF868EEDA
:10BA8000887A6CEE6B6A67EE8D7A07EE100AEDEE3F
:10BA9000267A6DEE29EAEFEE2C7AEFEEABEAECEEC9
:10BAA0008B7A6AEEC9AA77EE877A69EECE9AC6EDEE
:10BAB000007AD4ED047A28EE278AD4ED057AA7EE31
:10BAC0008C8AEFEEAB9AAAEEAE8AABEEAD8AA9EE07
:10BAD0008A8A85ED008ABDEC108BBDE8708300BFBB
:10BAE0000000F03F000000002DE9F04F2DED108B1D
:10BAF00004468DB010EE100AB0EE408A16461D4680
:10BB00000F46F4F719FD0FF21063D3E90023F4F7A1
:10BB100095FEF5F761F804F59C6393ED000A80EE5D
:10BB2000080A0DEE100A16F081F87B4209EE103A71
:10BB3000B8EEC99A04F2E44339EE009AFDEEC97AF0
:10BB4000CDED027A07EE907AF8EEE77A37EE800ACA
:10BB5000BDEEC09A93ED000A80EE080A16F066F872
:10BB6000734209EE903AF8EEE99A04F59D6379EE96
:10BB7000809AFDEEE97ACDED037A07EE906AF8EE51
:10BB8000E77A37EE800AFDEEC09A93ED000A80EE68
:10BB9000080A16F04BF86B420AEE103AB8EECAAA41
:10BBA00004F2EC433AEE00AAFDEECA7ACDED047A37
:10BBB00007EE905AF8EEE77A37EE800ABDEEC0AA9B
:10BBC00093ED000A80EE080A16F030F8269B5B42DF
:10BBD0000AEE903AF8EEEAAA04F5A0637AEE80AA9B
:10BBE000FDEEEA7ACDED057ADDED267AF8EEE77A1C
:10BBF00037EE800AFDEEC0AA93ED000A80EE080A37
:10BC000016F014F8279B5B420BEE103AB8EECBBA55
:10BC100004F5A1633BEE00BAFDEECB7ACDED067ADA
:10BC2000DDED277AF8EEE77A37EE800ABDEEC0BA8E
:10BC300093ED000A80EE080A15F0F8FF289B5B429E
:10BC40000BEE903AF8EEEBBA04F204537BEE80BAB6
:10BC5000FDEEEB7ACDED077ADDED287AF8EEE77AA6
:10BC600037EE800AFDEEC0BA93ED000A80EE080AB6
:10BC700015F0DCFF299B5B420CEE103AB8EECCCA03
:10BC800004F2FC433CEE00CAFDEECC7ACDED087A1E
:10BC9000DDED297AF8EEE77A37EE800ABDEEC0CA0C
:10BCA00093ED000A80EE080A15F0C0FF2A9B5B4264
:10BCB0000CEE903AF8EEECCA04F59F637CEE80CA75
:10BCC000FDEEEC7ACDED097ADDED2A7AF8EEE77A31
:10BCD00077EE807A93ED000A80EE080AFDEEE7CA5F
:10BCE00015F0A4FF2B9B5B4207EE903AF8EEE77A43
:10BCF00077EE807AFDEEE7FADDED2B7AF8EEE77A63
:10BD000077EE807ABDEEE7FA1FEE903A1FEE102A2A
:10BD1000934240F3FD810DB0BDEC108BBDE8F08F78
:10BD200007EE90AAB8EEE7EAF8EEEFEA2EEE0DEA9B
:10BD300004F5A56383ED00EA6EEE8DEA04F5A663D3
:10BD4000F1EE4E7AC3ED007A04F22453C3ED00EA1B
:10BD5000D4F8D07404F22C53C3ED00EA2546002633
:10BD6000B74213DC029B0093009B19EE102A93420A
:10BD700040F3CC810AF1010A1CEE903A9A45CFDDDE
:10BD80001FEE903A01330FEE903ABDE7AB6AD5ED66
:10BD900000DAD5ED028A5A1C22D17DEEAEDA78EEB9
:10BDA000CE8AC5ED01DAC5ED038AB0EE6D0A16F054
:10BDB0005FFD85ED050AB0EE6D0A16F085FB85ED99
:10BDC000040AB0EE680A16F07FFB85ED060AB0EEB5
:10BDD000680A16F0D5FD013685ED070A2C35BFE758
:10BDE000012B04BF7DEEAEDA78EE8E8AD9E707EE3E
:10BDF00090BAB8EEE72ADDED017AF8EEE71A07EE21
:10BE0000906AB8EEE71ADDED007A0BABF8EEE70AC0
:10BE10000AAAF8EEEE3AB8EECE3AF8EEED2AB0EE17
:10BE20004D0A29462046FFF7D1FD9DED0A7AD5ED52
:10BE3000017AD5ED638A77EEC77A78EEE78A18EE55
:10BE4000900AF4F779FBBCA3D3E900238046894626
:10BE5000F4F75AFE002800F01B81B3A3D3E90023B6
:10BE600040464946F4F708FAF4F7B6FE08EE900AA1
:10BE700095ED037ADDED0B7AAB6AC5EDC68A37EE38
:10BE8000677AD5ED657AC5F8403377EEC77A013722
:10BE9000C5EDC87A2C35D4F8D084B845A7DCDFEDE1
:10BEA000A48A04F5CA75002704F5A769B845C9ED49
:10BEB000008A05F12C0500F3008108F1FF3307EE3D
:10BEC000903AF8EEE77A9FED9A7A88EEA76A04F541
:10BED0004872002304F5A761984502F12C0281ED18
:10BEE000007A00F3F68087EE270A30EE060A16F095
:10BEF00051FA04F23C5383ED000A04F5A463D3ED38
:10BF0000007AB4EEE70AF1EE10FA40F18780DDED39
:10BF1000007A83ED000AF8EEE77A04F59C6367EE99
:10BF2000887AB8EEEE7AC3ED007A07EE906AF8EE02
:10BF3000E77A04F2E44367EE887A27EE087AC3EDE5
:10BF4000007ADDED017AF8EEE77A04F59D6367EE9D
:10BF5000887A04F2F445C3ED007A07EE90BAF8EE61
:10BF6000E77A04F2EC4367EE887AC3ED007A04F5D1
:10BF7000A06383ED007AB8EEED7A04F2045327EE65
:10BF8000087A83ED007AB8EECE7A04F5A16327EE45
:10BF9000087A83ED007A2A9B002B00F0A08004F53C
:10BFA000A6631868F4F7C8FA5BA3D3E90023F4F793
:10BFB0001BFBF4F711FE04F5A56328601868F4F77D
:10BFC000BBFA55A3D3E90023F4F70EFBF4F704FE04
:10BFD00007EE900A04F2FC43C3ED007A2B9BEBB111
:10BFE00004F22C5304F59E651868F4F7A5FA4AA3E9
:10BFF000D3E90023F4F7F8FAF4F7EEFD04F2245342
:10C0000028601868F4F798FA43A3D3E90023F4F7FB
:10C01000EBFAF4F7E1FD04F59F6528604548FAF76F
:10C02000B3FD1EEE903A01330EEE903A1EEE903ABA
:10C030001BEE102A93423DDD1EEE103A01330EEE48
:10C04000103A1EEE103A1BEE902A934250DD1DEE80
:10C05000903A01330DEE903A1DEE903A1CEE102A04
:10C06000934248DD0BF1010B1AEE903A9B4545DDFA
:10C07000019B01330193019B1AEE102A934240DD8C
:10C08000013619EE903A9E423EDD009B01336AE68E
:10C0900023A3D3E9002340464946F4F717FD0028BF
:10C0A0003FF4E6AE20A3D3E9002340464946F4F727
:10C0B000E5F8D9E625460027EDE615ED0B0A16F062
:10C0C00003FAD5ED567A20EE270A0137E0EE008A12
:10C0D000ECE652ED0B6A0133A6EEA67AFCE6B6EE6C
:10C0E000007A67EE877AC5ED007AF1EE677A71E73C
:10C0F000DDED06EA9AE79DED07EAA2E7DDED08DA55
:10C10000AAE7DDF814B0AFE7049BB3E7039EB8E7F6
:10C11000DDF824A030E600BF79AD3173C62D0941AA
:10C12000182D4454FB2109C0182D4454FB211940FB
:10C1300000000000180C0020182D4454FB21094079
:10C140002DE9F04F2DED028B00F5A463DFEDD67ADB
:10C15000D64AC0F8D0148BB0002680F8C46400F52D
:10C160009C6A1A6000F2E44900F2EC4300F59D6815
:10C17000CAED007A0793C9ED007AC8ED007AC3EDE5
:10C18000007A00F5A063C3ED007A00F5A163C3ED6A
:10C19000007A00F20453C3ED007A00F2FC43044637
:10C1A0000D46C3ED007AB0EE678A4FF02C0BB54216
:10C1B00000F3948107EE905AB8EEE77A04F2245324
:10C1C000C8EE077AC4F8D46404F59E6BC3ED007A18
:10C1D00017EE900AF4F7B0F9B1A3D3E90023F4F70E
:10C1E00003FA41EC100B16F0ABFF51EC100BF4F717
:10C1F000F3FC04F59F631860CBF8000094F9C53494
:10C20000032B00F0A981022B0BBF01230023002286
:10C21000012201260027022DD4BF00250125C4F8E4
:10C22000D834C4F8DC249FEDA20A33463A46394696
:10C230002046CDE90466CDE90277CDE90067FFF736
:10C2400053FC9FED9C0A33463A4629462046CDE9E9
:10C250000466CDE90277CDE90067FFF745FC9FED65
:10C26000960A33463A4629462046CDE90466CDE98A
:10C270000277CDE90067FFF737FC9FED900A334660
:10C280003A4629462046CDE90466CDE90277CDE954
:10C290000067FFF729FC9FED8A0A33463A46294694
:10C2A0002046CDE90466CDE90277CDE90067FFF7C6
:10C2B0001BFC3346CDE90466CDE90277CDE9006782
:10C2C0009FED800A3A4629462046FFF70DFCD4F838
:10C2D000D034042BCDE9046640F34181D4F8DC343A
:10C2E0000393D4F8D8349FED780A0096CDE9017312
:10C2F0003246334629462046FFF7F6FBCDE9046671
:10C30000D4F8DC340393D4F8D8349FED700A009647
:10C31000CDE901633246334629462046FFF7E4FB68
:10C32000CDE90466D4F8DC340393D4F8D8349FED17
:10C33000680A0096CDE90163324633462946204615
:10C34000FFF7D2FBCDE90466D4F8DC340393D4F8CC
:10C35000D8349FED600A0096CDE90163324633463A
:10C3600029462046FFF7C0FBCDE90466D4F8DC344B
:10C370000393D4F8D8340096CDE9016332463346AE
:10C38000B3EE000A29462046FFF7AEFBDAF80000BC
:10C39000F4F7D2F842A3D3E90023F4F74FFAF4F705
:10C3A0001BFC04F2B4452860D9F80000F4F7C4F887
:10C3B0003BA3D3E90023F4F741FAF4F70DFC04F5AD
:10C3C00097652860D8F80000F4F7B6F834A3D3E9ED
:10C3D0000023F4F733FAF4F7FFFB04F59665079BA7
:10C3E00028601868F4F7A8F82DA3D3E90023F4F720
:10C3F00025FAF4F7F1FB04F2AC4504F5A0632860DC
:10C400001868F4F799F826A3D3E90023F4F716FA8D
:10C41000F4F7E2FB04F59865286094F8C534023B14
:10C42000012B94BF04F5A16304F2045304F2A44564
:10C430001868F4F781F81AA3D3E90023F4F7FEF99A
:10C44000F4F7CAFB04F2BC431860DBF80000F4F711
:10C4500073F813A3D3E90023F4F7F0F9F4F7BCFB66
:10C4600004F2F44328601868F4F766F80CA3D3E9E3
:10C470000023F4F7E3F9F4F7AFFB04F59565012326
:10C48000286094F8401584F8C4341348FAF744FA45
:10C49000002384F840350BB0BDEC028BBDE8F08F73
:10C4A00079AD3173C62D09410000000000341E49EA
:10C4B0000000804600000046000080450000004566
:10C4C000000080440000004400008043000000435E
:10C4D0000000804200000042180C00200BFB0643C5
:10C4E000D3ED638AD3ED007A78EEE78A18EE900AEE
:10C4F000F4F722F802460B46CDE908233CA3D3E922
:10C500000023F4F701FB50B13BA3D3E90023DDE99D
:10C510000801F3F7B1FEF4F75FFB08EE900A18EE9E
:10C52000900AF4F709F802460B46CDE9082334A334
:10C53000D3E90023F4F7CAFA50B12FA3D3E90023BB
:10C54000DDE90801F3F79AFEF4F746FB08EE900ADE
:10C5500038EE288A01362AE600231A4659E69FED6E
:10C56000200A33463A4629462046CDE90277CDE9EE
:10C570000067FFF7B9FA9FED1B0A33463A46294692
:10C580002046CDE90466CDE90277CDE90067FFF7E3
:10C59000ABFA9FED150A33463A4629462046CDE9C7
:10C5A0000466CDE90277CDE90067FFF79DFA3346CF
:10C5B0003A46CDE90466CDE90277CDE900679FED03
:10C5C0000B0A29462046FFF78FFACDE90466CDE92C
:10C5D0000277CDE9006733463A46D1E6AFF30080F3
:10C5E0000000804300000043000080420000004241
:10C5F000182D4454FB210940182D4454FB211940A7
:10C60000182D4454FB2109C0024B03481978FFF749
:10C6100097BD00BF641900206819002000000000C9
:10C620002DE9F0412DED108B90F8C43484B0044610
:10C630000D46002B00F0EF8091F8383090F9C5845A
:10C64000022BBFEE00AAF7EE007A18BFB0EE67AA81
:10C65000B8F1030F40F0E480D1E90801F4F7BCFA27
:10C6600009EE900AD5E90601F4F7B6FA09EE100AC8
:10C67000F3F762FF78A3D3E9002306460F46F4F7E9
:10C6800043FA002840F0D58075A3D3E90023304653
:10C690003946F4F71BFA002840F0CE80F0EEC97A54
:10C6A00017EE900AF3F748FF6FA3D3E90023F4F7DE
:10C6B0000DFA002800F0C38004F2B443D3ED00FA71
:10C6C00004F5976393ED00BA04F59863D3ED00BACF
:10C6D00004F5996393ED00DA04F2CC43D3ED00DA6C
:10C6E00004F5966393ED00CA04F2AC43D3ED00CA9F
:10C6F00004F2BC4393ED00EAA8F10207B1EE4BBA95
:10C70000F1EE4CEAF1EE4E6AB0EE498AF0EE698A3B
:10C710000326B7EE006AFFB2B1EE6DFAB0EE480A3A
:10C720008DED036ACDED026A16F0A2F88DED010AD7
:10C73000B0EE480A15F0C8FE8DED000AB0EE680AAA
:10C7400016F096F8F0EE40AAB0EE680A15F0BCFEBE
:10C750009DED007ADDED015A9DED036ADDED026A83
:10C7600085EE875A012FC6EE073A6DEE005A6DEE40
:10C770002A4A88BFB0EE658AEFEE075A2CEEAA7AF5
:10C780002FEEA34A64EEA34A27EE057A6EEE803AB6
:10C7900088BFA5EE2D8AA5EE237A6BEE058A6CEE96
:10C7A000807A68EE8A8AECEE2A7A94BF20EE0E8AAE
:10C7B00026EE888A24EE0A4A78EE878A38EE278A9F
:10C7C00078EE848AABEEA58A013EEBEEA48A38EEC1
:10C7D000098A78EEA98AA1D1F0EE689A04F2A443FE
:10C7E000D3ED007A04F5956494ED007A79EEE77A5A
:10C7F000A7EE0A8A17EE900AF3F79EFE064618EE99
:10C80000100A0F46F3F798FEB8F1030F1AD1C5E9E5
:10C810000867C5E9060104B0BDEC108BBDE8F081E6
:10C82000D1E90201F4F7D8F909EE900AD5E904013B
:10C830001AE79FED078AD1E79FED068ACEE7B0EEB3
:10C84000498ACBE7C5E90267C5E90401E3E700BF10
:10C85000DB0FC93FDB0FC9BF152D4454FB21F93F46
:10C86000152D4454FB21F9BFAEA6F439CA20F93F77
:10C870002DE9F04790F8C4342DED068B04468A4626
:10C88000002B00F0088191F8383090F9C554022B44
:10C89000BFEE00AAF7EE007A18BFB0EE67AA032D2C
:10C8A00040F0FD80D1E90801F4F796F908EE100A8E
:10C8B000DAE90601F4F790F904F2A443D3ED007A23
:10C8C00004F5956308EE900A38EE278AD3ED007AD6
:10C8D000EAEE678A18EE900AF3F72EFEB0A3D3E9CA
:10C8E000002306460F46F4F70FF9002840F0E080D9
:10C8F000ADA3D3E9002330463946F4F7E7F8002822
:10C9000040F0D980F0EEE87A17EE900AF3F714FEC3
:10C91000A7A3D3E90023F4F7D9F8002875D0B0EE27
:10C92000680A15F0A5FFF0EE40AAB0EE680A15F00F
:10C93000CBFDF0EE409AB0EE480A15F099FFB0EE4C
:10C94000409AB0EE480A15F0BFFDCAEEA93A04F2CB
:10C95000B443F7EE007A87EEA96A93ED005A04F526
:10C960009763D3ED007A04F2BC4393ED007A04F5AB
:10C970009963D3ED006A04F2CC43D3ED002AAB1ED9
:10C9800060EE264ADBB2012B84BFB0EE644AA3EE10
:10C99000A24A04F59863E9EEE24A69EE266A93ED4D
:10C9A000003A04F5966304F2AC4426EE055A26EEEE
:10C9B000866AD4ED006AD3ED002A88BF27EE447A58
:10C9C000B0EE644A66EE894A22EEC02A64EEA34ABB
:10C9D00067EEE37AE3EE824A66EE806A67EE8A7A71
:10C9E000E2EE896A25EE0A5A98BF20EE077A77EEC2
:10C9F000A47A37EE267A77EE857AA3EE047AE3EE10
:10CA0000067A78EEC78A38EE678A18EE900AF3F74E
:10CA100093FD63A3D3E9002306460F46F4F774F8A9
:10CA200000284BD160A3D3E9002330463946F4F700
:10CA30004DF8DFED597A002818BFF0EE678A032D14
:10CA40003FD14DA7D7E9006718EE100AF3F774FD40
:10CA500032463B4604460D46F4F756F800285DD1B1
:10CA600047A7D7E900670FF21019D9E9008918EE36
:10CA7000100AF3F761FD32463B4604460D46F4F7D3
:10CA800025F8002855D1CAE9084518EE900AF3F7B1
:10CA900053FDCAE90601BDEC068BBDE8F087D1E97C
:10CAA0000201F4F799F808EE100ADAE9040101E747
:10CAB000DFED3A8AA9E7DFED388AA6E7DFED378AAE
:10CAC000BDE70FF2C409D9E900892BA7D7E90067B0
:10CAD00018EE100AF3F730FD42464B4604460D4669
:10CAE000F4F712F880BB0FF2A809D9E9008922A750
:10CAF000D7E9006718EE100AF3F71EFD42464B46D1
:10CB000004460D46F3F7E2FF48BBCAE9024518EEBA
:10CB1000900AF3F711FDCAE90401BCE732463B462F
:10CB200020462946F3F7A8FBF4F756F808EE100A5A
:10CB30008AE742464B4620462946F3F79FFBF4F727
:10CB40004BF808EE100A92E732463B46204629464B
:10CB5000F3F792FBF4F740F808EE100AB8E7324614
:10CB60003B4620462946F3F789FBF4F735F808EEF3
:10CB7000100ABFE7AFF30080182D4454FB21194081
:10CB8000182D4454FB2119C0182D4454FB21094091
:10CB9000182D4454FB2109C0DB0FC9BFDB0FC93F6F
:10CBA000152D4454FB21F93F152D4454FB21F9BFA9
:10CBB000AEA6F439CA20F93F38B5214D04464FF4EA
:10CBC00087712846F8F701FE95F82C300BB1C307A2
:10CBD00004D41B480122BE21F8F71EFD1848BE21CF
:10CBE000F8F7ACFD43B2D3B90122154884F84425C7
:10CBF000BE21F8F711FD94F94455EB1E18BF01232F
:10CC000084F845350F4BD3E90001F3F7E5FF2946DA
:10CC100000EE100A2046BDE83840FEF717BE013886
:10CC2000C0B2022881BF0123074A84F84435137833
:10CC300092BF84F8443543F002031370DBE700BF72
:10CC4000FC050020A8200020A111002091F8383018
:10CC50000BB1FFF70DBE704738B591F83830054677
:10CC60000C460BB1FFF7DCFC95F94435032B08D1DA
:10CC7000D4E90823C4E90A23D4E90623C4E90C2330
:10CC800038BDD4E90223C4E90A23D4E90423F5E733
:10CC90002DE9F84355EC114B06460F4630A3D3E976
:10CCA00000232046294659EC108BF3F70FFF40B9BB
:10CCB0002DA3D3E9002320462946F3F725FF0028BA
:10CCC00034D02BA3D3E9002340464946F3F7D4FAE6
:10CCD0002B4622468046894625A1D1E90001F3F77B
:10CCE000CBFA022304460D4686F83830204620A3AE
:10CCF000D3E900232946F3F707FFC8B11EA3D3E900
:10CD0000002320462946F3F7B7FA04460D4697F963
:10CD10004435032B1DD1C6E90889C6E90645C6E995
:10CD20000A89C6E90C453046BDE8F8830123DBE7F4
:10CD300013A3D3E9002320462946F3F7D1FE0028A8
:10CD4000E5D00DA3D3E9002320462946F3F796FA50
:10CD5000DBE7C6E90289C6E90445E0E7AFF30080F6
:10CD6000152D4454FB21F9BF152D4454FB21F93FE7
:10CD7000182D4454FB210940182D4454FB2119401F
:10CD8000182D4454FB2109C0F8B51C4690F94435D0
:10CD9000032B154639D1D1E90823C5E90023D1E990
:10CDA0000623C4E9002391F83830022B19D126A3B9
:10CDB000D3E90023D5E90001F3F760FAC5E90001E2
:10CDC000294900220023D1E90001F3F793FED4E9B9
:10CDD000002308B31CA1D1E90001F3F74DFAC4E91F
:10CDE0000001D4E900671AA3D3E90023304639468D
:10CDF000F3F78AFEA0B116A3D3E9002330463946E3
:10CE0000F3F73AFAC4E90001F8BDD1E90223C5E914
:10CE10000023D1E90423C4E70FA1D1E90001DCE735
:10CE20000FA3D3E9002330463946F3F74FFE00281D
:10CE3000EAD007A3D3E9002330463946F3F71EFAB8
:10CE4000E0E700BFAFF30080182D4454FB210940F8
:10CE5000182D4454FB211940182D4454FB2109C0BE
:10CE6000182D4454FB2119C0A82000200000000008
:10CE70002DE9F0478A46164672B6234B186862B60B
:10CE8000F3F738FB1CA3D3E90023F3F7D7FCDAE967
:10CE90000223F3F7F1F904460D46B6B118A7D7E916
:10CEA000006732463B4620462946F3F723FE80B909
:10CEB0000FF24C09D9E900890026002732463B468B
:10CEC00020462946F3F702FE60B9CAE90045BDE8ED
:10CED000F0872046294632463B46F3F7CDF9044613
:10CEE0000D46DEE72046294642464B46F3F7C6F993
:10CEF00004460D46E2E700BF921054B57AFB444168
:10CF0000182D4454FB211940282100200000000066
:10CF10002DE9F0471646D1E900238A461046194606
:10CF2000F3F7FCFD78BB72B6294B186862B6F3F7CD
:10CF3000E1FA1FA3D3E90023F3F780FCDAE9002329
:10CF4000F3F79AF904460D46DEB11BA7D7E900674F
:10CF50000FF26C09D9E9008932463B462046294642
:10CF6000F3F7C8FD88B90FF26009D9E9008914A761
:10CF7000D7E9006742464B4620462946F3F7A6FD0F
:10CF800060B9CAE90245BDE8F08720462946424615
:10CF90004B46F3F771F904460D46DDE72046294676
:10CFA00032463B46F3F76AF904460D46E2E700BF16
:10CFB000921054B57AFB4441182D4454FB2109408A
:10CFC000182D4454FB211940182D4454FB2109C04D
:10CFD00028210020000000002DE9F84F2DED048BE2
:10CFE00091ED029B8A46B0EE490AF0EE690A15F00F
:10CFF0007BFC9AED048B55EC104BB0EE480AF0EE3A
:10D00000680A15F0F5FC59EC108BB0EE480AF0EE0A
:10D01000680A15F069FCDFF850B151EC100BDBE940
:10D020000C23F3F7E1FA22462B46F3F7DDFADBE9AE
:10D030000A2306460F4640464946F3F7D5FA02460C
:10D040000B4630463946F3F719F941EC100B14F052
:10D0500051FE3DA3D3E900238AED060B51EC180BDA
:10D06000F3F70AF93AA3D3E9002321F00041F3F7DB
:10D070002DFD002854D134A3D3E9002351EC180B23
:10D08000F3F7FCF832A3D3E9002321F00041F3F7D2
:10D090001DFD002847D1B0EE480AF0EE680A15F0F1
:10D0A000EFFC57EC106BB0EE490AF0EE690A15F090
:10D0B0009FFCDBE90A23B0EE408AF0EE608A20464E
:10D0C0002946F3F791FADBE90C2304460D46304676
:10D0D0003946F3F789FA02460B4620462946F3F70C
:10D0E000CBF8B0EE480AF0EE680A41EC110B14F0F0
:10D0F00035FE19A3D3E9002351EC100BF3F7BEF86A
:10D1000004460D4614A3D3E9002320462946F3F72D
:10D11000FBFC60B9CAE90845BDEC048BBDE8F88F9B
:10D1200000240025EEE70CA5D5E90045EAE70CA3AD
:10D13000D3E9002320462946F3F79EF8CAE90801FF
:10D14000EAE700BFAFF30080152D4454FB21F93FFF
:10D150002010238F8444A03E182D4454FB21094005
:10D16000182D4454FB211940A82000202DE9F84334
:10D1700091ED020B2DED028B0C4615F0B5FB94EDF5
:10D18000048B57EC106BB0EE480AF0EE680A15F00D
:10D190002FFC59EC108BB0EE480AF0EE680A15F03F
:10D1A000A3FB114D51EC100BD5E90C23F3F71CFA3E
:10D1B00032463B46F3F718FAD5E90A2306460F46EE
:10D1C00040464946F3F710FA02460B4630463946C8
:10D1D000F3F754F841EC100B14F08CFDBDEC028B0E
:10D1E00084ED060BBDE8F883A820002000000000B5
:10D1F0002DE9F84F2DED048B91ED088B8A46B0EEAA
:10D20000480AF0EE680A15F06FFB9AED069B55ECA4
:10D21000104BB0EE490AF0EE690A15F0E9FB59EC43
:10D22000108BB0EE490AF0EE690A15F05DFBDFF8ED
:10D23000E8B051EC100BDBE90C23F3F7D5F92246EB
:10D240002B46F3F7D1F9DBE90A2306460F464046A1
:10D250004946F3F7C9F902460B4630463946F3F71B
:10D260000DF841EC100B14F045FD8AED040BB0EE07
:10D27000480AF0EE680A15F0BBFBB0EE408AF0EE0B
:10D28000608AB0EE490AF0EE690A15F0F9FBDBE9B5
:10D290000A232046294657EC106BF3F7A5F9DBE982
:10D2A0000C2304460D4630463946F3F79DF90246F5
:10D2B0000B4620462946F2F7DFFFB0EE480AF0EEB3
:10D2C000680A41EC110B14F049FD0FA3D3E90023C8
:10D2D00051EC100BF2F7D2FF0BA3D3E90023044665
:10D2E0000D46F3F711FC40B12046294608A3D3E9C7
:10D2F0000023F2F7C1FF04460D46BDEC048BCAE9DA
:10D300000245BDE8F88F00BF182D4454FB210940A9
:10D31000182D4454FB211940A820002000000000D3
:10D3200038B537482DED048B55EC104BFAF7D0FB90
:10D33000B4EE400AF1EE10FA9FED329A4FD6304823
:10D34000FAF7C6FBF0EE408A2D48FAF7A1FBB4EEDF
:10D35000400AF1EE10FA45D62948FAF799FBB0EEEB
:10D36000408A23A3D3E9002320462946F2F786FF0B
:10D3700002460B4620A1D1E90001F3F75FFA2246ED
:10D380002B46F2F77BFFF3F727FC00EE100A15F0AF
:10D39000F7FADFED1D7A9FED1D7A38EE278AF7EE5A
:10D3A000006AC7EE087A88EE897A67EE877A86EE99
:10D3B000807ADFED176A27EE267A67EE877AF5EE38
:10D3C000C07AF1EE10FA48BFDFED127A17EE900A3C
:10D3D000F3F7B2F8BDEC048B41EC100B38BDF0EE66
:10D3E000498AB1E7B2EE048ABBE700BFAFF3008021
:10D3F00000000040EAD4B63F00000060F0B3693F8F
:10D400001800002000807C440080884300808D4309
:10D41000348F9B3900000000F8B590F94435032B98
:10D4200005460C4636D0D1E9046721A3D3E9002391
:10D4300030463946F2F720FF1FA3D3E9002321F03D
:10D440000041F3F743FB88BB19A3D3E9002330461F
:10D450003946F2F713FF18A3D3E9002321F0004166
:10D46000F3F734FB10BB21462846FFF7B5FD2846ED
:10D4700094ED060BFFF754FFD4E9060153EC102B93
:10D48000F2F7FCFEC4E9060121462846BDE8F84053
:10D49000FFF7AEBE91ED060BFFF742FFD4E90601A0
:10D4A00053EC102BF2F7EAFEC4E90601F8BD00BF09
:10D4B000152D4454FB21F93FD8D7FDB2A555D43ED4
:10D4C00038B504460D46FFF7A7FF29462046BDE8BC
:10D4D0003840FFF7C1BBF8B50546174601221E4686
:10D4E0000C46FFF715FD95F94435032B03D1214672
:10D4F0002846FFF771FD21462846FFF7E1FF67B197
:10D500005EB195F94435032B08D1D4E90823C7E966
:10D510000023D4E90623C6E90023F8BDD4E9022399
:10D52000C7E90023D4E90423F5E7D0B557EC106B25
:10D530000446FFF7F5FE304653EC102B3946F2F760
:10D540009BFE41EC100B2046BDE8D040FFF7E8BE43
:10D55000F8B590F94435032B05460C4636D0D1E991
:10D56000046721A3D3E9002330463946F2F784FE4D
:10D570001FA3D3E9002321F00041F3F7A7FA88BBEA
:10D5800019A3D3E9002330463946F2F777FE18A3F2
:10D59000D3E9002321F00041F3F798FA10BB2146AC
:10D5A0002846FFF719FD284694ED060BFFF7BDFF4F
:10D5B000D4E9060153EC102BF2F75EFEC4E9060134
:10D5C00021462846BDE8F840FFF712BE91ED060B54
:10D5D000FFF7ABFFD4E9060153EC102BF2F74CFE3A
:10D5E000C4E90601F8BD00BF152D4454FB21F93FE5
:10D5F000D8D7FDB2A555D43E38B504460D46FFF741
:10D6000025FB29462046BDE83840FFF7A1BF2DE99C
:10D61000F04114460F460646054698460FCC0FC506
:10D620000FCC0FC50FCC0FC594E80F0085E80F0095
:10D6300031463846FFF7E0FF97F94435032B0BD10D
:10D6400031463846FFF7D4FD384601223146FFF710
:10D650000FFC3046BDE8F081B8F1000FF4D0314640
:10D660003846FFF7B9FCEFE7044B002283F8C424E7
:10D6700083F84025012283F844257047681900206B
:10D680002DE9F04F2DED028B1D461378A1B0412BF3
:10D69000DDE92CA9DDF8B88004460E46174656D1C0
:10D6A0005378572B0CD12B78002B40F02082AE48BA
:10D6B000FEF7A0F8012021B0BDEC028BBDE8F08F91
:10D6C0003F2B11D12B78002B40F0118239220A70A8
:10D6D00090F8162130324A7090F81721CB70303212
:10D6E0008A7089F80030E5E7A3F13102082A13D8DF
:10D6F0002B78002B40F0FB8101219C4802F0B4FE06
:10D700009B480121FDF78AFB7B78303B84F8173179
:10D71000012384F81631CDE72B2B40F0E8812D78DA
:10D72000002D40F0E48190F8173190F816210BB1EC
:10D730009A4203D9082388F80030BBE701F0A6F924
:10D740000028B7D0A4F8165188F80000B2E7432BA0
:10D7500079D15378532B03D12D7825B10020AAE736
:10D760004D2BFBD1F8E794F8173194F816210BB143
:10D770009A422ED97F4894F83151DFF8F081F4F7BE
:10D780000CFBD8E90A2351EC100BF2F775FD0022CF
:10D7900021F000410023F3F7A3F900283DD106252D
:10D7A0000123CDE90E5304F1100CBCE80F006D46C7
:10D7B0000FC5BCE80F000FC5BCE80F000FC59CE803
:10D7C000030085E803002046D4E9022301F016F99E
:10D7D00011E0204601F05AF948B97B784D2B1AD157
:10D7E000212373706449304612F0ABFA13E0A4F8B9
:10D7F000165188F800007B784D2B0CD1A0F1100356
:10D80000DBB200F12104082BE4B218D85B493046A2
:10D8100012F097FA7470002363E75948F4F7BDFAE1
:10D82000D8E90C2351EC100BF2F726FD002221F071
:10D8300000410023F3F754F90028B0D0B0E774702A
:10D840000028E8D1CEE7442B11D15378002B85D1A5
:10D850004C4A1278012A03D17F220A707370DAE7EA
:10D860004B70232201230A708AF80030D3E7472B3C
:10D8700040F0B3815378722B1ED12B784BB16A786C
:10D88000002A7FF46BAF482B14D0612B12D00623F3
:10D8900051E7022530A3D3E90023D4E90201F2F7CE
:10D8A000A3FE2B4641EC100B002237483146F7F718
:10D8B000B3F8B0E70325EDE7642B1DD12B784BB10E
:10D8C0006A78002A7FF44AAF482B01D0652BDED15D
:10D8D000032500E0022522A3D3E90023D4E90601B1
:10D8E000F2F782FE00950123002241EC100B26483E
:10D8F0003146F7F769F98EE7612B16D12B78482B63
:10D900000DD06C2B7FF42AAF6B78002B7FF426AF01
:10D91000022513A3D3E90023D4E90801BFE76B78FC
:10D92000002B7FF41BAF0325F3E77A2B2ED12B7846
:10D93000482B0DD0002BAAD1022509A3D3E900233F
:10D94000D4E90A01F2F750FE009500230122CCE74A
:10D950000325F2E7AFF30080C4ACAEA4C88E0E403E
:10D96000F8C1631ADCA54C4068190020F01F0020A4
:10D97000F8180020A0160020526902084F6902081A
:10D9800048140020B81E002002000020582B7FF40D
:10D99000E5AEA97800297FF4E1AE2B78302B40F07A
:10D9A000A880002389F800306B78303B152B00F2FB
:10D9B0009B80DFE803F00B181A1C1E20222B37393E
:10D9C0009999999999999948607A828AAC4B186883
:10D9D000F2F7B2FDA2A3D3E90023F2F705FEF3F7B5
:10D9E000B3F8024619E0A74BF1E7A74BEFE7A74BC7
:10D9F000EDE7A74BEBE7A74BE9E7A74B93F84425E7
:10DA0000023A012A08D803F2BC43E0E7A24B93F89C
:10DA10004425023A012AF6D80022A049304611F0E6
:10DA200085F847E69E4BD2E790F8163190F817211B
:10DA30003046934298BF0A46984911F077F8994BBF
:10DA400000221A6036E6974B1A68934B2C2101FB93
:10DA50000233D3F8AC01F2F76FFD83A3D3E90023BF
:10DA6000F2F7C2FD022341EC100B01228E48314631
:10DA7000F6F7D2FF1EE68B4B1A68874B2C2101FB71
:10DA80000233D3F8B001F2F757FD79A3D3E90023AD
:10DA9000F2F7AAFD022341EC100B00938248012308
:10DAA00000223146F7F790F804E67E4B1A687A4B6D
:10DAB0002C2101FB0233186ACDE77A4B1A68764BAA
:10DAC0002C2101FB0233586ADDE7764C724B226849
:10DAD0002C2101FB023330469A6A704911F026F876
:10DAE000236801332360E5E5012389F8003003232F
:10DAF00021E6392B7FF432AE6B78323B072B3FF6B1
:10DB00002DAE01A252F823F029DB000839DB000812
:10DB10003FDB000867DB000879DB00088BDB0008CF
:10DB20005DD70008D1DB0008D0F83201F2F704FD20
:10DB300041EC100B5D4947E0D0F81801F6E710A85A
:10DB40005B490122FDF71AFB534B5A4A93F84515DE
:10DB5000594B3046002918BF13469DF87820574985
:10DB600010F0E4FF57E690F83021554902F0010229
:10DB7000304610F0DBFF4EE690F83121514B134454
:10DB800013F8013C3370002368E6D0F83201DFED72
:10DB90004E7A07EE100AC7EE877A17EE900AF2F770
:10DBA000CBFC4A4B04460D46D3E9010132A3D3E92D
:10DBB0000023F2F743FE02460B4620462946F2F7C1
:10DBC0003DFE41EC100B42493046F6F7AFFE22E62F
:10DBD00001F074FB10EE100AA8E74D2B40F05F81B6
:10DBE0005378412B78D12B78002B7FF4B7AD00F11F
:10DBF000080B59462848FFF7FBFA274801225946E7
:10DC0000FFF736F901230F9394F831310E9304F1A5
:10DC100010070FCF6D460FC50FCF0FC50FCF0FC524
:10DC200097E8030085E803009BE80C00204601F01C
:10DC30009FF828490446304612F083F8A4F11003F7
:10DC4000DBB2082B00F2268104F12103337000239C
:10DC500089F8003001238AF8003088F8004029E56F
:10DC600079AD3173C62D0941C4ACAEA4C88E0E4047
:10DC7000F8C1631ADCA54C4000000020DCA54C4034
:10DC80000C1E0020101E0020141E0020181E002054
:10DC90001C1E0020201E002068190020847102082C
:10DCA000281E0020B41E0020020000205669020831
:10DCB000F8180020E27302084C6902085C69020847
:10DCC000766702086969020800247449A0160020DA
:10DCD0006169020811670208442B25D12B78002BBB
:10DCE0007FF43CAD00F1080190F83121012300F0F0
:10DCF000AFFC9D490546304612F023F85DB994F813
:10DD00000031012B04BF3023337094F80031022B13
:10DD100004BF31233370002389F8003001238AF8CF
:10DD2000003088F80050C5E44E2B57D18F4B93F943
:10DD30004435032B3FF4DBAE10AF01228C4938464B
:10DD4000FDF70AFA2A789DF8783022B9012B6A701B
:10DD500008D177232B702B78652B32D16B782BB1C0
:10DD60000320F1E4022B35D16523F3E701230F9360
:10DD700004230E930DF1480CBCE80F006D460FC54F
:10DD8000BCE80F000FC5BCE80F000FC59CE80300FE
:10DD900085E80300204697E80C0000F0E9FF03281F
:10DDA000DED0A0F11003DBB2082B14D908B9302360
:10DDB00033700023737089F8003001238AF8003033
:10DDC000C2E4772BCCD16B78002BC9D101230F9300
:10DDD0000523CEE7182000F12103E9E7502B3DD1C0
:10DDE0002B78002B7FF4BAAC604D95F94435032BAA
:10DDF0003FF47DAE0DF1400B58465D490122FDF721
:10DE0000ABF9204600F0E6FB28B1A0F11003DBB22D
:10DE1000082BE0D9CDE75748594603F0E1F900282F
:10DE2000F3D105F2AC4205F59665002313602B6033
:10DE300001220623CDE90E3212AF0FCF6D460FC57A
:10DE40000FCF0FC50FCF0FC597E8030085E803007C
:10DE500020469BE80C0000F08BFFA2E7532B7FF4D9
:10DE60007DAC2B78002B7FF479AC01230F9390F8D5
:10DE700031310E9300F110070FCF6D460FC50FCF54
:10DE80000FC50FCF0FC597E8030085E80300D4E95D
:10DE90000223CBE6002C7FF4DAAE3023D6E6532BF8
:10DEA0007FF45CAC5378722B13D100F108012A4641
:10DEB0003148F7F72DF908B905233CE4D4E902010C
:10DEC00025A3D3E90023F2F7B9FCC4E90201FFF767
:10DED000F1BB642B13D100F11801012326482A4617
:10DEE000F7F73CFA0028E7D0D4E906011CA3D3E9F0
:10DEF0000023F2F7A3FCC4E90601FFF7DBBB612BAB
:10DF000013D100F1200101231B482A46F7F726FA16
:10DF10000028D1D0D4E9080111A3D3E90023F2F7F6
:10DF20008DFCC4E90801FFF7C5BB7A2B26D100F1AF
:10DF30002801002310482A46F7F710FA0028BBD022
:10DF4000D4E90A0106A3D3E90023F2F777FCC4E978
:10DF50000A01FFF7AFBB00BFC4ACAEA4C88E0E4031
:10DF6000F8C1631ADCA54C406769020868190020F3
:10DF7000F81800205C20002002000020582B7FF4BD
:10DF8000EDABAB782C2B7FF482AC2B78302B40F0B0
:10DF9000A0816B78303B152B3FF6A9AD01A252F85A
:10DFA00023F000BFFDDF00081DE0000839E0000895
:10DFB00055E0000871E000088DE00008A9E00008C5
:10DFC000D9E00008E9E0000805E10008EFDA000800
:10DFD000EFDA0008EFDA0008EFDA0008EFDA0008FD
:10DFE000EFDA0008EFDA000831E1000869E1000823
:10DFF000A5E10008DBE1000815E20008E81C10F0CC
:10E00000D0FCF2F787FAC0A3D3E90023F2F716FC9D
:10E01000F2F7E2FDC24B1860FFF74CBBE81C10F0B2
:10E02000C0FCF2F777FAB8A3D3E90023F2F706FCB5
:10E03000F2F7D2FDBB4BEEE7E81C10F0B2FCF2F7B2
:10E0400069FAB1A3D3E90023F2F7F8FBF2F7C4FDB4
:10E05000B54BE0E7E81C10F0A4FCF2F75BFAAAA3CA
:10E06000D3E90023F2F7EAFBF2F7B6FDAF4BD2E7B4
:10E07000E81C10F096FCF2F74DFAA3A3D3E90023B5
:10E08000F2F7DCFBF2F7A8FDA94BC4E7E81C10F09F
:10E0900088FCF2F73FFA9CA3D3E90023F2F7CEFB0A
:10E0A000F2F79AFDA34BB6E7A34C94F84435023B34
:10E0B000012B3FF6FFAAE81C10F073FCF2F72AFAD6
:10E0C00091A3D3E90023F2F7B9FBF2F785FD04F23F
:10E0D000BC442060FFF7EEBA974C94F84435023BFD
:10E0E000012B7FF6E7AAE6E7E81C10F05AFCF2F7EE
:10E0F00011FA85A3D3E90023F2F7A0FBF2F76CFD38
:10E100008E4B88E7E81C10F04CFC01288C4B7FF408
:10E1100097AC196801297FF793ACCBB284F817311B
:10E120000133854884F81631FDF7B8FBFFF7C2BA12
:10E1300084480223EA1C10A9F6F70AFF00283FF4DE
:10E14000A6AB7F4B7C4C1B682C2202FB0344DDE911
:10E1500010016FA3D3E90023F2F770FBF2F73CFD47
:10E16000C4F8AC01FFF7A6BA022300937548012357
:10E17000EA1C10A9F6F7E8FF00283FF488AB704BC3
:10E180006D4C1B682C2202FB0344DDE9100162A3E5
:10E19000D3E90023F2F752FBF2F71EFDC4F8B001F9
:10E1A000FFF788BA67480223EA1C10A9F6F7D0FEE9
:10E1B00000283FF46CAB624B5F4C1B682C2202FBC7
:10E1C0000344DDE9100152A3D3E90023F2F736FB43
:10E1D000F2F702FD2062FFF76DBA0223009359485F
:10E1E0000123EA1C10A9F6F7AFFF00283FF44FAB5C
:10E1F000534B514C1B682C2202FB0344DDE91001F8
:10E2000045A3D3E90023F2F719FBF2F7E5FC6062BE
:10E21000FFF750BA4A4EE81C3468474D10F0C1FB76
:10E220002C2707FB045495F94435A062346807FB9A
:10E230000454032BC4F8B4013ED1D4F8AC01F2F776
:10E240007BF9CDE91201D4F8B001F2F775F9CDE907
:10E250001401284610A9FEF7BFFEDDE91801346855
:10E26000F2F7BAFC07FB0454C4F88C01DDE916018F
:10E27000F2F7B2FCC4F89401206AF2F75DF9CDE937
:10E280001201606AF2F758F9CDE91401284610A985
:10E29000FEF7A2FE3368DDE9180107FB0355F2F72C
:10E2A0009BFC2860DDE91601F2F796FCA860336854
:10E2B00001333360FFF7FEB9D4F8AC31C4F88C31C8
:10E2C000D4F8B031C4F89431236A2360636AA36040
:10E2D000EDE7392B7FF442AA6B78323B072B3FF6F0
:10E2E0003DAA01A252F823F049E3000823E4000804
:10E2F0005DD700087BE40008A9E400085DD70008AA
:10E30000DFE40008FBE4000879AD3173C62D094154
:10E31000C4ACAEA4C88E0E40F8C1631ADCA54C4054
:10E320000C1E0020101E0020141E0020181E0020AD
:10E330001C1E0020201E002068190020281E00201E
:10E34000B01E002002000020734A037812781343A5
:10E3500064D1E81C10A911F007FB51EC100BF2F787
:10E360003BFC94ED468AC4F83201054618EE100ACB
:10E37000F2F7E2F8064628460F46F2F7DDF8674B5B
:10E3800080468946002230463946F2F72DF902468A
:10E390000B4640464946F2F799FB38B1F6EE007A53
:10E3A00068EE277A17EE903AC4F83231D4F8320189
:10E3B000F2F7C2F83246804689463B463046394637
:10E3C000F1F75CFF02460B4640464946F2F79CFBDC
:10E3D00028B138EE088A18EE103AC4F83231D4F871
:10E3E0003251204600F06AFF07EE905AF4EEC07AF0
:10E3F000F1EE10FA06D5204600F060FF10EE103A5C
:10E40000C4F832314648062304F59872BF21F7F765
:10E4100001FA204600F0E8FEFFF74CB91723FFF79A
:10E420008AB93D4A0023127889F8003003781343F3
:10E43000F4D1EB7890ED468A313B042B06D8DFE827
:10E4400003F01914050F030038EE088A18EE103A8D
:10E450002046C4F8323100F031FFB4EEC08AC7E77D
:10E46000F7EE087A28EE278AF0E7F7EE087A88EECA
:10E47000278AEBE7F6EE007AF4E72A4B93F8453566
:10E48000002B3FF417A9EB78A3F13002012A3FF6E5
:10E4900013AD303B90F8302118BF012363F3000225
:10E4A00084F83021FFF706B9EB78452B05D0572BC0
:10E4B0000FD0422B0FD1032300E0012384F8313128
:10E4C0001748062304F59872BF21F7F7A3F9FFF761
:10E4D000F1B80223F2E7052388F80030F0E7EB7883
:10E4E000A3F13002012A3FF6E7AC303B90F830212F
:10E4F00018BF012363F34102D2E7EB78312B7FF49D
:10E50000DBAC90F81431002B3FF4D4A8012380F841
:10E510001531FFF7CFB800BF5C0100200000E03FDD
:10E52000FC0500206819002008B50548F3F750FDE8
:10E5300020B9BDE808400348F3F74ABD08BD00BF55
:10E54000A01600204814002010B51248124CF3F712
:10E5500024FCD4E90A2351EC100BF1F78DFE0022C4
:10E5600021F000410023F2F7BBFA88B10B48F3F722
:10E5700014FCD4E90C2351EC100BF1F77DFE0022C2
:10E5800021F000410023F2F7ABFA003818BF012058
:10E5900010BD00BFA0160020F01F0020481400206E
:10E5A000006803689B6B18471FB501680B6801A8DA
:10E5B0009B6998479DF80C0005B05DF804FB037853
:10E5C000012B06D190F80831022B84BF022380F87A
:10E5D0000831704770B5184E04463046FFF7E4FF27
:10E5E00010B11624204670BD144D2846FFF7DCFFFD
:10E5F0000028F6D196F84430C3B195F84430ABB159
:10E600000F4B1B78022B13D023789BB90D4B1C7832
:10E610000CB11724E6E7FFF787FF0028F9D10A4875
:10E6200002F0D0FE002818BF1524DBE71224D9E73A
:10E630001324D7E71424D5E7A0160020481400209F
:10E64000802000205C0100205C20002000000000F1
:10E650002DE9F04F9FB004460E4615461F46FFF7C2
:10E66000B9FF122880460AD1FFF76EFF80B1AA4891
:10E670000121FCF7B1FB2046FFF7ACFF8046B8F163
:10E68000000F05D147B1A54B9B7C2BB14FF015086E
:10E6900040461FB0BDE8F08F0FCE04F1C8070FC78A
:10E6A0000FCE0FC70FCE0FC796E80F0087E80F00F9
:10E6B0009B4E96F9443504F1C80A032B5146304667
:10E6C00064D1FEF795FD944900220EA8FCF756FD93
:10E6D0009DF87030914884F800315146059302F05E
:10E6E0007FFD80460028D3D196F8452596F944351C
:10E6F000002A00F0C180032B4BD1D4E93A67DFF840
:10E700001C92D9F8080080F00040F1F715FFCDE920
:10E710000601D9F80C00F1F70FFF3246CDE90801E8
:10E720003B46DDE90601F2F7EFF9002834D078A383
:10E73000D3E9002330463946F1F7A0FDCDE90001C9
:10E74000DDE9080132463B46F2F7C0F938B370A361
:10E75000D3E9002330463946F1F78EFDCDE90201B9
:10E76000704BD3F829B0D3F82590FFF7EDFE6C4B32
:10E7700030B393F94435022B14D194F83131022B84
:10E780001CD184F80031CDE9006764E0FEF724FC79
:10E7900099E7D4E93467B2E7CDE90067D0E7CDE97E
:10E7A0000267DDE70022002330463946F2F78EF992
:10E7B00020B10223E5E7C4E9346779E00123E0E70B
:10E7C0005846F1F7B9FECDE90A014846F1F7B4FE23
:10E7D000534B062DCDE90C0193F9449509D9B9F1B4
:10E7E000030F20D1C4E93A6794F80031022B6ED0B0
:10E7F00042E04FF0010B0BFA05F313F0480F40F025
:10E80000A68013F0240F3BD113F0120F11D1B9F1F0
:10E81000030F94F8003109D1C4E93A67062DE3D11A
:10E82000059A9A4290E0C4E93467DDE7C4E93467A9
:10E83000F4E7DDE9060184F800B132463B46F2F721
:10E8400063F900289FD0DDE90023DDE90A01F2F732
:10E850003DF90028ADD1324A94F8003192F94425AF
:10E86000032A9DED007B40F0BE8084ED3A7B042DB1
:10E8700066D1012B7FF40AAF012384F8003126E032
:10E88000022384F80031DDE9080132463B46F2F705
:10E890001DF9A0B1DDE90223DDE90C01F2F734F93D
:10E8A00058B3B9F1030F84F800B184D1C4E93A67D1
:10E8B000052D3FF4EBAE062DDED10123B0E7B9F113
:10E8C000030F17D1C4E93A67052D40F09280144830
:10E8D00090F94435032B514640F08880FEF788FCC0
:10E8E00051460F48FEF7B8F90D4800225146FEF791
:10E8F000BFFACDE6C4E93467E6E7B9F1030F9DED51
:10E90000027B11D184ED3A7BDEE700BFAFF30080DC
:10E91000182D4454FB211940F81800205C200020D9
:10E9200068190020A016002084ED347BCCE79DED13
:10E93000027B94F80031B9F1030F43D184ED3A7BA7
:10E94000052D7FF46BAF022B3FF44EAF9EE6059B87
:10E95000012B17D1DDE9060132463B46F2F7D4F828
:10E9600048B1DDE90023DDE90A01F2F7AFF820B193
:10E97000022384F80031CDE900679DED007B94F817
:10E980000031D8E7059B022BF5D1DDE908013246BD
:10E990003B46F2F79BF8C0B1DDE90223DDE90C014B
:10E9A000F2F7B2F80028C2D0B9F1030F84F800B131
:10E9B00016D1C4E93A67052D3FF468AE062D3FF441
:10E9C00065AE11E784ED347BBAE7B9F1030F94F833
:10E9D000003102D1C4E93A67B2E7C4E93467AFE76E
:10E9E000C4E93467E7E784ED347B40E7FEF7F4FAE7
:10E9F00076E7062D7FF46BAF022311E782B030B5C6
:10EA000085B008A981E80C009DF86430054633B153
:10EA1000002319488DF858301A46FEF75CFD9DF822
:10EA20006020002308A92846FFF712FE0446E8B933
:10EA3000FFF78AFD18B111480121FCF7EFF902AB8D
:10EA400005F1C8016A460C48FEF79EF99DED000BE2
:10EA50000B48F3F78DF90B489DED020BF3F788F99E
:10EA6000094B064801211974FCF7F8F8204605B057
:10EA7000BDE8304002B0704768190020F818002047
:10EA8000A0160020481400205C200020F0B590F86B
:10EA9000164190F81731A342A1B006464DD3012C80
:10EAA000274F24D010AD27490422284606F1C80478
:10EAB000FCF764FB224801222146FEF729FA97F968
:10EAC0004435032B03D11E482146FEF785FA0095F5
:10EAD00096F8172196F8161119482346FCF7FCFE04
:10EAE00048BB96F81631013386F8163123E0164BF1
:10EAF000D3E90001F2F770F897F9441500EE100A17
:10EB00003846FCF7A3FE0F9496F831310E9306F1C8
:10EB100010050FCD6C460FC40FCD0FC40FCD0FC421
:10EB200095E8030084E803003046D6E90223FFF7A6
:10EB300065FF0028B6D021B0F0BD0520FBE700BF7F
:10EB400068190020F8180020A82000200023A0F851
:10EB500016310148FCF758BE68190020000000007B
:10EB6000DFF858C12DE9F84F0323654680F80831D6
:10EB700000F1880406460F460FCD0FC40FCD0FC419
:10EB80000FCD0FC495E80F0084E80F00DCE9020107
:10EB900000220023F1F790FF20BB97F83830012BBB
:10EBA00022D00FF2E80BDBE900AB0FF2E809D9E95C
:10EBB0000089D7E9064539A3D3E900232046294631
:10EBC000F1F784FFC8B1D6E9140323F000412AA36A
:10EBD000D3E90023F1F798FF78B1C6E9248904232B
:10EBE00086F80831BDE8F88F0FF2B80BDBE900AB0F
:10EBF0000FF2B809D9E90089DBE72EA3D3E9002396
:10EC000020462946F1F762FF0028EBD01E4C18A3DE
:10EC1000D3E90023D4E90E01F1F758FF0028E1D031
:10EC2000D4E900450022002320462946F1F762FF7F
:10EC3000D7E9048922462B4668B10FA1D1E900012A
:10EC4000F1F71AFB42464B46F1F754FF0028C9D0B2
:10EC5000C6E924ABC3E70AA1D1E90001F1F70CFB37
:10EC600042464B46F1F73CFFF0E700BFAFF30080B0
:10EC7000152D4454FB21E93F152D4454FB21F93F48
:10EC8000152D4454FB21F9BFA8200020D221337F49
:10EC90007CD9024065732D3852C100406544E74A73
:10ECA0001857C63F182D4454FB21E93F66732D3891
:10ECB00052C1F03F7744E74A1857D63FF01F002073
:10ECC00030B590F80831053B012B85B004460FD8CC
:10ECD000D0E94823D0E92401F1F7CEFAD4E94A2358
:10ECE000C4E92401D4E92601F1F7C6FAC4E92601F2
:10ECF0001A4802AB6A4604F18801FEF745F894F819
:10ED000008311748062B9DED000B1ED1154B1B78C3
:10ED1000012B1AD1F3F772F89DED020B1248F3F7AD
:10ED20006DF894ED470A0E48F3F7CCFA054628B97A
:10ED300094ED470A0C48F3F7C5FA05460FF0C0FBFF
:10ED4000C4F81001284605B030BDF3F789F89DEDF1
:10ED5000020B0548F3F784F8E3E700BF68190020C9
:10ED6000A016002080200020481400200000000091
:10ED700082B0F0B595B01AA981E80C009DF8AC30CE
:10ED8000044633B1002362488DF8A0301A46FEF7DE
:10ED9000A2FB1AA99DF8A82001232046FFF758FCE2
:10EDA0001428014608D12046FFF709FC084615B093
:10EDB000BDE8F04002B070470028F7D1554B5648E7
:10EDC00001251D74FBF74AFFFFF7BEFB18B152483F
:10EDD0002946FCF723F851484D4F012101F078FAFC
:10EDE00000230022C4E94823C4E94A2397F94435A3
:10EDF000032B22D04A4B1B78012B1ED0494B93F892
:10EE00004130012B19D0D4E9360323F000413AA355
:10EE1000D3E90023F1F75AFE78B139A3D3E90023EF
:10EE2000C4E94823C4E94A2394F80031022B04D1F1
:10EE300035A3D3E90023C4E94A233749032204A8B0
:10EE4000FCF79CF904AE052384F808310FCE4FF08F
:10EE5000010C04F1480584F800C00FC50FCE0FC5A2
:10EE60000FCE0FC596E80F0004F1C80685E80F0025
:10EE70000FCE04F188050FC50FCE0FC50FCE0FC5FD
:10EE800096E80F0085E80F00C4F80CC197F94435E7
:10EE9000032B09D094F8802094F8C0309A4203D014
:10EEA00004A92046FFF75CFE94F80B1111B11E482F
:10EEB000F7F74EFE1D4B02931D4B019300220323D7
:10EEC0000093194801231146F7F7FBFD84F80B0165
:10EED00080B12046FFF7F4FE014600287FF466AFBC
:10EEE000114894F80B1141F28832F7F7FBFC1148F6
:10EEF000F7F7DEF8002159E778DAA10D1C10F93F89
:10EF0000399D52A246DF713F399D52A246DF71BF43
:10EF1000681900205C200020F81800205C01002007
:10EF200080200020F01F0020180C00206D690208CE
:10EF3000DDF10008C8010020F0B590F80831022B7F
:10EF400095B004460BD1012380F808310023A0F8C6
:10EF500014319948F3F77BFC9848F3F778FCFFF7F6
:10EF6000E3FA78BB94F80831042B13D10323944EB1
:10EF700084F8083104F188050FCE0FC50FCE0FC5F8
:10EF80000FCE0FC596E80F0085E80F002046FFF76B
:10EF900097FE17E0013B052B14D8DFE813F0D200F1
:10EFA0001300060013009F00D20094F830319B0735
:10EFB00040F1898094F81531002B40F084800123C2
:10EFC00084F814317C48F2F784FF002840F0E9808F
:10EFD0000FF076FAC4F810017A4D95F86030012BE5
:10EFE0006FD1E868784FF1F7A7FA71A3D3E900234E
:10EFF000F1F724FC754B0022F1F720FC02460B468A
:10F00000D4E93201F1F73AF9C4E932012869F1F79C
:10F0100093FA67A3D3E90023F1F710FC6B4B0022AE
:10F02000F1F70CFC0B460246D4E93601F1F726F95C
:10F0300004F1C805C4E93601002229463846FDF727
:10F0400067FF94F80831053B012B3AD80FF038FAE6
:10F05000D4F81031C01AB0F57A6F32D20FCD04AEA9
:10F060000FC60FCD0FC60FCD0FC695E80F0086E86F
:10F070000F00D4E94823DDE90601F1F7FDF8D4E9F2
:10F080004A23CDE90601DDE90801F1F7F5F897F922
:10F090004435032BCDE9080103D104A93846FDF717
:10F0A0009BFF494802AB6A4604A9FDF76DFE9DED42
:10F0B000000B4148F2F7D4FE9DED020B3F48F2F7FA
:10F0C000CFFE15B0F0BD0023A4F81431052384F859
:10F0D000083104F1880504F1C8064DE73A4BD4E93C
:10F0E000480193F9445500220023F1F7E5FCF0B103
:10F0F000032D22D1D4F80C31DBB1D4F80C3104F15A
:10F10000C806013BC4F80C310FCE04F188050FC5C9
:10F110000FCE0FC50FCE0FC596E80F0085E80F0084
:10F1200000220023C4E94823C4E94A232EE7032D23
:10F13000E0D0062384F80831DFE7062384F808319D
:10F1400040E700251F482570FBF78CFD204894F808
:10F150000B11F7F7E1FB1F4884F80B510378012BE3
:10F1600005D194F80831012B15D102F0C5FD1448E2
:10F1700090F84130012B05D194F80831012B0DD1C5
:10F1800001F066F91448002384F8083115B0BDE891
:10F19000F040F6F78DBF02F0D7FDE8E701F0E8F99F
:10F1A000F0E70648F2F795FE00283FF411AF13E7A9
:10F1B000D485BD587EDBCA40A0160020481400202C
:10F1C000F01F0020F8180020681900200000694096
:10F1D000180C002080200020C80100200148FFF703
:10F1E000ABBE00BFB81E0020F8B52DED048BD0F8E3
:10F1F0003231DFED2F7A2F4D07EE103A87EE878AF6
:10F200000446D5E90101F1F7E7FC07EE900A88EE24
:10F21000279A84ED479A84ED019A19EE100AF1F7C6
:10F220008BF906460F4602460B461DA1D1E90001A7
:10F23000F1F704FB02460B46F1F720F8F1F7CCFC9E
:10F24000324608EE900A3B4617A1D1E90001F1F7DA
:10F25000F5FA0B460246F1F711F8F1F7BDFC89EE1D
:10F26000280A08EE100A2846F2F766FE94ED470ACF
:10F27000284680EE080AF2F78BFE0F4D284694EDE3
:10F28000470A80EE280AF2F757FE284694ED470A0F
:10F2900080EE080ABDEC048BBDE8F840F2F778BEBA
:10F2A000A14187461857B63FE79AD29E46DFA13F55
:10F2B00000247449A01600204814002008B5124804
:10F2C0002DED028BFFF76CF907EE900AF8EEE77A66
:10F2D000B2EE098A0D48C8EE278AFFF761F907EEFA
:10F2E000900AF8EEE77AB7EE007AC8EE276AC7EE22
:10F2F000267AC7EE286ABDEC028B77EEA67A87EEF7
:10F30000270A30EE000A08BDA0160020481400208D
:10F3100038B50446464890F82C302DED028B04F5A4
:10F320009875002B72D1424806232A46BF21F6F772
:10F3300071FA3F4806232A46BF21F6F719FA94F8D6
:10F34000303123F0030384F830313A4BD3E9010123
:10F3500033A3D3E90023F1F771FA374B0022F1F719
:10F3600043F902460B4630A1D1E90001F1F766FAF4
:10F37000F1F732FC08EE100AC4F818012046FFF736
:10F380009DFFB4EEC08AF1EE10FA06D52046FFF7D5
:10F3900095FF30EE000A84ED460AD4F832319FED35
:10F3A000277AD4ED467A06EE903AF4EEC76AF1EE8B
:10F3B00010FAC4BF17EE903AC4F83231D4F83231A3
:10F3C000B6EE007A27EE877A06EE903AB4EEE67A49
:10F3D000F1EE10FAC4BF17EE103AC4F83231D4F887
:10F3E000323177EEA77A07EE103ABDEC028BF4EEDD
:10F3F000C77AF1EE10FA48BF17EE903A204648BFA0
:10F40000C4F83231BDE83840FFF7EEBE0622BF2116
:10F41000F6F796F9002886D18BE700BFAFF300809E
:10F42000F8C1631ADCA54C400000000080842E4126
:10F43000FC050020A01600200000144000247449A0
:10F440000C4B0022C3E944221A70C3F808214FF084
:10F450008642C3F81821084A00200021C3E9480168
:10F46000C3E94A0110689288C3F83001A3F8342137
:10F47000704700BFB81E0020D46302082DE9F04792
:10F480002DED028B82B098460C9B00251D701378E1
:10F49000472BDDE90D7904468A4616461ED153787E
:10F4A000582B57D198F80030392B53D198F80130A8
:10F4B000302B4FD198F80260002E4BD1017B0122F6
:10F4C00000F062FA10EE100AF1F736F841EC100B7A
:10F4D000A7495046F5F72AFA3E703AE04D2B7ED107
:10F4E000537803F0DF02472A3CD10123A14801AA47
:10F4F00008EB0301F5F74EFC90B3BDF90430002B87
:10F5000024DB98F80020772A0CD1227B02212046A8
:10F5100000F012FC89F800007378672B19D10023E2
:10F520003B7016E0652A02D1227B0321EFE76E2AA9
:10F5300005D1227B0221204600F092FCEAE7732AE3
:10F5400002D1227B0321F6E70320E3E7052389F8B4
:10F5500000300125284602B0BDEC028BBDE8F087E3
:10F560000623F4E7772B0CD198F80060002EF1D138
:10F57000427B42F21073022100F0DEFB89F80000AA
:10F58000AAE7652B08D198F80060002EE2D1427BF3
:10F5900042F210730321EFE76E2B0AD198F8006056
:10F5A000002ED7D1827B42F21073022100F058FC6A
:10F5B000E4E7732B08D198F80060002ECAD1827B53
:10F5C00042F210730321F1E7702BC3D198F8006069
:10F5D000002EBFD1684A417B00F0B6FDCEE7512B2B
:10F5E00027D1567836B96548FEF7E9FF204600F086
:10F5F00095F971E7652E01D0772E0BD198F8005060
:10F60000002D40F0B1802A460121204600F01AF971
:10F610003D709EE76E2E01D0732E9BD198F800505E
:10F62000002D40F0A1802A460121204600F040F93B
:10F63000EEE7522B8ED1514B567893ED018ADFEDD8
:10F64000507A412E28EE278A26D101A9404610F093
:10F650008BF9019B434551EC100B3FF460AFF1F780
:10F66000BBFA9FED487A07EE900AF4EE477AF1EE86
:10F6700010FA48BFF0EE477AF4EEC87AF1EE10FACD
:10F68000D8BFB0EE678ADFED407A28EE278A0A23DA
:10F69000637384ED058A42E7452E26D101A94046D1
:10F6A00010F062F9019B434551EC100B3FF437AF6A
:10F6B000F1F792FA9FED337A07EE900AF4EE477A6B
:10F6C000F1EE10FA48BFF0EE477AF4EEC87AF1EEA8
:10F6D00010FAD8BFB0EE678ADFED2B7A28EE278AC2
:10F6E0000A23A37384ED068A19E72848314610F0EF
:10F6F00060FA00283AD098F80030002B7FF42AAF47
:10F700004D2E0DD8422E28D9A6F143030A2B24D81A
:10F71000DFE803F01923231F0D23232323231D00D8
:10F72000532E18D0303EF6B26673A673F7E6022663
:10F730006673A6732246164802F80C6F0323C52190
:10F74000F6F768F8EBE605236373A373E7E6062391
:10F75000FAE70723F8E70823F6E7303EF6B2022E71
:10F760006673A673E6D9DAE60025F3E60546F1E608
:10F770007569020802000020E8930100B81E00200D
:10F78000E12E6542FA9BEE32000070437B6902086D
:10F79000FC05002008B50548F2F71AFC20B9BDE8C1
:10F7A00008400348F2F714BC08BD00BFA0160020B3
:10F7B0004814002030B5044600F10C05134890F8B9
:10F7C0002C3085B023B903232A46C521F6F722F849
:10F7D0002A460E480323C521F5F7CAFF06236373A3
:10F7E000A3730B4B02930B4B019300220323009353
:10F7F000114601230848F7F764F90146064840F628
:10F80000C41205B0BDE83040F7F76CB8FC05002025
:10F810008B690208C5020108180C0020037810B596
:10F82000042B4FF0010208BF0523114608BF0370E7
:10F83000044600F007F8012220461146BDE81040BA
:10F8400000F036B810B40478042C034604D11AB979
:10F850005DF8044BFFF7E2BF187C012821D901298C
:10F8600003D0884201D005281BD1D3ED017AF5EEF3
:10F87000407AF1EE10FA0BD101210B4819741AB13C
:10F880005DF8044BF2F7E3BF5DF8044BF2F7D0BF2D
:10F8900000221A74002205485DF8044B5A60FBF7F9
:10F8A000E1B95DF8044B7047A0160020F81800205D
:10F8B00010B40478042C034604D11AB95DF8044B43
:10F8C000FFF7ACBF587C012821D9012903D0884219
:10F8D00001D005281BD1D3ED027AF5EE407AF1EE86
:10F8E00010FA0BD101210B4859741AB15DF8044B81
:10F8F000F2F7ADBF5DF8044BF2F79ABF00225A74DD
:10F90000002205485DF8044B9A60FBF7ABB95DF83F
:10F91000044B704748140020F818002010B500224E
:10F9200004460121FFF78EFF20460022BDE810406B
:10F930000121FFF7BDBF000008B5114B2DED028B73
:10F940005868B0EE408AF0F7F7FD0BA3D3E9002327
:10F95000F0F74AFE0B4B0022F0F746FEF1F73CF9B8
:10F9600000EE100AB4EEC80AF1EE10FA58BFB0EE7D
:10F97000480ABDEC028B08BD00000020DCA54C400D
:10F98000B81E002000005E4008B50A294AD8DFE80A
:10F9900001F00646090C0F15181B1E303C00B5EE91
:10F9A000000A08BDB7EE000AFBE7B0EE000AF8E770
:10F9B000B1EE000ABDE80840FFF7BEBFB2EE000A94
:10F9C000F8E7B3EE040AF5E79FED1B0AF2E71B4BDD
:10F9D0005868F0F7B1FD16A3D3E90023F0F704FE51
:10F9E000174B0022F0F700FEF1F7F6F800EE100AD0
:10F9F000D7E7124B5868F0F79FFD0DA3D3E900231A
:10FA0000F0F7F2FD0F4B0022ECE7012A02D190ED56
:10FA1000050AC6E7022A05D190ED060AC1E7B6EE4F
:10FA2000000ABEE79FED080ABBE700BFAFF3008006
:10FA300000000020DCA54C4000004042B81E002021
:10FA400000005E4000006E40000000002DE9F04F15
:10FA5000DFF8CC8093B00D4602222F4902A8FBF7B5
:10FA60008DFB98F810409DF840300193DDE9046764
:10FA7000002C4ED0DFF8AC9099F94435032B21D1FE
:10FA8000DDE90AABEB1E012B1FD899F845356BB1A8
:10FA9000019B012B0AD1D8F8080080F00040F0F754
:10FAA0004BFD32463B46F1F72FF848B91B4BD3F8D4
:10FAB0002500F0F741FD52465B46F1F725F830B3DB
:10FAC000002420E0B246BB46DCE7022D1BD199F8AA
:10FAD000453563B1019B022B09D1D8F80C00F0F732
:10FAE0002BFD32463B46F0F7F1FF0028E8D10B4BE7
:10FAF000D3F82900F0F720FD52465B46F0F7E6FF09
:10FB0000B0FA80F46409204613B0BDE8F08F042DEC
:10FB1000DCE70124F7E700BFF8180020A01600205A
:10FB20005C200020681900202DE9F04391B00446C4
:10FB30000222884668463E49FBF720FB3D4A9DF875
:10FB40003830A374147CDDE90C67002C68D0A8F170
:10FB50000302012A31D8022B374D13D1D5F82900E1
:10FB6000F0F7EAFC02460B4630463946F0F7CCFF88
:10FB70008146002856D1B8F1040F32D0204611B08A
:10FB8000BDE8F083D5F82500F0F7D6FC02460B4619
:10FB900030463946F0F79AFF8146002842D1B8F145
:10FBA000040FEBD1D5F82900F0F7C6FC02460B464E
:10FBB00030463946F0F7A8FF1DE0B8F1020FDDD15D
:10FBC000022B1D4B1AD1D3F82500F0F7B5FC0246E5
:10FBD0000B4630463946F0F779FFB0FA80F46409F5
:10FBE000CCE7D5F82500F0F7A7FC02460B463046D7
:10FBF0003946F0F76BFF60B14C46BFE7D3F82900F8
:10FC0000F0F79AFC02460B4630463946F0F77CFF87
:10FC1000E3E705A3D3E90023304627F00041F5E7E9
:10FC20000124ABE70024A9E73FD038C6A6F1F43F92
:10FC3000F81800205C20002048140020F8B5324B52
:10FC400093F8443006460F46154623B92F4B93F8D8
:10FC50004430002B55D02C48FEF7A6FC10B11624DA
:10FC60002046F8BD2948FEF79FFC0028F7D12B1F3E
:10FC7000012B05D9264B1B78022B07D11324EFE764
:10FC8000FFF788FD0028F5D01724E9E7214804781C
:10FC900014B1FEF794FCF7E7012F0AD0042D08D029
:10FCA000022FDDD129463046FFF73EFFD0B915249B
:10FCB000D6E729463046FFF7C9FE0028F7D0737B08
:10FCC000022B03D9022FEDD0042DEAE7124801F0F0
:10FCD00055FB0028EBD10C480321F2F78DFA0028E0
:10FCE000F0D0E4E7B37B022BBAD80B4801F046FB17
:10FCF0000028DCD105480321F2F77EFA0028AFD0B6
:10FD0000D5E71224ACE700BFA0160020481400205D
:10FD100080200020B81E00205C20002003299FEDD9
:10FD2000040A04480CBF02210121F2F7FEBA00BF09
:10FD30000000C07FA0160020F8B504462DED028B10
:10FD400017461E460D46A9B30378043B012B31D953
:10FD50000A460121FFF772FF68BB0122394620469F
:10FD60002574FFF711FE002E08BF6FF06046B0EE5D
:10FD7000408A0EF0A5FBF0EE007AB4EEE78A30443C
:10FD8000F1EE10FA60622BD81C491D48F1F75AFEBB
:10FD90001A491C48F1F756FE0A2F0FD0032D4FF0D9
:10FDA000010308BFB1EE488A1748237084ED018A29
:10FDB000FAF758FF0020BDEC028BF8BD0223237038
:10FDC000DFED127A0E4888EE270ADFED117A80EE19
:10FDD000270AF2F70DF929462046FFF79FFFE9E7CA
:10FDE00002230A2F2370EBD0074BD3ED017A032DAA
:10FDF0000CBF38EE678A38EE278AE1E7E09304000B
:10FE0000A016002048140020F818002000007043BD
:10FE1000E12E654210B590B00C4600220C496846B0
:10FE2000FBF7ACF99DF83830022B0AD1032C0AD12C
:10FE30009FED080A0121084810B0BDE81040F2F714
:10FE400074BA032CF4D19FED030A0221F3E700BF3B
:10FE5000F81800200000C07F4814002000000000B7
:10FE6000F8B504462DED028B17461E460D460029B7
:10FE700050D00378043B012B4CD90A460221FFF7EE
:10FE8000DDFE002847D10222394620466574FFF77F
:10FE90007BFD354B5868F0EE408AF0F74DFB30A300
:10FEA000D3E90023F0F7A0FB304B0022F0F79CFBD6
:10FEB000F0F792FE08EE100AF4EEC88AF1EE10FA9E
:10FEC000D8BFB0EE688A002E08BF6FF060460EF013
:10FED000F7FAF0EE007AB4EEE78A3044F1EE10FA69
:10FEE000A0622FD822492348F1F7ACFD20492248CF
:10FEF000F1F7A8FD0A2F13D001232370A37C022B56
:10FF00000CD1022D08BFB1EE488A1C4884ED028A4C
:10FF1000FAF7A8FE0020BDEC028BF8BD032DF1E737
:10FF200002232370DFED167A134888EE270ADFEDEF
:10FF3000157A80EE270AF2F75BF829462046FFF78C
:10FF400069FFE7E702230A2F2370EBD00B4BD3EDB9
:10FF5000027A032D0CBF38EE678A38EE278AE1E774
:10FF600000000020DCA54C40B81E002000006E40C0
:10FF7000E0930400A016002048140020F818002088
:10FF800000007043E12E6542F8B504462DED048B68
:10FF90000EF096FA236AC01AF0F7BCFA624B002200
:10FFA000F0F74CFCF0F718FE0122E17B05462046F5
:10FFB000FFF7EAFC5D4B5868B0EE408AF0F7BCFAF8
:10FFC00053A3D3E90023F0F70FFB594B0022F0F7BE
:10FFD0000BFBF0F701FE08EE900A18EE100AF0F79E
:10FFE000ABFA064618EE900A0F46F0F7A5FA514B09
:10FFF0000022F0F7F9FA02460B4630463946F0F790
:020000040801F1
:1000000083FD18B1B6EE008A28EE888AB4EE688ABD
:10001000F1EE10FA2846C8BFB0EE688AF0F78CFA05
:100020003DA3D3E90023F0F709FC9FED3D1B41EC14
:10003000100B12F0D1F957EC106B13F0D1F83046D9
:1000400053EC102B3946F0F717F933A3D3E900230B
:10005000F0F7CAFAF0F7C0FD09EE100AB0EE490A4F
:1000600012F032FAF0EE409AB0EE490A12F000FCBB
:10007000314B93ED017AD3ED027AA8EE297A40F262
:1000800002232382E8EE007A2046B5EEC07AF1EE34
:1000900010FA48BF032384ED057AF5EEC07A42BF1B
:1000A000B0EEC77A237484ED057AF1EE10FAC4ED50
:1000B000067A41BF0323F0EEE77AC4ED067A637453
:1000C000217C9FED1E8AFFF729FE617C2046FFF709
:1000D000A1FE94ED057AD4ED077A194887EE270A38
:1000E000B4EE680AF1EE10FAC8BFB0EE680A84ED0B
:1000F000050A80EE080AF1F77BFF124894ED060A24
:1001000080EE080ABDEC048BBDE8F840F1F770BF43
:1001100000000020DCA54C406E861BF0F921194040
:10012000BC4026C50B64E23F00408F40B81E002053
:1001300000006E400000E03FF8180020F3DB564658
:10014000A016002048140020F0B50378032B91B0CE
:1001500004460E46174605D1FFF7E0FB002528466A
:1001600011B0F0BD018A51BB0422FFF767FD0546BF
:100170000028F4D1082E28BF0826032E38BF0326F6
:10018000E673002F08BF6FF060470EF099F9206208
:1001900038442A460B49C4E909006846FAF7EEFFDD
:1001A0009DED0C0B12F0A0FB51EC100BF0F714FDC1
:1001B000E0612046FFF7E8FE03232370CEE7172512
:1001C000CDE700BFF818002038B503780446002BAF
:1001D0003BD0037C012B39D1D0ED017AF5EE407A8A
:1001E000F1EE10FA07D13248F1F7F2FE70BB20743D
:1001F0003048FAF737FD637C012B36D0637C012B46
:1002000044D82378032B08D1227C637C012A49D966
:10021000012B49D92046FFF7B7FE2378043B012B79
:1002200010D8FFF7B7FA054660B920822248F5F7E3
:100230003FFF2378042B05D12048257090F840100B
:1002400000F012F9238A03B9237038BD237C012BF7
:10025000D1D90EF035F9636AC01A0028CBDB002231
:1002600001212046FFF7EEFAC5E7D4ED027AF5EE5C
:10027000407AF1EE10FAC4D11148F1F7A9FE002836
:10028000BCD160740B48FAF7EDFCBAE70EF018F930
:10029000A36AC01A0028B4DB002201212046FFF720
:1002A00007FBAEE7012BCDD92046FFF737FBB4E7BC
:1002B000A0160020F8180020C8010020F01F002020
:1002C000481400200148FFF77FBF00BF5C010020F9
:1002D0007047000038B51178069D68291DD1527805
:1002E000432A09D11B78C3B900F068F82870059B30
:1002F00000221A70012038BD462A0ED11C7864B93C
:10030000012100F0B1F8064A28700F2302F8014BD2
:100310000448D821F5F77EFAE9E70020EBE700BFB3
:1003200080200020FC0500202DE9F041204B93F9AE
:1003300044150129044625D11BA3D3E90023C0E9B4
:100340000223DFF8748018A3D3E90023D8E9100151
:10035000F0F74AF9174B1D6893F90C702A68C4E945
:1003600004015668D8E9100100220023F0F7AEFB23
:10037000B8B102370CBF4FF0FF316FF001012846D2
:10038000B04709E0002200230329C0E90223C0E9A5
:100390000823D6D1C0E90623002384F83830BDE80D
:1003A000F0813946EBE700BF152D4454FB21F93F9E
:1003B00068190020A0160020A820002070B5204B4E
:1003C0001B7890B0064633B91E48017831B1042934
:1003D00001D1FFF7A3FA172010B070BD1A4C94F8A2
:1003E0006030581E4342434186F842302046FAF7B7
:1003F00015FD20460121FAF7EFFC0123134886F88A
:10040000413090F94435032B02D13146FCF7F0FE20
:1004100004230022CDE90E3206F108050FCD6C460B
:100420000FC40FCD0FC40FCD0FC495E8030084E8AF
:100430000300034896E80C00FEF79AFCCCE700BFE7
:10044000B81E00205C010020F81800206819002068
:10045000002390F8421080F841300148FAF7DEBCE2
:10046000F818002000000000F8B5394B1B7804464E
:100470000F463BB9374B1E783EB1042E02D11846C9
:10048000FFF74CFA17263046F8BD334DFFF74CFF07
:1004900031462846FAF7C2FC4FF07E5342F2107103
:1004A0002E482B600023EB602B61F6F7C1FB9FED1C
:1004B000260B2B48F1F718FB9FED230B2948F1F78A
:1004C00013FB294B93F94435032B35D194ED080BDD
:1004D0002348F1F74DFC94ED060B2248F1F748FC58
:1004E0001F48F1F75AFC1F4884ED0A0BF1F755FC41
:1004F00084ED0C0BD5F81530194800EE103AF1F7E1
:10050000BBFAD5F81930174800EE103AF1F7B4FAF3
:100510009FED160A1248F1F76BFD9FED140A114882
:10052000F1F766FD002FAED00B480021FAF754FC1E
:100530000748FEF70BFBA6E794ED020B0848F1F71E
:1005400017FC94ED040BC8E7000000000000000059
:10055000B81E00205C010020F8180020180C0020B4
:10056000A0160020481400206819002088C3E43A2F
:10057000002180F84110FFF777BF0000034B0022F5
:1005800083F8402083F84220704700BFF01F00200E
:100590002DE9F0432DED048B99B01C46249B4FF0C0
:1005A000000983F8009013784C2BDDE92575064689
:1005B000884640F055815378422B07D12478002C8F
:1005C00040F04C8100F033FA3C7012E0432B19D11B
:1005D000A948012308AA2146F4F7DCFB78B1BDF94C
:1005E00020100029C0F23881304600F08CFA87F8DC
:1005F0000090012019B0BDEC048BBDE8F083062308
:100600002B70F6E7492B2FD12678CEB1472E40F03C
:1006100025816678002E40F021810CAB009303AA5F
:1006200008AB08AC00F048F90FCC944D0FC50FCCC7
:100630000FC50FCC0FC594E80F0085E80F0011E03F
:100640000CAB009303AA08AB00F036F98C4B039A6D
:100650008C4953F8224040460FF09CFA2146404610
:100660000FF098FA3E70C4E7522B5DD194F80090D9
:10067000B9F1000F40F0F2800CAB009302AA08AB76
:1006800008AC00F019F90FCC7C4D0FC50FCC0FC58D
:100690000FCC0FC594E80F0085E80F00784B029A45
:1006A000784953F8224040460FF074FA21464046FC
:1006B0000FF070FA74494046EFF77AFD78B36AA3F9
:1006C000D3E90023DDE90801EFF78EFF022341ECB7
:1006D000100B4A46684803A9F4F79EF96949404659
:1006E0000FF058FA03A940460FF054FA60A3D3E97B
:1006F0000023DDE90C01EFF777FF022341EC100B3B
:1007000000935D4801234A4603A9F4F75DFA5D4969
:1007100040460FF03FFA03A940460FF03BFA30463F
:1007200000F0A5F900235FE0572B4DD108AB4846F8
:100730001F464A46215C03F8012B2C2905D00130C5
:100740000C2803F8011C1A70F4D1225C2C2A04EB4B
:10075000000335D10022944613F8010F18A901FABD
:1007600082F15C7801F853CC01F8540C0132002C72
:10077000F2D1DFF80C91A04659F8041B03A8EFF75B
:1007800017FD08B90FFA88F408F10108B8F1100F45
:10079000F2D13E4B304693ED028B93ED069B00F079
:1007A00023F978B1B0EE491AF0EE691AB0EE480AB2
:1007B000F0EE680A22463946304600F009FA18E79A
:1007C0000024E6E70F231BE74E2B05D12478002CED
:1007D00044D100F04CF9F7E6242B07D12378002B05
:1007E0003CD100F0D9F801233B7002E7442B04D13F
:1007F00023789BBB00F0C0FA94E74C2B04D12478FB
:1008000064BB00F0CFFADFE6212B04D124782CBBA7
:1008100000F0E2FAD8E63F2B09D12478F4B900F0D1
:10082000B0F91B49024640460EF080F9CCE66F2B2A
:1008300014D11148012308AA2146F4F7ABFA002885
:100840003FF4DDAEBDF82030BDF920100E2B03D8EB
:10085000304600F051F9CCE60523D1E60323CFE67C
:100860004846C7E6AFF30080C4ACAEA4C88E0E40C5
:10087000F8C1631ADCA54C4002000020C01E002015
:10088000880100204264020893690208B81E002013
:100890008471020810B5C96901EB021104460246D1
:1008A0001023034889B2F4F763FF204610BD00BF50
:1008B000FC050020000000002DE9FF4104460D4624
:1008C0009046014602680A9E68461F46FFF7E2FF0F
:1008D0009DF80B301A090F2A02D0A1698A420CD068
:1008E0000023002000212B70C8F80030C7E9000168
:1008F000C6E9000104B0BDE8F0816C4603CCA278E3
:100900006960AA7221882860002203F00F03EA724E
:100910002981BDF80C00C8F80030EFF7EBFD1A4B49
:10092000BDF80E400022EFF75FFE184B0022EFF7F4
:100930005BFEC7E900012046EFF7DCFD124B002209
:10094000EFF752FE124B0022EFF74EFE114B002242
:10095000EFF792FCC6E90001D7E9000108A3D3E94B
:100960000023EFF76BFFC7E9000105A3D3E90023DC
:10097000D6E90001EFF762FFBAE700BFAFF30080EE
:10098000F8C1631ADCA54C400000F03E00807640C0
:1009900000806640008056401FB54FF0FF3304468C
:1009A00003602268636801329A42226011DA2146AC
:1009B0006846FFF76FFF9DF800309DF80B20242B51
:1009C00003D1A369B3EB121F03D0D4E900239A42E9
:1009D000E7DBD4E900239A42A5BF03F1FF330020EF
:1009E0000120236004B010BD1FB54FF0FF33044653
:1009F00003602268636801329A4222600CDA214661
:100A00006846FFF747FF9DF80B301B090F2B03D0FB
:100A1000D4E900239A42ECDBD4E900239A42A5BF33
:100A200003F1FF3300200120236004B010BD1FB587
:100A300004462268013A002A226010DB21466846FB
:100A4000FFF728FF9DF800309DF80B10242B23683A
:100A500003D0A269B2EB111F05D0002BE9DA002008
:100A6000206004B010BD002BF9DB0120F9E71FB5B1
:100A700004462268636801329A42226011DA2146F4
:100A80006846FFF707FF9DF800309DF80B20242BE8
:100A900003D0A369B3EB121F03D0D4E900239A4219
:100AA000E7DBD4E900239A42A5BF03F1FF3300201E
:100AB0000120236004B010BD1FB500230360818BAB
:100AC00010236A4604460B48F4F752FE9DF80020B6
:100AD0009DF80B30242A4FEA131302D0A2699342E7
:100AE00005D0204604B0BDE81040FFF7C0BF01208C
:100AF00004B010BDFC0500200E2902D88161FFF76B
:100B0000DBBF00207047F0B5002485B005460E46D7
:100B1000274623466A68A24205DCB74218D12B60FB
:100B2000012005B0F0BD224629466846FFF7B2FE17
:100B30009DF800309DF80B20242B04D0AB69B3EB5B
:100B4000121F08BF0137B7422346E8D00134E1E75E
:100B50000020E6E77FB50024054626466B68A342E1
:100B600002DC304604B070BD224629466846FFF7D5
:100B700091FE9DF80B301B090F2B18BF0136013475
:100B8000ECE710B54468FFF7E5FF201A10BD000040
:100B900082B0F8B5002906AC84E80C0012DB43688B
:100BA0008B420FDDC569094F264605EB0115002470
:100BB000291916F8012B89B238460134F4F72CFDB7
:100BC000102CF5D1BDE8F84002B07047FC050020BC
:100BD0002DE9F04F87B00C46064602AF0868496819
:100BE0003B4603C32089A17A18809970B36942EA11
:100BF000031251EC100B8DF8132054A3D3E90023FA
:100C000059EC118BEFF7F0FC50A3D3E90023044615
:100C10000D4640464946EFF7E7FCDFF81C91824657
:100C20008B464FF0000842464B4620462946EFF7D8
:100C300061FF002861D1DFF800914FF00008002229
:100C4000002320462946EFF741FF00285ED13A4BAA
:100C5000002220462946EFF7F1FD384B80468946B1
:100C6000002250465946EFF74FFF002857D1344B2A
:100C7000002250465946EFF729FF002854D12F4B48
:100C8000002250465946EFF7F9FA2E4B04460D461E
:100C9000002240464946EFF7A7FC41EC100B12F04A
:100CA0004FFA294B00222046294659EC108BEFF7CA
:100CB000C5FD244B0022EFF797FC41EC100B12F01E
:100CC0003FFA4946404655EC104BEFF765FF294681
:100CD000ADF814002046EFF75FFF06ABADF8160045
:100CE00013E903008DE80300304697E80C003168F3
:100CF000FFF74EFF07B0BDE8F08F20462946424679
:100D00004B46EFF7B9FA04460D468CE720462946D4
:100D100042464B46EFF7B2FA04460D468FE7DFF83E
:100D20001CB04FF0000AAAE7DFF814B04FF0000A39
:100D3000A5E700BFAFF300800080764000805640FA
:100D4000008056C00000F04000806640F8C1631A81
:100D5000DCA54C400B1E0BDB42689A4208DDC169E2
:100D6000044801EB03110B31F02289B2F4F754BCB3
:100D7000704700BFFC0500201FB50446026801460D
:100D80006846FFF787FD9DF80B20A369B3EB121FA0
:100D900006D12168204604B0BDE81040FFF7DABF55
:100DA00004B010BD30B5044685B000256368AB4281
:100DB00001DC05B030BD2A4621466846FFF76AFDD2
:100DC0009DF80B20A369B3EB121F03D129462046DF
:100DD000FFF7C0FF0135E9E738B5054600246B6829
:100DE000A34200DC38BD21462846FFF7B3FF01349B
:100DF000F5E70000002340F2423110B5C0E90631AA
:100E000004460E488288531EA2F2423222EAE2725F
:100E100023621311636083B190F82C303BB92046F4
:100E2000FFF7DAFF2046BDE81040FFF745BE12B2DB
:100E3000F4F786FC0028F2D1F4E710BDFC05002091
:100E40002DE9F3411D46089B0E46002119701378C9
:100E5000472BDDE90987044640F084805378682BEE
:100E600016D12D78002D40D10368DFED937A00EE86
:100E7000103A27EE800A12F01DFB904902463046D8
:100E80000DF054FE88F80050012002B0BDE8F0815A
:100E90006F2B0DD12D7845BB4368DFED877A00EECF
:100EA000103A27EE800A12F005FB85490246E6E774
:100EB000582B1AD12B78452B17D1AB78ABB988F8C2
:100EC00000306B78442B0CD8382B0ED9393B0B2BC8
:100ED0000BD8DFE803F00C0A0A0A0A0A0A0A2434CB
:100EE0004345652B1DD0772B25D00020CDE78068AA
:100EF000EFF722FB6EA3D3E90023EFF775FB714BED
:100F00000022EFF771FBEFF767FE00EE100A12F018
:100F1000D1FA6D49024630460DF008FEB4E7C068CC
:100F2000E6E76A4BD3F82530DFED637A00EE103A3E
:100F300027EE800AEBE7654BD3F82930F4E7634BE3
:100F4000D3F82900EFF7F8FA59A3D3E90023EFF714
:100F50004BFB5F4B0022EFF771FCD4E75D4BE1E701
:100F60005C4BE9E7532BC0D15378682B21D15A4809
:100F700001230DF106022946F3F70CFF002845D0A6
:100F8000BDF9060000F11E039BB23C2B00F28B80E2
:100F9000EFF7C0FA46A3D3E90023EFF74FFCEFF7D2
:100FA0001BFE20604D4810232246C821F4F732FC76
:100FB0006AE76F2B2DD1484801230DF1060229461F
:100FC000F3F7E8FE10B3BDF90600A0F13C039BB2B5
:100FD0001E2B68D8EFF79EFA35A3D3E90023EFF76D
:100FE0002DFCEFF7F9FD3E4B606093F94435032B80
:100FF00007EE100AD6D1DFED3B7AB4EEE77AF1EED8
:1010000010FACFDD17EE903A6360CBE706233B7012
:101010003AE7582B7FF469AF2B78452B7FF465AF07
:10102000AB782C2B7FF461AFE81C0DF0BAFCEFF726
:1010300071FA2D4B0022EFF7D7FAEFF7CDFD6B7861
:10104000392B07EE900A18D0412B7FF44EAF9FED5D
:10105000277AF4EEC77AF1EE10FA24DB9FED247ABA
:10106000F4EEC77AF1EE10FA1DD89FED137AC7EEB1
:10107000877A17EE903AE36094E79FED1C7AF4EEDE
:10108000C77AF1EE10FA0EDB9FED197AF4EEC77A0B
:10109000F1EE10FA07D89FED087AC7EE877A17EEBF
:1010A000903AA3607EE70523B1E700BFAFF300806D
:1010B00000000020DCA54C40E12E6542CC6902080E
:1010C000D46902080000104084710208A0160020B4
:1010D00000002E404814002002000020FC050020E3
:1010E000681900200000AE420000D03F0000B4C3E9
:1010F0000000B44300000000D0B504468068EFF75C
:101100001BFA17A3D3E9002306460F46EFF7FCFCB2
:1011100078B1174BA360E068EFF70EFA10A3D3E99C
:10112000002306460F46EFF7EFFC68B1104BE36073
:10113000D0BD0DA3D3E9002330463946EFF7C6FCF6
:101140000028E8D00B4BE5E707A3D3E9002330469E
:101150003946EFF7BBFC0028EAD0064BE7E700BFB3
:10116000182D4454FB211940182D4454FB2119C05B
:10117000DB0FC940DB0FC9C01FB50446134890F808
:101180002C30E3B9114810232246C821F4F742FB62
:1011900022461023C8210D48F4F7EAFA2046FFF74B
:1011A000ABFF0B4B02930B4B0193022300930022E6
:1011B000012364210848F5F784FC04B010BD102217
:1011C000C821F4F7BDFA0028DCD1E1E7FC050020D6
:1011D000DB690208ED190108180C0020000000006E
:1011E0002DE9F843D1E90667054600680C46EFF79C
:1011F000A3F932463B46EFF73FF855A3D3E9002366
:10120000EFF782FC002840F09F806868EFF794F9C0
:1012100002460B4630463946EFF72EF84CA3D3E989
:101220000023EFF771FC002840F09080504DD5F876
:101230002500EFF781F94F4B93F94435032B804696
:10124000894621D1D4E9086732463B46EFF714F8C6
:101250003FA3D3E90023EFF757FC10B11520BDE8F9
:10126000F883D5F82900EFF767F902460B463046B8
:101270003946EFF701F836A3D3E90023EFF744FC32
:101280000028EBD10020EAE7D4E9026732A3D3E9D2
:10129000002330463946EFF737FC002843D030A30F
:1012A000D3E9002330463946EEF7E6FFC4E90201F0
:1012B000D4E90267404632463B464946EEF7DCFF3A
:1012C00023A3D3E90023EFF71FFC0028C6D1D5F8EC
:1012D0002900EFF731F902460B4630463946EEF762
:1012E000CBFF1BA3D3E90023EFF70EFC0028B5D1F9
:1012F000D4E90445204ED6F82500EFF71DF9224623
:101300002B46EEF7B9FF12A3D3E90023EFF7FCFB5E
:101310000028A3D1D6F82900EFF70EF902460B46B4
:1013200020462946A5E710A3D3E9002330463946D5
:10133000EFF7CCFB0028BBD009A3D3E9002330464C
:101340003946EEF79BFFB1E7102088E7112086E7CA
:10135000000000A0F7C6A03E182D4454FB21094010
:10136000182D4454FB211940182D4454FB2109C069
:10137000A01600206819002048140020104B1B788C
:1013800013F0130F1AD1437CC3B9837CB3B9C37C68
:10139000A3B9037D93B9437D83B9837D73B9C37DBD
:1013A00063B9037E53B9437E43B9837E33B9C37EA9
:1013B00023B9007F003818BF012070470120704713
:1013C000A11100200D4A12789207034611D10C4951
:1013D00091F854206AB191F8550060B1DA7D5AB99C
:1013E0001A7E4AB95A7E3AB9987E003818BF012051
:1013F0007047012070471046704700BFA1110020C0
:10140000A820002010B504462648FDF7CDF808B105
:10141000012010BD2448FDF7C7F80028F8D1E37D6E
:10142000002B2ED1237E63BB637E53BBA37E43BBC5
:10143000637C53BBA37C63B91C4AE37C92F94425CB
:10144000032A08D1FBB9237DEBB9637DEBB9A37DFA
:1014500043B10C20DDE7D3B9237DC3B9637DC3B9A4
:10146000A37DB3B9E37EB3B9237FA3B9104B18783A
:10147000820712D1C30612D410F0080018BF0D2045
:10148000C7E70320C5E70520C3E70220C1E7062020
:10149000BFE70420BDE70720BBE70F20B9E70E2018
:1014A000B7E700BFA01600204814002068190020EC
:1014B000A111002010B50A480A4CFDF780F801225E
:1014C00011462046FEF7BEF9012220461146FEF7DE
:1014D000EFF9BDE8104004480021F9F79FBC00BFB8
:1014E000B81E00205C010020F818002010B50B4841
:1014F0000C46FDF764F80A4801222146FEF7A2F9DE
:10150000022C04D0074B93F94435032B05D1BDE8D9
:10151000104005480021F9F781BC10BDB81E00201D
:101520005C01002068190020F818002010B50A4856
:101530000C46FDF744F8094801222146FEF7B8F9A8
:10154000074B93F94435032B05D1BDE810400548FE
:101550000021F9F763BC10BDB81E00205C0100201B
:1015600068190020F81800202DE9F04FB64AB74955
:101570001368002BBFB0C4BF03F1FF331360437C7B
:101580001293837C1B93C37C1993037D1893437D33
:101590001793837D1693C37D1593037E1493437E27
:1015A0001A93837E1C93C37E13930446037F1D937B
:1015B00002221EA8F9F7E2FD9DED287B237C9DF811
:1015C000B050DDE92067DDE924898DED107BDDE990
:1015D0002AAB002B00F0E2812068EEF7ADFF424617
:1015E0004B46EFF791FA003818BF0120607460682D
:1015F000EEF7A2FF4B464246EFF768FA0038944BED
:1016000018BF0120A07493F84535002B00F06881C5
:10161000012D00F052810023022DE37640F05C8121
:10162000E068EEF789FF32463B46EFF74FFA0028B5
:1016300000F05281844BD3F80090B9F1000F40F0D4
:101640004B81DFF8148298F83021D10740F14A81AC
:101650007E4991F86060012E40F044810A222EAF4D
:101660001A6038463246F9F789FD0423CDF83C90DC
:101670000E930DF1C00EBEE80F00EC46ACE80F0073
:10168000BEE80F00ACE80F00BEE80F00ACE80F00AA
:101690009EE803008CE80300404697E80C00FDF745
:1016A00067FB20B129462046FFF720FF2677694EC9
:1016B000D6F82500EEF740FFDDE91023EEF7DCFD5C
:1016C0005FA3D3E90023EFF71FFA20B120460321DF
:1016D000FFF70CFF0120E074D6F82900EEF72CFF8D
:1016E00002460B46DDE91001EEF7C6FD54A3D3E92F
:1016F0000023EFF709FAE0B1534BD3F80080B8F1BB
:10170000000F40F04581524A92F8452562B1012D03
:101710000AD1514F97F83021D20705D54B4991F89E
:101720006020012A00F0E58020460221FFF7DEFE5E
:1017300001204A4B2075D3F82500EEF7FDFE5246F6
:101740005B46EEF799FD3EA3D3E90023EFF7DCF902
:1017500038B1012D40F01E8103212046FFF7E6FE3F
:1017600001203E4B6075D3F82900EEF7E5FE0246F6
:101770000B4650465946EEF77FFD31A3D3E90023CF
:10178000EFF7C2F9002800F00181012D40F004813B
:1017900002212046FFF7CAFE0123A3752D4E022128
:1017A0003046F1F76AF8E07548B196F82D3013B17C
:1017B000159B012B03D003212046FFF797FE2548F8
:1017C0000121F1F75AF8207648B196F82D3013B17F
:1017D000149B012B03D002212046FFF787FE1F4EEA
:1017E00002213046F1F749F8607660B196F82D3065
:1017F00013B11A9B012B06D0012D0CBF032102212E
:101800002046FFF793FE15480121F1F736F8A07640
:1018100060B196F82D3013B11C9B012B06D0012D21
:1018200014BF032102212046FFF780FE084B93F9E5
:101830004415032940F0BB8012E000BFAFF30080E5
:10184000000000A0F7C6A03E7C200020F818002071
:1018500068190020A0160020B81E0020481400209F
:10186000637C13B12046FFF761FEA37C1BB102210C
:101870002046FFF75BFE139B0BB9E37EBBB91D9BB4
:101880000BB9237F9BB9199B0BB9E37C7BB9189BE0
:101890000BB9237D5BB9179B0BB9637D3BB9169BD5
:1018A000002B40F09780A37D002B00F09380204612
:1018B0003FB0BDE8F04FFFF7FDBDA06880F00040ED
:1018C000EEF73AFE32463B46EFF71EF930B1032100
:1018D0002046FFF70BFEE576002308E0E076FBE705
:1018E000E376F9E702212046FFF700FE0123237784
:1018F000DDE60A222EAE1A6030462A46F9F73EFC93
:101900000523CDF83C800E930DF1C00EBEE80F000C
:10191000EC46ACE80F00BEE80F00ACE80F00BEE8F4
:101920000F00ACE80F009EE803008CE80300384687
:1019300096E80C00FDF71CFA20B102212046FFF7C3
:10194000D5FD2575284ED6F82500EEF7F5FD524653
:101950005B46EEF791FC22A3D3E90023EFF7D4F81E
:1019600000287FF4F9AE6075D6F82900EEF7E4FDA3
:1019700002460B4650465946EEF77EFC18A3D3E9C3
:101980000023EFF7C1F800287FF402AF002304E73B
:101990000020CEE60221E0E60321FAE66374A37498
:1019A000E37423756375A375E3762377F6E6129BDC
:1019B00023B9637C13B12046FFF77CFD1B9B002BF2
:1019C0007FF459AFA37C002B3FF455AF2046FFF7BF
:1019D00071FD50E73FB0BDE8F08F00BFAFF300806E
:1019E000000000A0F7C6A03E481400200148FFF701
:1019F000BBBD00BF5C20002010B5074B074A03F1B8
:101A00001000114653F8044B42F8044B8342F9D1BD
:101A100000230B7410BD00BFDA6302085C200020B5
:101A200008B5117868291BD15278502A09D11B7842
:101A3000B3B900F0B3F800B90120049B187001207D
:101A400008BD512A04D11B7853B900F019F8F4E706
:101A5000522A05D11B781BB9012100F097F9EAE75A
:101A60000020EDE708B50448FCF79EFD10B90348D7
:101A7000FCF79AFD08BD00BFA01600204814002006
:101A80002DE9F0430378032B91B0044650D0022B8C
:101A900050D02B4B1D782B4B1B781D434CD1FFF79F
:101AA000E1FF00284AD1284F97F86060731E5E421C
:101AB000294638465E41F9F7B1F9012239466846B0
:101AC000F9F74AFBDDE902892378E372494640468B
:101AD000EFF782F8C4F80100DDE90401EFF77CF8C4
:101AE0009DF83830C4F80500637263B9174B93F85A
:101AF0004535DBB10022002340464946EEF7E6FFBC
:101B0000A0B1022363720123D8211148A372621C81
:101B10000F23F3F77FFE0D48F9F76CFE0A483146B4
:101B2000F9F77CF9284611B0BDE8F0830123E9E715
:101B30000B25F7E70A25F5E71725F3E71625F1E763
:101B4000B81E00205C010020F81800206819002051
:101B5000FC05002038B504460F4890F82C30651C71
:101B60009BB90D480F232A46D821F3F753FEE37A99
:101B700023702046FFF784FF0F2307482A46D82109
:101B8000F3F7F6FDE37A237038BD0F22D821F3F77F
:101B9000D7FD0028E5D1EFE7FC0500202DE9F04155
:101BA000837AA0B00646002B00F08C800378022BCD
:101BB0006FD003F0FD03012B00F08680464B93F8B5
:101BC000443023B9454B93F84430002B7ED0FFF7C7
:101BD00049FF00287CD14248424A037812781343D7
:101BE00078D1FCF7F7FC0446002853D13E4890F822
:101BF00060305A1E53425341B3742146F9F70EF92F
:101C00000123F7183A46D82196F8008037483370F8
